:020000040800F2
:10000000000002201125010891900008939000083B
:100010009590000897900008999000080000000053
:100020000000000000000000000000009B9000089D
:100030009D900008000000009F900008A19000081B
:1000400055250108552501085525010855250108A4
:100050005525010855250108552501085525010894
:10006000552501085525010855250108C1750008C9
:100070005525010855250108552501085525010874
:100080005525010855250108552501085525010864
:10009000552501085525010855250108C19200087C
:1000A0005525010855250108552501085525010844
:1000B0009D92000855250108552501085525010880
:1000C0005525010855250108552501085525010824
:1000D0005525010855250108D59300085525010827
:1000E0005525010855250108A5900008552501084A
:1000F00055250108552501085525010855250108F4
:1001000055250108552501085525010855250108E3
:1001100055250108552501085525010855250108D3
:1001200055250108552501085525010855250108C3
:1001300055250108552501085525010855250108B3
:10014000552501085525010855250108D5900008B9
:100150005525010855250108552501085525010893
:100160005525010855250108552501085525010883
:100170005525010855250108552501085525010873
:08018000552501085525010871
:10018800C4E7050800000020B00D0020B00D0020D5
:10019800403F002008B5074B186808F017FF0DF01E
:1001A8009BF9054B054806221A70BDE8084001F086
:1001B8009EBA00BFAC280020342800200C11002073
:1001C80008B5034801F093FA024B00221A7008BDE3
:1001D800041A00203428002008B5054B012200200D
:1001E8001A7005F06FFC0348BDE8084001F07FBABB
:1001F800C42E0020D01600202DE9F041144C2046D2
:1002080003F0BFFD00201349134A03F071FB1349A3
:10021800134A0746002003F06BFB1249124A0646B0
:10022800002003F065FBD22105463A4623460A2002
:1002380003F076FCD22132462346FA2003F070FC04
:100248005A20D2212A462346BDE8F04103F068BC73
:10025800E414002096D40508C90100089FD40508B5
:10026800E1010008A7D405089D01000808B5054B61
:10027800012200201A7005F025FC0348BDE808405B
:1002880001F035BAC42E0020D016002008B5034866
:1002980001F02DFA024B00221A7008BD041A002042
:1002A8003428002008B5054B07221A700DF014F900
:1002B8000348BDE8084001F01ABA00BF34280020FE
:1002C800E41400202DE9F041144C204603F059FDB8
:1002D80000201349134A03F00BFB1349134A07463E
:1002E800002003F005FB1249124A0646002003F0DD
:1002F800FFFAD22105463A4623460A2003F010FCAD
:10030800D221324623465A2003F00AFCAA20D221E1
:100318002A462346BDE8F04103F002BC0C11002038
:1003280096D4050895020008B0D40508AD02000867
:10033800B9D4050875020008014801F0D8B900BF12
:10034800F812002010B5094C204603F01AFD0020D1
:100358000749084A03F0CCFAD221024623464FF453
:100368008270BDE8104003F0DBBB00BF1818002006
:10037800C2D405084103000870B50C4C0C4D206828
:100388004FF6E076314602F0F7FD2068294602F084
:10039800A1FD6068314602F0EFFD6068294602F071
:1003A80099FDBDE8704003F025BF00BFB00D0020E7
:1003B8009FDA050838B52B4CFFF7DEFF002005F063
:1003C80081FB237A23B90A203221274A05F088FCC9
:1003D800637A23B90A206421244A05F081FC214C60
:1003E800A37A23B90A209621214A05F079FCA37A39
:1003F8001C4DFBB16B7AEBB12B7ADBB100232B726E
:100408006B72AB721B4B286801221A704FF6E071B1
:1004180002F0B2FD2868184902F05CFD68681749C7
:1004280002F058FD0BF0C3F803F0E4FE144803F0A3
:1004380025FF0DE00B4C4FF47841206802F09CFD3D
:100448002068104902F046FD60680F4902F042FD3D
:10045800FFF792FF00200BF06DF80C48BDE838401C
:1004680001F045B9B00D0020C9D40508D7D4050856
:10047800E6D4050834280020F4D40508A0DA0508D5
:100488008096980008D50508A2DA0508041A002005
:1004980008B500200BF04EF80248BDE8084001F00E
:1004A80026B900BF041A002038B5FFF765FF0DF024
:1004B8002BF83C213F220023DF2005F0F3FB4FF40B
:1004C80080600DF085FD124C3E223C21DF20002388
:1004D80005F0E8FB012323720E4B4FF6E075186810
:1004E80008F074FD2068294602F046FD20680A4994
:1004F80002F0F0FC6068294602F03EFD606807499A
:1005080002F0E8FC03F076FE054B00221A7038BDB5
:10051800B00D0020AC2800201AD505082DD50508F7
:100528003428002038B5FFF727FF0CF0EDFF6E21C7
:100538003F220023DF2005F0B5FB4FF486400DF085
:1005480047FD124C3E226E21DF20002305F0AAFB56
:10055800012363720E4B4FF6E075186808F036FDFC
:100568002068294602F008FD20680A4902F0B2FC1A
:100578006068294602F000FD6068074902F0AAFC9D
:1005880003F038FE054B00221A7038BDB00D00206C
:10059800AC28002040D5050851D50508342800208E
:1005A80010B5FFF7E9FE0CF0AFFFA0213F220023B2
:1005B800DF2005F077FB4FF402400DF009FD114CE8
:1005C8003E22A021DF20002305F06CFB0123A3724B
:1005D8000D4B186808F0FAFC20684FF6E07102F03D
:1005E800CBFC2068094902F075FC6068084902F0F4
:1005F80071FC03F0FFFD64200AF074FE054B002235
:100608001A7010BDB00D0020AC28002062D5050876
:10061800A0DA0508342800202DE9F74F3A4D3B4E63
:100628000024284603F0ADFB224623464FF6FF710F
:1006380037480094019402F063FC4FF6E0780427F1
:10064800F06041462246234632480097019402F062
:1006580057FC23463060414622462F4800970194B4
:1006680002F04EFC2D4970602D4A204603F040F9F7
:100678002C492D4A0746204603F03AF92B492C4AC3
:100688008046204603F034F92A492B4A8146204601
:1006980003F02EF929492A4A8346204603F028F90F
:1006A80021468246F2682B46204603F039FA5A2141
:1006B80032682B460A2003F033FA6E2172682B4603
:1006C8000A2003F02DFA9B213A462B46FA2003F024
:1006D80027FA692142462B46FA2003F021FA3721EE
:1006E8004A462B46FA2003F01BFAC82152462B46ED
:1006F800AA2003F015FAF020C8215A462B4603B069
:10070800BDE8F04F03F00CBA88150020B00D0020AA
:1007180076D505087ED5050891D50508A0D5050824
:10072800A9050008A8D505082D05000898D50508CD
:10073800B1040008B0D5050899040008B7D5050824
:10074800BD03000838B50C4C4FF6E0752068294603
:1007580002F012FC2068094902F0BCFB60682946D7
:1007680002F00AFC6068064902F0B4FB03F042FD9F
:10077800BDE8384003F03EBDB00D00207ED5050829
:10078800BED5050870B52DED028B9FED248A88B083
:100798000A26F0EE488A03E0B0EE608AF0EE418A5D
:1007A8000CF017F98DED000ACDED010A9DE8030064
:1007B80004AB83E80300F0EE680AB0EE480A9DED4A
:1007C800041ADDED051A8DED028ACDED038A0BF0D2
:1007D800BBFECDED010A8DED000A9DE8030002ADD8
:1007E80085E80300013E6C46DDED020A9DED031A23
:1007F800D2D19FED0B0A0CF0E3F88DED000ACDED98
:10080800010A9DE8030085E80300DDED030A9DED7C
:10081800020A08B0BDEC028B70BD00BF00000000EA
:10082800CDCCCC3D2DE9F74F564D574CDFF86491B0
:10083800DFF864814FF6E07005F018F9286810F0C9
:100848006BFD064668680F4610F066FD3246CDE936
:1008580000013B464946204615F06CFB2246002322
:100868000520372105F03CFA2869484F484E10F01A
:1008780053FD824668698B4610F04EFD5246CDE91D
:1008880000015B463946204615F054FB22460023FA
:100898000520692105F024FA286B10F03DFD8246F9
:1008A800686B8B4610F038FD5246CDE900015B4677
:1008B8004146204615F03EFB002305209B21224699
:1008C80005F00EFA31462A6C204615F033FB224615
:1008D80000239B21A22005F003FA4FF4FC6005F0E9
:1008E800C5F8A86810F018FD8246E8688B4610F035
:1008F80013FD5246CDE900015B464946204615F0F6
:1009080019FB224605205021002305F0E9F9A869C2
:1009180010F002FD8246E8698B4610F0FDFC524655
:10092800CDE900015B463946204615F003FB224617
:1009380000230520822105F0D3F9A86B10F0ECFC08
:100948008246E86B8B4610F0E7FC5246CDE9000181
:100958005B464146204615F0EDFA00230520B421F8
:10096800224605F0BDF931466A6C204615F0E2FAD8
:10097800A220B4212246002303B0BDE8F04F05F0C1
:10098800AFB900BFCC3C0020C00D0020E3D505085E
:1009980006D60508D1D50508F5D5050808B50020FF
:1009A80005F090F80A4B1B780B2B0BD8DFE803F007
:1009B8000A0A0A0A0A0A08060A0A0A0A054802E08E
:1009C800054800E00548BDE8084000F090BE00BFBB
:1009D80034280020E41400200C110020041A002000
:1009E8002DE9F14F2D4C204603F0CBF900202C497E
:1009F8002C4A02F07DFF2C492C4A8146002002F047
:100A080077FF2B492B4A0746002002F071FF2A493D
:100A18002A4A0646002002F06BFF2949294A054662
:100A2800002002F065FF2849284A8046002002F08D
:100A38005FFF2749274A8246002002F059FFD2214A
:100A480083464A462346E62003F06AF828203A46B9
:100A58002346014603F064F84621324623462820FF
:100A680003F05EF864212A462346282003F058F84C
:100A7800822142462346282003F052F85246234654
:100A88002820A02103F04CF828205A46BE212346EE
:100A980001B0BDE8F04F03F043B800BFD016002006
:100AA8000BD60508A509000814D605087512000814
:100AB8001FD605085112000829D605082D1200086E
:100AC80034D60508091200083FD60508E5110008C4
:100AD80049D60508C1110008023810B50A2800F2E5
:100AE8003C83DFE810F00B000F006400D2008A019D
:100AF8002001170231023A03A102F502BDE81040B5
:100B08000AF0C2BD00204FF6E0710AF01BFF632017
:100B18004FF6E0710AF016FFB3204FF4F0610AF0C7
:100B280011FFC7204FF6E0710AF00CFF4FF6FF7077
:100B380004F09CFFDC2100237D20D34A05F0D0F887
:100B48004EF29C7004F092FF052001210023CF4A49
:100B580005F0C6F8052052210023CD4A05F0C0F85B
:100B6800B62100230520CB4A05F0BAF84FF4F0600F
:100B780004F07CFF0121002340F21310C34A05F062
:100B8800AFF8002340F213105221C24A05F0A8F82A
:100B9800B621C14A40F21310002305F0A1F84EF225
:100BA8009C7004F063FF0520A221BC4A68E0002085
:100BB8004FF6E0710AF0C6FE31204FF6E0710AF0F8
:100BC800C1FE63204FF6E0710AF0BCFE95204FF697
:100BD800E0710AF0B7FEC7204FF6E0710AF0B2FEE6
:100BE8004EF29C7004F042FF052001210023AC4A1C
:100BF80005F076F8052020210023AA4A05F070F8B0
:100C0800052052210023A84A05F06AF8052084210E
:100C18000023A64A05F064F8B62105209D4A002362
:100C280005F05EF84FF4F06004F020FF012140F277
:100C3800131000239A4A05F053F840F213102021AC
:100C48009B4A002305F04CF840F213105221914AB8
:100C5800002305F045F840F213108421954A00233B
:100C680005F03EF8B621944A40F21310002305F02F
:100C780037F84FF6FF7004F0F9FE904A7D20DC212A
:100C88000023BDE8104005F02BB800204FF6E071B6
:100C98000AF058FE27204FF6E0710AF053FE4F2065
:100CA8004FF6E0710AF04EFE77204FF6E0710AF039
:100CB80049FE9F204FF6E0710AF044FEC7204FF628
:100CC800E0710AF03FFE4EF29C7004F0CFFE052062
:100CD800012100236F4A05F003F80520162100239F
:100CE800774A04F0FDFF05203E210023754A04F0F1
:100CF800F7FF052066210023734A04F0F1FF8E21D7
:100D080000230520714A04F0EBFF0520704AB62144
:100D1800002304F0E5FF4FF6FF7004F0A7FE7D20E6
:100D2800DC216C4AACE700204FF6E0710AF00AFEBD
:100D380031204FF6E0710AF005FE63204FF6E071AE
:100D48000AF000FE95204FF6E0710AF0FBFDC7207F
:100D58004FF6E0710AF0F6FD4EF29C7004F086FE44
:100D68000520012100235C4A04F0BAFF0520202158
:100D780000235A4A04F0B4FF052052210023584AA0
:100D880004F0AEFF052084210023564A04F0A8FF92
:100D9800B62105203F4A002304F0A2FF4FF4F0607B
:100DA80004F064FE012140F2131000234E4A04F0BF
:100DB80097FF40F2131020214C4A002304F090FFC3
:100DC80040F213105221334A002304F089FF40F205
:100DD80013108421464A002304F082FFB621454AB5
:100DE80040F21310002304F07BFF4FF6FF7004F06D
:100DF8003DFE7D20DC21404A42E700204FF6E071AD
:100E08000AF0A0FD31204FF6E0710AF09BFD632047
:100E18004FF6E0710AF096FD95204FF6E0710AF062
:100E280091FDC7204FF4FC610AF08CFD4EF29C70D6
:100E380004F01CFE052001210023304A04F050FF75
:100E48000520202100232E4A04F04AFF05205221C4
:100E580000232C4A04F044FF8421002305202A4A59
:100E680004F03EFF4FF4F06004F000FEB6210520C8
:100E7800264A002304F034FF4FF6FF7004F0F6FD15
:100E88008720234ADC21FBE61FD6050853D6050830
:100E98004ED6050820DC050852D6050880D6050878
:100EA8006CD6050857D6050867D605085CD6050828
:100EB80061D6050866D605086BD6050829D6050843
:100EC8006FD6050873D6050877D605087BD60508BA
:100ED8007FD6050883D605088FD6050893D605085A
:100EE80097D605089AD60508A3D605089FD60508FB
:100EF8009ED60508A2D60508A7D60508B2D60508C5
:100F080078D6050870D60508C2D6050837DD050865
:100F180049D6050800204FF6E0710AF013FD63205A
:100F28004FF4FC610AF00EFD4FF6E071C7200AF09D
:100F380009FD4FF6FF7004F099FD002004F098FEBB
:100F4800A520D721854A9BE6042004F091FE0020C5
:100F58004FF6E0710AF0F6FC31204FF6E0710AF026
:100F6800F1FC63204FF6E0710AF0ECFC95204FF697
:100F7800E0710AF0E7FCC7204FF6E0710AF0E2FCE6
:100F88004EF29C7004F072FD052001210023744A82
:100F980004F0A6FE052020210023724A04F0A0FEDA
:100FA800052052210023704A04F09AFE052084216E
:100FB80000236E4A04F094FE0520B6216C4A0023F3
:100FC80004F08EFE4FF6E07004F050FD40F20B1076
:100FD8000121684A002304F083FE40F22B102021EF
:100FE800654A002304F07CFE40F223105221634A34
:100FF800002304F075FE40F21B108421604A002390
:1010080004F06EFEB6215F4A002340F2131004F08C
:1010180067FE4FF6FF7004F029FD002004F028FE5B
:101028006E20D221584A90E0042004F021FE0020CE
:101038004FF6E0710AF086FC27204FF6E0710AF0BF
:1010480081FC4F204FF6E0710AF07CFC77204FF6C8
:10105800E0710AF077FC9F204FF6E0710AF072FC0D
:10106800C7204FF6E0710AF06DFC4EF29C7004F058
:10107800FDFC052001210023444A04F031FE05202F
:1010880016210023424A04F02BFE05203E210023AE
:10109800404A04F025FE052066213F4A002304F05B
:1010A8001FFE05208E213D4A002304F019FEB621BB
:1010B8003B4A0023052004F013FE4FF6FF7004F0AE
:1010C800D5FC002004F0D4FD6420D221354A3CE050
:1010D800042004F0CDFD00204FF6E0710AF032FC48
:1010E80043204FF6E0710AF02DFC85204FF6E071A1
:1010F8000AF028FC4FF6E071C7200AF023FC4EF2F4
:101108009C7004F0B3FC05200121274A002304F059
:10111800E7FD05204521254A002304F0E1FD0520CF
:1011280087211F4A002304F0DBFDB621204A002353
:10113800052004F0D5FD4FF6FF7004F097FC002061
:1011480004F096FD1B4A7D20D221002304F0C8FD3F
:101158000420BDE8104004F08BBD10BDB8DA0508C6
:10116800B6D60508C2D60508C1D60508C4D60508EE
:10117800C8D60508CDD605086CD60508D4D6050806
:10118800D8D60508DDD60508E3D60508E9D605084A
:101198009FD60508A4D60508EED60508F1D6050899
:1011A80080D60508F4D60508FDD60508B2D6050888
:1011B80020DC050894DB050810B5064C0648062314
:1011C800237000F094FA2078FFF786FCBDE8104001
:1011D8000CF0CCBEC42E00206019002010B5064CBF
:1011E80006480723237000F082FA2078FFF774FC82
:1011F800BDE810400CF0BABEC42E002060190020D3
:1012080010B5064C06480523237000F070FA2078C4
:10121800FFF762FCBDE810400CF0A8BEC42E002009
:101228006019002010B5064C06480423237000F00E
:101238005EFA2078FFF750FCBDE810400CF096BE2F
:10124800C42E00206019002010B5064C0648032360
:10125800237000F04CFA2078FFF73EFCBDE8104000
:101268000CF084BEC42E00206019002010B5064C76
:1012780006480223237000F03AFA2078FFF72CFC86
:10128800BDE810400CF072BEC42E0020601900208A
:1012980070477047704770470E4A002310B51370A7
:1012A8000D4A0E4C13700AF0ADFB05F0A5FB0AF0D1
:1012B80084F90AF0A1FB20684FF6E07101F05CFEAA
:1012C8002068074901F006FE02F094FFBDE81040CF
:1012D80002F090BF380F0020DF0E0020DC0D002048
:1012E80001D705080E4A012310B513700D4A0024D2
:1012F80014700D4A204613700AF01CF9204604F0B9
:10130800E1FB0A4B03221A700AF056FC0BF015F9A0
:10131800074B08481C70BDE8104000F0E8B900BF52
:10132800C42E0020DF0E0020DD0E0020342800200F
:10133800A43A00209C13002038B50D4B0D4D002415
:101348001C700D4B28681C700C4B4FF6E0711C701C
:1013580001F012FE28680A4901F0BCFD02F04AFFBC
:10136800204604F0AFFB0748BDE8384000F0BFB99D
:10137800380F0020DC0D0020DF0E0020342800206C
:10138800A4DA0508041A002007B50E4B0E481A788F
:10139800D2F1010238BF00221A700C4B05221A70D4
:1013A80000F0A5F9022201238DE80C00B02060218D
:1013B800102232230CF062FF03B05DF804EB02F058
:1013C80019BF00BF380F0020541200203428002015
:1013D8002E4A002310B513702D4A13700CF0BEFB73
:1013E8000446002842D02B4C4FF6E071206801F0EB
:1013F800C3FD2068284901F06DFD60684FF6E07173
:1014080001F0BAFD6068254901F064FDA0684FF657
:10141800E07101F0B1FDA068214901F05BFD02F027
:10142800E9FE4FF47A6009F05DFF20684FF6E0713D
:1014380001F0A2FD20681B4901F04CFD60684FF6E1
:10144800E07101F099FD6068164901F043FDA0685C
:101458004FF6E07101F090FDA068124901F03AFDE5
:1014680002F0C8FEBDE8104002F0C4BE0CF034F82B
:10147800204604F027FB0C4B0C4804221A7000F09D
:1014880036F9BDE81040FFF75DB900BF380F0020FE
:10149800DF0E0020DC0D002011D7050825D7050830
:1014A80035D70508A3DA0508342800208815002058
:1014B8002DE9F04F634DDFF8E89187B000244FF62F
:1014C800FF78284602F05DFC4146224623465E48E6
:1014D8000094019401F014FD4FF6E0760427039080
:1014E80031462246234659480097019401F008FDE9
:1014F80031462246234656480097019401F000FDE4
:1015080041462246234648460097019401F0F8FCDC
:10151800504E414630602246234648460097019483
:1015280001F0EEFC2346706041462246484600978B
:10153800019401F0E5FC4849B060484A204602F0B1
:10154800D7F94749474A0746204602F0D1F94649A4
:10155800464A8046204602F0CBF94549454A81462D
:10156800204602F0C5F94449444A8246204602F022
:10157800BFF943490490434A204602F0B9F920468E
:101588004149424A02F0B4F94149424A8346204659
:1015980002F0AEF94049414A84462046CDF808C0D9
:1015A80002F0A6F921460590039A2B46204602F040
:1015B800B7FA052132682B46A52002F0B1FA692155
:1015C80072682B46782002F0ABFA7D21B2682B4670
:1015D800782002F0A5FA1E213A462B46052002F093
:1015E8009FFA42462B464121052002F099FA6421D0
:1015F8004A462B46052002F093FA872152462B468D
:10160800052002F08DFAD2215A462B46602002F0BE
:1016180087FADDF808C0D22162462B46052002F081
:101628007FFAD221059A2B46B02002F079FA049A63
:101638004FF48070D2212B4607B0BDE8F04F02F07E
:101648006FBA00BF2C16002045D705084FD70508EC
:101658005CD70508DC0D002067D70508991200083B
:101668006FD705089B12000877D705089D12000858
:101678007FD705089F12000887D70508411300087F
:101688008FD70508A112000897D70508D9130008B5
:101698009FD7050891130008A8D70508ED12000880
:1016A800A0DA050808B500F023FEFEF7A5FD00F056
:1016B8004FF800F06FF8FEF7AFFFFEF703FEFFF7F5
:1016C8008FF901F0E9FAFFF7F3FE00F0D5FFFEF716
:1016D80039FE01F03BF901F0DBF900F06DFB00F099
:1016E80081FD00F061FABDE8084000F02FBB10B59D
:1016F800044628B90F48104A104B532102F0A2FFA4
:101708000F4B1868844213D010B1C3690021984761
:10171800002004F0D7F9002004F0BEF94FF6FF705E
:1017280004F0A4F9E369204601219847044B1C60A2
:1017380010BD00BFB0D7050824150408CCD705088C
:10174800E80D00200048D2E7041A00200CF0CAB9BE
:1017580010B5084C204602F014FB00200649074A41
:1017680002F0C6F8D22102462346FA20BDE810400E
:1017780002F0D6B9C40F0020EAD7050855170008AB
:10178800024B034801221A70FFF7B1BF342800202A
:101798002C1600202DE9F743374D384F384E0024DA
:1017A800284602F0EEFA2246234647F6FF713548EE
:1017B8000094019401F0A4FB4FF6FF78814641465E
:1017C8002246234638460094019401F099FB41468D
:1017D80030602246234638460094019401F090FB7D
:1017E800414670602246234638460094019401F031
:1017F80087FB2346B0604146224638460094019450
:1018080001F07EFB2049F060204A204602F070F883
:101818001F49204A0746204602F06AF821468046BA
:101828004A462B46204602F07BF93C2132682B467B
:10183800192002F075F95A2172682B46192002F016
:101848006FF97821B2682B46192002F069F99621C0
:10185800F2682B46192002F063F9D2213A462B464A
:10186800EC2002F05DF99C20D22142462B4603B0C1
:10187800BDE8F04302F054B99C130020A0DA050833
:10188800EC0D0020DCD70508E9D705088917000802
:10189800F2D705085D1A000870B5474E474C3278F4
:1018A80047492DED028B142592B005FB02420C32FC
:1018B8000FA814F03FFB33780D2B05FB03F504EB61
:1018C800050332D8D3ED016A9B6807EE103A6359D5
:1018D800B8EEE68A06EE903ADFED3A7AF8EEC78A75
:1018E800B8EEE67A88EE278AC8EEA78AC7EE277A86
:1018F80017EE900A0FF010FD02460B466846324973
:1019080014F018FB18EE100A0FF006FD02460B46FD
:1019180005A82E4914F00EFB18EE900A0FF0FCFCF7
:1019280002460B460AA82A4929E093ED017A9B68EA
:1019380007EE903A635906EE903AF8EEE78AF8EE29
:10194800E67AB8EEC78A17EE900A0FF0E5FC024671
:101958000B4668461F4914F0EDFA18EE100A0FF00E
:10196800DBFC02460B4605A81B4914F0E3FA18EE07
:10197800900A0FF0D1FC0B46184902460AA8184CE9
:1019880014F0D8FA2068174901F0A4FA20680FA9C2
:1019980001F0A0FA6068694601F09CFAA06805A900
:1019A80001F098FAE0680AA901F094FA02F022FC22
:1019B80012B0BDEC028B70BDB228002000000020E0
:1019C800FBD7050800007A4406D8050817D805088B
:1019D80028D8050839D805084AD805085BD8050865
:1019E800EC0D0020A9DA050808B5124B124A1B783D
:1019F8000D2B8CBF00210121117014225A430F496D
:101A080088588B184FF47A720D495043086059680A
:101A18004A430C490A609A680B4B1A6009F048FD62
:101A280009F0EAFF094B0A4800221A70BDE808408D
:101A3800FFF75DBEB2280020800F002000000020C4
:101A4800B4280020D42E0020A82E002034280020FE
:101A5800041A0020C8E700BF4FF6FF7070474FF622
:101A6800FF7070471FB5002947D04FF2DE7004F0B1
:101A780029F8002004F0FCF80F2003F0F7FF1F4CB2
:101A88001F4A412101230A2004F02AF9042004F006
:101A9800EFF8236828209621042B24DC0123194A17
:101AA80004F01EF903A90DF10E02206804F0A0FB52
:101AB8000F2003F0DBFFBDF80C00BDF80E10143842
:101AC8000F242822002380B2009403F0FFFFBDF802
:101AD8000E10BDF80C000094143989B22822012395
:101AE80003F0F4FF09E0084A012304F0F9F81E2086
:101AF800A521064A012304F0F3F81FBDFC0D0020C0
:101B08006CD805087FD805089BD80508B1D8050802
:101B180037B51E4C2368042B05462BDC01A80DF1B4
:101B2800060104F063FBBDF80630BDF8042018492F
:101B380004200CF0A5FC2368002B04DA1548164A8B
:101B4800164B592105E0042B05DD1248124A144BA7
:101B58005A2102F077FD04EB8302BDF8041001332B
:101B68009180BDF806102360052BD18008D1201D77
:101B780004F0BEFB00230B482360FFF7B8FD03E029
:101B880028460121FFF76EFF3EBD00BFFC0D002077
:101B9800C8D805080DD90508361504082FD9050831
:101BA80046D905087417002037B50B4C204602F0BB
:101BB800E8F80A4B0A49009300250120094A0A4B14
:101BC800019501F086FF294602462346284603B0C0
:101BD800BDE8304001F0A4BF401400206D1A000891
:101BE800611A0008671A0008191B00084FF6FF70F1
:101BF80070474FF6FF70704730B54FF6E07087B00A
:101C080003F060FF002004F033F80F2003F02EFFEC
:101C180000212C4A2C4C01230A2004F061F80020F2
:101C280003F024FF042004F023F80A201921274A8E
:101C3800012304F055F82521254A01230A2004F040
:101C48004FF81F2003F012FF01230A203721214AF1
:101C580004F046F82378002B31D001231E2096216A
:101C68001D4A04F03DF862881C4902A814F062F984
:101C780001231E20A22102AA04F032F8A2881849E2
:101C880002A814F057F9AE2102AA01231E2004F07D
:101C980027F80F2003F0EAFE6088A188143880B284
:101CA8000F2528220023009503F010FFA1886088E3
:101CB8000095143989B22822012303F007FF07B0E1
:101CC80030BD00BF74D90508140E002086D9050858
:101CD800A6D90508C6D90508E9D90508FBD9050814
:101CE80008DA050801B187E7704713B50DF1060159
:101CF80001A804F02FFA144B01221A705988BDF874
:101D08000420891A0E311C2919460AD89C88BDF866
:101D18000600201A0E301C2803D8996801319960F2
:101D280001E000238B60084B9968012905DD00223A
:101D38009A601A70FFF706FD05E05A80BDF8062084
:101D48009A80FFF759FF1CBD140E002037B50B4CC5
:101D5800204602F016F80A4B0A4900930025012094
:101D6800094A0A4B019501F0B4FE2946024623466A
:101D7800284603B0BDE8304001F0D2BE74170020F9
:101D8800ED1C0008F51B0008FB1B0008F31C0008ED
:101D980008B5064B00221A70054B186813F060FD51
:101DA8000448BDE80840FFF7A2BC00BF3428002063
:101DB80098380020041A00202DE9F04F514D524E5A
:101DC80085B00024284601F0DCFF2246234647F66A
:101DD800FF714E480094019401F092F84FF6FF7796
:101DE800039039462246234649480094019401F05D
:101DF80087F83946306022462346464800940194C5
:101E080001F07EF84FF001087060224623464FF635
:101E1800E0714148CDF80080019401F071F8234643
:101E2800B060394622463D48CDF80080019401F063
:101E380067F83B49F0603B4A204601F059FD3A49B2
:101E48003A4A0746204601F053FD3949394A804647
:101E5800204601F04DFD3849384A8146204601F0B8
:101E680047FD3749374A8246204601F041FD364949
:101E7800364A8346204601F03BFD21468446039AB4
:101E8800CDF808C02B46204601F04AFE3C213268B6
:101E98002B46142001F044FE3C2172682B46EC20AE
:101EA80001F03EFEB421B2682B460F2001F038FE47
:101EB800D2213A462B46E62001F032FE6421424602
:101EC8002B46052001F02CFE4A462B46052087218B
:101ED80001F026FE52462B460520D22101F020FEB5
:101EE800D2215A462B46502001F01AFEDDF808C0D0
:101EF8009B20D22162462B4605B0BDE8F04F01F089
:101F08000FBE00BF68100020200E002015DA05085B
:101F18001FDA050828DA05089EDA0508A0DA050898
:101F2800E9D70508991D000898D50508811F0008FC
:101F3800A8D50508812000082BDA050889210008A2
:101F480033DA0508452100083BDA050801210008B5
:101F580008B50BF0D9FA4FF441400CF039F8044BAE
:101F6800186807F033F8034B09221A7008BD00BF40
:101F7800AC2800203428002010B50C4CFFF7E8FFEF
:101F88000B4A0023B420052103F0AAFEA0684FF6EF
:101F9800E07100F0F1FFA068064900F09BFF0BF02C
:101FA800B3FABDE8104002F025B900BF200E0020AA
:101FB800A6DA050843DA0508264B2DE9F743188801
:101FC800C00013F045FC054628B90520B421224A73
:101FD8002B4603F085FE214BDFF878801D60002436
:101FE8000BF092FA26461E4FDFF8889023E009F09E
:101FF800B7F83B68D9F8000045F8083C7B6845F815
:10200800043C184B1B68C01806F0E0FF164B186814
:1020180009F068F9B8F8000094FBF0F080B24FF4CA
:10202800FC63009328210246322303F0ABFC04F53D
:102038009E7401360334B8F800300835B342D6DA56
:102048000A4B186806F0C2FF094B09221A70BDE84E
:10205800FE8300BF9C3C00205CDA0508983800200D
:10206800643A00203028002060280020AC28002096
:1020780034280020A038002010B5094CFFF79CFF39
:10208800A0684FF6E07100F077FFA068054900F0FE
:1020980021FF0BF039FABDE8104002F0ABB800BFE1
:1020A800200E00206ADA050810B5074C4FF6E071DB
:1020B800A06800F061FFA068044900F00BFFBDE8CC
:1020C800104002F097B800BF200E002084DA0508FF
:1020D80010B5074C4FF6E071A06800F04DFFA068FE
:1020E800044900F0F7FEBDE8104002F083B800BFD5
:1020F800200E00209ADA050810B50C4C0B2323702B
:102108000B4B01221A70002002F0AAFF0948FFF7C2
:10211800EEFA2078FEF7E0FC074B032093ED000A67
:102128000BF001FABDE81040D2E700BFC42E002032
:10213800E00E002060190020D403002038B50C4DB3
:102148000C232B700B4B01241C70002002F088FF1D
:102158000948FFF7CCFA2878FEF7BEFC074B204663
:1021680093ED000A0BF0DFF9BDE83840B0E700BF97
:10217800C42E0020E00E002060190020D4030020A7
:1021880010B50C4C092323700B4B01221A70002048
:1021980002F066FF0948FFF7AAFA2078FEF79CFCD0
:1021A800074B022093ED000A0BF0BDF9BDE8104083
:1021B8008EE700BFC42E0020E00E0020601900202A
:1021C800D40300200BF050BD034A044800231370C9
:1021D800034A1370FFF78BBAA43A0020041A0020B0
:1021E800342800202DE9F743384D394EDFF8FC80BC
:1021F8000024284601F0C5FD2246234647F6FF7114
:1022080034480094019400F07BFE4FF6FF77814636
:1022180039462246234630480094019400F070FE67
:10222800394630602246234640460094019400F027
:1022380067FE394670602246234640460094019462
:1022480000F05EFE2346B0603946224640460094C0
:10225800019400F055FE2149F060214A204601F022
:1022680047FB2049204A0746204601F041FB21460A
:1022780080464A462B46204601F052FC3C213268F3
:102288002B46282001F04CFC5A2172682B46192055
:1022980001F046FC7821B2682B46192001F040FC79
:1022A8009621F2682B46192001F03AFCD2213A46D1
:1022B8002B46EC2001F034FC0520D22142462B4667
:1022C80003B0BDE8F04301F02BBC00BFB011002003
:1022D800300E0020B4DA0508BCDA0508E9D705088D
:1022E800D1210008C7DA0508CD210008A0DA0508C1
:1022F80010B50B4C204601F044FD00200146224653
:1023080000F05EFE00200749074A01F0F1FAD221E9
:10231800024623464FF48270BDE8104001F000BC2D
:1023280060190020CFDA05085923000870B5C924C0
:102338000AE0A8B200223146013502F021FDF02D55
:10234800F7D10134EF2C02D00025A6B2F1E770BD19
:1023580010B51A4C2378092B08D1194A0023137099
:10236800184A1370FFF7E2FF174823E00A2B0ED133
:10237800164B186813F074FA154A00231370114AA3
:102388001370144A1370FFF7D1FF134812E00020AE
:1023980002F066FE114A00231360114A13800D4BA8
:1023A80002221A700F4B186806F010FE22780E4BA6
:1023B8000E481A70BDE81040FFF799B9342800207C
:1023C800E00E0020DF0E0020681000209838002062
:1023D800E10E0020A43A0020B0110020280F0020B0
:1023E800360F0020AC28002058280020F8120020C2
:1023F800034B01224FF4FC601A7003F037BB00BF97
:10240800DF0E002007B50A4A0023137004228DE866
:102418000C00C6201022232356210BF02FFF054B5A
:1024280005480A221A7003B05DF804EBFFF75FB99C
:10243800DF0E002034280020B011002007B50A4A1A
:102448000023137004228DE80C0097201022232308
:1024580056210BF013FF054B054809221A7003B0EB
:102468005DF804EBFFF743B9DF0E002034280020A5
:102478006810002007B50B4B00221A7008220323AE
:102488008DE80C004920102223233D210BF0F6FE95
:10249800054B064801221A7003B05DF804EBFFF7FC
:1024A80026B900BFDF0E0020342800202C1600209B
:1024B80008B50A4B00201870094B1870094B082200
:1024C8001A70094B187003F0FDFA084B08480122EE
:1024D8001A70BDE80840FFF70AB900BF380F00209E
:1024E800DF0E002034280020C42E0020B038002041
:1024F800C40F002070B51F4C1F4E20684FF6E075C2
:10250800294600F039FD20681C4900F0E3FC6068AA
:10251800294600F031FD6068194900F0DBFCA0682D
:10252800294600F029FDA068164900F0D3FC01F007
:1025380061FE4FF47A6008F0D5FE2068294600F065
:102548001BFD2068314600F0C5FC6068294600F094
:1025580013FD6068314600F0BDFCA068294600F014
:102568000BFDA068314600F0B5FCBDE8704001F0F5
:1025780041BE00BF400E0020A3DA050811D70508A8
:1025880025D7050835D705080C4B10B500241C7055
:102598000B4B01221A70204608F0CCFF204603F0AE
:1025A80091FA084B0B221A7009F006FB09F0C5FFD7
:1025B8000548BDE81040FFF79AB800BFDF0E0020BD
:1025C800C42E002034280020D01600200F4A0023F3
:1025D80010B513700E4A13700BF0C0FA044628B1F8
:1025E800FFF788FFBDE8104001F004BE03F06AFA67
:1025F80009F008FA074B1C70074B07221A7009F0FC
:10260800FBF90648BDE81040FFF771B8380F002005
:10261800DF0E0020C42E002034280020E4140020FF
:10262800104A002310B513700F4A13700BF096FA76
:10263800044628B1FFF75EFFBDE8104001F0DABD9F
:1026480003F040FA09F0DEF906F018FD074B1C709C
:10265800074B06221A7009F0CFF90648BDE810406A
:10266800FFF745B8380F0020DF0E0020C42E0020E9
:10267800342800200C1100202DE9F04F674DDFF8B9
:10268800F09189B000244FF6FF78284601F079FBD5
:1026980041462246234662480094019400F030FCEB
:1026A8004FF6E076042703903146224623465D48DC
:1026B8000097019400F024FC3146049022462346FA
:1026C80059480097019400F01BFC414605902246AA
:1026D800234648460097019400F012FC534E4146A9
:1026E80030602246234648460097019400F008FCD3
:1026F800234670604146224648460097019400F000
:10270800FFFB4B49B0604B4A204601F0F1F84A49BB
:102718004A4A0746204601F0EBF84949494A8046AB
:10272800204601F0E5F84849484A8146204601F02C
:10273800DFF84749474A8246204601F0D9F846491A
:10274800464A8346204601F0D3F84549454A84461F
:102758002046CDF808C001F0CBF843490690434A1B
:10276800204601F0C5F821460790039A2B462046DB
:1027780001F0D6F92146049A2B46C82001F0D0F979
:102788000A21059A2B46C82001F0CAF9552132685A
:102798002B46782001F0C4F9692172682B4678200D
:1027A80001F0BEF9B2682B4678207D2101F0B8F916
:1027B8003A462B460520282101F0B2F9D22142469B
:1027C8002B46052001F0ACF9D2214A462B4656206B
:1027D80001F0A6F9D22152462B46A62001F0A0F915
:1027E800B4215A462B46052001F09AF9DDF808C0B5
:1027F800B42162462B46562001F092F9B421069A7C
:102808002B46A62001F08CF9079AF620D2212B46F8
:1028180009B0BDE8F04F01F083B900BF041A0020E9
:10282800D4DA05084FD705085CD70508400E002004
:10283800DDDA05087D240008E5DA05089125000899
:10284800EEDA050829260008F7DA0508D525000874
:1028580000DB0508B924000809DB05084524000841
:1028680012DB05080D2400081BDB0508F923000806
:10287800A0DA050810B5064C4FF6FF71206800F085
:102888007BFB044B20681968BDE8104000F022BBB0
:102898004C0E00209402002008B5002003F012F925
:1028A800054B1868054B196800F014FB0448BDE88F
:1028B8000840FEF71CBF00BF4C0E0020900200200D
:1028C8002C1600200088A0F5C87080B2092808B529
:1028D80005D90848084A094B8C2101F0B3FE084B7A
:1028E8001880084BFF21197008F004FDBDE8084066
:1028F800C0E700BF22DB05084815040845DB0508CA
:10290800A81A0020AA1A00200088A0F5967080B2A4
:10291800092808B505D90848084A094B802101F05B
:1029280091FE084B1880084B0121197008F0E2FC51
:10293800BDE808409EE700BF22DB05085D150408D6
:1029480045DB0508A81A0020AA1A0020F7B50024BC
:102958003348344D01F015FA224623464FF6FF71ED
:1029680031480094019400F0CBFA0426224623460D
:1029780007464FF6FF712D480096019400F0C0FA03
:102988002346286022464FF6FF7128480096019496
:1029980000F0B6FA26496860264A204600F0A8FFEB
:1029A800214606463A4620461D4B01F0B9F82A68EA
:1029B8001B4B2046282101F0B3F83246AA20D22129
:1029C800174B01F0ADF80F254FF4967440F2351609
:1029D80020461949194A00F08BFF01340246782134
:1029E80028460F4BA4B2233501F09AF8B442ADB291
:1029F800EED10F254FF4C87440F2991620461049BD
:102A0800104A00F075FF013402469B212846044B0A
:102A1800A4B2233501F084F8B442ADB2EED1FEBDC4
:102A2800BC1800204C0E002076DB0508B1DA05083A
:102A380082DB0508A12800088BDB0508112900089E
:102A48008DDB0508CD28000808B5FFF713FF002027
:102A5800014608F04FFCBDE8084001F0CBBB00BFC1
:102A680007B5032308228DE80C00492010222323F0
:102A78003D210BF003FC044B044801221A7003B0FB
:102A88005DF804EBFEF733BE342800202C16002036
:102A98002DE9F743314E324F324D0024304601F0D4
:102AA80070F92246234647F6FF712F480094019497
:102AB80000F026FA4FF6FF78814641462246234623
:102AC80038460094019400F01BFA414628602246DB
:102AD800234638460094019400F012FA4146686093
:102AE8002246234638460094019400F009FA23460A
:102AF800A8604146224638460094019400F000FA46
:102B08001A49E8601A4A204600F0F2FE21460746B4
:102B18004A463346204601F003F83C212A683346EA
:102B2800192000F0FDFF5A216A683346192000F089
:102B3800F7FF7821AA683346192000F0F1FF9621A3
:102B4800EA683346192000F0EBFFEC20D2213A4620
:102B5800334603B0BDE8F04300F0E2BF5412002052
:102B6800A0DA0508540E00208FDB0508E9D7050810
:102B7800692A00081C4B1A781C4B10B51A7009F00A
:102B880021F81B4B1B4A00241C6002202346CA2143
:102B980003F0A6F8204608F0CDFC174B1C80174B15
:102BA8001C70174B1B78023B052B1CD8DFE803F081
:102BB80003070B13170FBDE81040FEF757BBBDE81E
:102BC8001040FEF741BBBDE81040FEF72BBBBDE847
:102BD8001040FEF703BBBDE81040FEF711BBBDE88F
:102BE8001040FEF7E9BA10BD58280020342800200C
:102BF800280F00209FDA0508AC380020A43A0020EE
:102C0800C42E002008B5084B186806F0DFF900202C
:102C180002F058FF08F0D0FF044B05480B221A7049
:102C2800BDE80840FEF763BDAC280020342800202A
:102C3800D0160020114B10B500241C70104B1868DA
:102C480006F0C4F9204602F03DFF0E4B1B780B2B13
:102C58000ED8DFE803F006060D0D0D0D0A080D0D60
:102C68000D06094802E0094800E00948FEF73FFD63
:102C7800084B1C70BDE8104008F09EBFC42E002011
:102C8800AC28002034280020041A0020E414002076
:102C98000C110020A43A00202DE9F041144C2046E4
:102CA80001F06FF800201349134A00F021FE134980
:102CB800134A0746002000F01BFE1249124A064636
:102CC800002000F015FED22105463A462346E620AC
:102CD80000F026FF4B2132462346642000F020FFF7
:102CE800642069212A462346BDE8F04100F018BF58
:102CF800F81200200BD605083D2C000897DB0508C4
:102D08000D2C0008A3DB05087D2B000808B508B1C9
:102D180043682BB90348044A044B9B2101F092FCF9
:102D2800586908BDB0DB050871150408D2DB050831
:102D380008B5FFF7EBFF8068123080B208BD08B510
:102D4800FFF7E4FF4068063080B208BD2DE9F84F70
:102D580004468846FFF7DAFF6689E589074606F1E3
:102D6800030905F10F0AB8F1000F1FD01F2002F068
:102D78007DFE2046FFF7DCFF83462046FFF7DFFF96
:102D8800294603465FFA8BF2F0B202F0AFFE042048
:102D980002F06EFF0B364FF6FF70033502F066FE49
:102DA800B0B2A9B23A68012302F09AFF3D69204601
:102DB80041464A465346A847BDE8F88F13B504462E
:102DC8000DF1060101A803F0C5F92046FFF79EFFA3
:102DD8006389BDF80410BDF80620C91AE389D21A20
:102DE8000339C3680F3A204698471CBDF7B5044617
:102DF80014200D4616461F4612F02AFD089BC76090
:102E08000361064B0649074A80E870000093019069
:102E1800054B002000F05DFEFEBD00BF552D0008EB
:102E2800472D0008392D0008C52D0008704708B542
:102E380008B143682BB90448044A054BAD2101F099
:102E480001FC586908BD00BFF1DB050889150408B5
:102E5800D2DB0508F8B505460E46FFF7E8FF836B99
:102E680004461BB128463146984700E018466F894A
:102E780094F83C30ED890EB9034310D0208E02F04F
:102E8800F5FD608E02F008FE94F8350002F0F0FEC1
:102E980094F8343038462946224602F021FF0023B0
:102EA80084F83C30F8BD08B5FFF7C1FF90F835004D
:102EB800BDE8084002F0F1BE38B5FFF7B8FF044698
:102EC80013F0BEF8054694F8350002F0E1FE6843B9
:102ED80080B238BD38B50D46FFF7A9FF29462E2226
:102EE800044613F0DDF850B1204629462E2213F08F
:102EF80029F9002384F82E30012384F83C3038BDAA
:102F08002DE9F743074640200E461546984612F02D
:102F18009FFC044628B91148114A124B4E2101F072
:102F280091FB114B114A12498DE818000020114BF2
:102F380000F0CFFD39468146FFF7CCFF9DF82830D9
:102F4800268684F835300B9B6586A363002384F8B6
:102F5800348084F83C304846BDE8FE83F1DB050840
:102F6800A11504080FDC05085D2E0008AF2E000827
:102F7800C12E0008352E000810B50C46FFF757FF84
:102F88000123048680F83C3010BD00BF4FF4A070C8
:102F98007047C82070477047074B1B78022B07B54E
:102FA80008D1064B1B78022B04D001A80DF10601AD
:102FB80003F0D0F80EBD00BFA43A0020C42E0020B4
:102FC80073B50A4B06460D4614460093002008497F
:102FD800084A094B019000F07CFD29460246234629
:102FE800304602B0BDE8704000F09ABD9F2F00083F
:102FF800952F00089B2F0008A12F000813B502ABDE
:1030080003E90600436843B1027C0124082A9C7046
:1030180004D11B692146984700E01C4620461CBD88
:1030280030B500282BD0058B002425E0036A1A7CD4
:10303800012A05D15B681A888A421BD1187F30BDE6
:10304800052A06D15B681A888A4213D193F82C00A6
:1030580030BD032A06D15B681A888A420AD193F8E0
:10306800250030BD062A05D15B681A888A4201D13D
:10307800D87A30BD01340430AC42D7D3002030BDFB
:1030880008B1817501207047F8B504460D46D0B1E6
:10309800E175D0F898309847012D0DD127460026C4
:1030A80006E0F86900F10802436906CA9847013644
:1030B800238B04379E42F4D3D4F89830204629460F
:1030C80098470120F8BDF8BDF8B5054608461746EB
:1030D8000E4612F0B5FF013FB84234BF04463C46E5
:1030E8003CB128463146224613F02CF800232B55D4
:1030F800F8BD2C70F8BDF7B504460020009001908B
:1031080000296CD00E8B68E000F1080351F82330D9
:103118001D7C042D04D15D682D88954247D001306F
:1031280000F1080351F823301D7C012D04D15D689E
:103138002D8895423BD0013000F1080351F8233027
:103148001D7C052D04D15D682D8895422FD0013056
:1031580000F1080351F823301D7C032D04D15D686C
:103168002D88954223D0013000F1080351F823300F
:103178001D7C022D04D15D682D88954217D0013041
:1031880000F1080351F823301D7C072D04D15D6838
:103198002D8A95420BD0013000F1080351F82330F5
:1031A8001D7C062D08D15D682D88954203D103F159
:1031B8000801204615E0013000F1080351F82350BA
:1031C8002B7C082B09D16F683F88974204D105F101
:1031D800080120461A4605E00130B04294D3204643
:1031E8006946082212F0E4FD2046FEBDF8B5054602
:1031F8000F461646002830D04388032B2FD02020B6
:1032080012F026FB044600282BD040F80C5B394608
:103218000C22FFF759FF1820E66112F019FB064649
:10322800B8B102230374012363760F4B44606360D3
:103238000E4BA360002323766B8805EB83020133D2
:103248009BB2012B50606B800CD16A685268137670
:1032580008E0204612F004FB04E0064602E00026DF
:1032680000E006463046F8BDEE9404088C91040848
:1032780037B5456802AB03E906003DB3037C01247A
:10328800042B85F8314022D1688E02F0EFFB95F8C7
:10329800300002F0EDFC95F8343043B9BDF8020077
:1032A800BDF80610AA1C234602F01AFD0FE0012BF8
:1032B80003D1084840F2395104E0022B07D10548F0
:1032C80040F24151044A054B01F0BCF92C46204616
:1032D8003EBD00BF22DC05086260040820DC05084A
:1032E800F8B504460F46164610B3838A0A2B20D039
:1032F800202012F0ADFA0546E8B14460102200F132
:1033080008003946FFF7E0FE4FF6FF73A08A2B80CE
:103318001F236B8000232B76831D013080B2012888
:10332800EE6144F82350A08207D1A3691876F8BD4E
:10333800F8BD0020F8BD0120F8BD0120F8BD2DE939
:10334800F3471D464B1C984282460C461746BDF86B
:1033580028600DDD95420BDC01320AF101035B1A8E
:10336800521BC8B2D2B29BB22946009602F0B6FBF5
:10337800AAF1020A3046C4EB0A0A02F077FB4FF0C2
:1033880000084FF001091FFA8AFA0BE0601C08EBED
:10339800050180B289B252460023009602F096FBDE
:1033A80009F101097B1B08F1010899451FFA88F802
:1033B800ECD3BDE8FC87F8B5C7B2144638461E46BC
:1033C8000D4602F095FB621E92B23846294602F07D
:1033D8008FFB304602F04AFB022606E0A21B92B29F
:1033E8003846294602F084FB0136A642F6D3F8BDDA
:1033F80073B504460E4600F11E00154600920023E0
:103408003C2280B21E3E02F061FBB1B220463C2253
:103418000123009502F05AFB7CBD73B504460E46A5
:103428000138154600920023032280B2013E02F0C3
:103438004DFBB1B2204603220123009502F046FB62
:103448007CBDF7B5089D2E7BEF7A1C463604AB7A17
:1034580006EB0726F618431A687B06EB00602D1862
:1034680000200190121B08462146009501F026FF16
:10347800FEBD30B5456885B004AB03E906007DB1F3
:1034880001242C736D68BDF80800BDF80A109DF87A
:103498000C209DF80E300095FFF7D3FF204600E082
:1034A800284605B030BD2DE9F04385B004AB03E9EB
:1034B80006004468BDF80860BDF80C70002C41D0C7
:1034C800012384F8263094F825300BB9A26800E06F
:1034D8006268FFB2BDF80A109DF80E3000923046BF
:1034E8003A46FFF7AEFF04F10C08022002F0C0FBD9
:1034F800404612F0A5FD054600B1451E0F3F0024C9
:10350800153E1FFA87F90DE002F0BCFB02F0C0FB84
:1035180004FB106189B248462022002302F0FAFB1E
:103528000134E4B2AC42EFD3002002F09FFAB8B203
:10353800B1B24246012302F0EDFB002002F098FBF5
:10354800012000E0204605B0BDE8F0832DE9F043F6
:1035580085B004AB03E906004568BDF80860BDF80E
:103568000C70002D3CD001236B762B7EBDF80A1021
:10357800012B0CBF6A68AA689DF80E300092FFB252
:103588003A463046FFF75DFF0C35022002F070FB2B
:10359800284612F055FD0E3F81460024163E1FFABC
:1035A80087F80DE002F06EFB02F072FB04FB10617D
:1035B80089B240462022002302F0ACFB0134E4B279
:1035C8004C45EFD9002002F051FAB8B2B1B22A4600
:1035D800012302F09FFB002002F04AFB012000E0DB
:1035E800284605B0BDE8F0832DE9F04F85B00546C3
:1035F800DDF84090029148469046039312F020FD72
:10360800DDF838A0DDF83CB00646294600242F46F0
:1036180011E024B1B4420CBF5B46534600E0039B63
:1036280001F10805ADB200932846029A4346FFF718
:1036380008FF01342946B442EBDD002002F016FAF7
:10364800022002F015FB7D1D08F10508A8B21FFA3B
:1036580088F14A46012305B0BDE8F04F02F040BBAF
:1036680070B5406886B006AB03E9060000282ED086
:10367800012380F82D308668164BF21A534243EB2B
:10368800020390F82C205AB1002B134D134B144A07
:1036980008BF1D46134B00F11C0418BF13460AE06F
:1036A800002B0D4D0D4B0E4A18BF1D460D4B00F15A
:1036B8000C0408BF1346BDF81200BDF81410BDF87D
:1036C8001620009601950294FFF78EFF012006B0A0
:1036D80070BD00BFD26904080E660408B46B040804
:1036E800F0670408966D040870B5446886B006ABA8
:1036F80003E9060004B301236377A668104B227F11
:10370800F11A4B4243EB01030AB10BB904E01BB9B0
:1037180066680C4D0C4B01E00C4D0D4BBDF81200CA
:10372800BDF81410BDF8162000960C3401950294CB
:10373800FFF75AFF012000E0204606B070BD00BF29
:103748001E7504085A7104083C730408F4760408CA
:10375800CA7804082DE9F04385B004AB03E90600F4
:103768004468BDF80860BDF80A90BDF80C50BDF873
:103778000E80002C00F08C800123A374022067685F
:1037880002F076FA4FF6FF7002F086F9002002F098
:103798006DF9EDB25FFA88F8A6F1160189B23046E4
:1037A8002A4643460097FFF74CFE277A002F2ED172
:1037B800A28A234600E00137974204D29969097E1C
:1037C80004330029F7D002F05DFA02F061FAA9F19A
:1037D80016091FFA89F90E2101FB10914FF6FF72A5
:1037E80008F101085FFA88F389B2009248462A4630
:1037F800FFF7A5FD022002F03BFA1F2002F036F980
:10380800A38A002B38D0103DE8B2303E2CE0E368A4
:103818005C68A28A2346013A002700E001379742F4
:1038280004D29969097E04330029F7D002F02AFAF4
:1038380002F02EFA0E2101FB10914FF6FF7208F1EB
:1038480001085FFA88F389B2009248462A46FFF7D2
:1038580076FD022002F00CFA1F2002F007F9A38A75
:1038680053B1103DE8B21A3E0637B1B254F82720DA
:103878000123083202F04EFA002002F0F9F94FF65F
:10388800FF7002F009F91F2002F0F0F8012000E0B3
:10389800204605B0BDE8F0832DE9F0410546362005
:1038A800884614461F4611F0D3FF0646E0B120F8BB
:1038B800025B41462E22FFF707FCBDF8183086F858
:1038C800344073861820012386F8307086F831302A
:1038D80011F0BEFF044618B104234660037404E0E7
:1038E800304611F0BDFF00E004462046BDE8F081F7
:1038F800F8B5064624200F46154611F0A9FF0446E0
:10390800D8B10F4B068083600E4B394643601022B6
:1039180000F10C00FFF7D8FB0126002318202562D0
:103928002377667711F094FF054610B1446006745A
:1039380004E0204611F094FF00E005462846F8BD53
:103948001E750408786F0408F8B506462C200F4643
:10395800154611F07DFF0446E8B120F80C6B394696
:103968001922FFF7B1FB0D4BA562A3600C4B6360F6
:10397800002384F825301820012384F8263011F01C
:1039880067FF054618B103234460037404E020462A
:1039980011F066FF00E005462846F8BD2A8E0408A7
:1039A800C88A040810B50446142011F051FF20B14C
:1039B80000234380014B0480036110BDF5310008EA
:1039C80038B50546442011F043FF0446C0B10E4BFC
:1039D800058243600D4B0360012383740023037247
:1039E80083820B4B0364182011F032FF054618B18F
:1039F80007234460037404E0204611F031FF00E01F
:103A08000546284638BD00BFBE860408B4820408AF
:103A1800E93200082DE9F04105463420884614466D
:103A28001F4611F015FF064620B3144B058083602E
:103A3800134B41464360102200F10C00FFF744FB92
:103A4800214606F11C001022FFF73EFB002386F8F2
:103A58002C3018200123376386F82D3011F0F8FE3A
:103A6800044618B105234660037404E0304611F09B
:103A7800F7FE00E004462046BDE8F081D26904085C
:103A88002C6404082DE9F041044614200D4616461E
:103A9800984611F0DDFE0746B8B1069B0480036125
:103AA8000023C37201234560068180F80A800373EE
:103AB800182011F0CDFE044618B1062347600374A0
:103AC80004E0384611F0CCFE00E004462046BDE88C
:103AD800F0812DE9F041044618200D461646984617
:103AE80011F0B6FE0746B8B101238370069B048027
:103AF8000361079B45608660C0F80C80436118200D
:103B080011F0A6FE044618B108234760037404E0C8
:103B1800384611F0A5FE00E004462046BDE8F081D5
:103B28002DE9F34198461B8B1D2B05460C4617467D
:103B38004FF0000000F2B480B5F5A07F009001902E
:103B480000F2AE80F02900F2AB80127CADF80610CE
:103B5800511EADF80250072900F28A80DFE801F013
:103B680045595E04456A14767B684E4A7A611A881C
:103B780093F834303A80013BDBB2012B7FD8ADF8A3
:103B88000240ADF806507AE005F11602ADF80020C3
:103B980004F11602ADF8042002AE434A16E9030008
:103BA8007A6107F1080282E8030003F10802013391
:103BB80048F82270A8F818307B681A8A187A3A8070
:103BC80000286CD1FFF7FCFE384943685960384932
:103BD800DF600126163D196002461E72A8B2E1B2E6
:103BE8004346FFF79DFF30465AE0012A0CBF314B90
:103BF800314B78687B6130F80C3B3B8012F020FA3F
:103C0800431CDB001A34ED18ADF80440ADF8005041
:103C180035E07B68294A1B687A6102E0284A7B689C
:103C28007A611B8814353B80ADF800501434ADF828
:103C3800044024E07B68234A7A611A883A801A890A
:103C48009B7AAD18ADF80050E418F0E77E681E4B7B
:103C58007B61338838463B8073689847013D451936
:103C6800ADF80050B36838469847013C0419DEE7C0
:103C78001648174A174B40F21A3100F0E3FC02AA23
:103C880012E9030007F1080383E80300B8F81830C5
:103C980003F10802013348F82270A8F8183001200F
:103CA800BDE8FC81793200085D370008AA7E040867
:103CB800A07A0408F136000869360008553500086E
:103CC800AF3400087B3400080530000822DC050802
:103CD8007260040820DC0508F8B51646002834D0C0
:103CE8001378002B2ED0028B002327E0046A257C52
:103CF800042D21D165682F888F421DD195F8313068
:103D080053B16F8E01F0D8FE04F10802688663692A
:103D1800204606CA98476F86A81C31462E22FFF710
:103D2800D3F995F831307BB104F108026369204674
:103D380006CA98470120F8BD013304309342D5D311
:103D48000020F8BD1846F8BD0120F8BD70B5B8B11F
:103D5800068B0446002310E0256A287C04280AD133
:103D68006D682888884206D11046A91C2E22FFF7C4
:103D7800ABF9012070BD01330434B342ECD3002009
:103D880070BD38B5044620B3134BC361134BC0F85C
:103D98009830134BC0F89C30124B00257822C0F89D
:103DA800A0308575C5750583294600F1200012F0FD
:103DB80041F8D4F898302046294698470A4A13888B
:103DC800312B07D8094941F82340013313800120DA
:103DD80038BD38BD284638BD913000088930000804
:103DE80029300008FF300008640E0020AC1A0020BB
:103DF8002DE9F0410446002800F0B380078B024605
:103E08000025A8E0136A1E7C042E00F08780012E8E
:103E180023D1586803888B4240F09B8005F108073E
:103E280011F01EFD54F827004FF00008C0F8048078
:103E380011F016FD228B531E9D4208D007322383B2
:103E480054F8221044F8271044F8228002E044F87D
:103E5800278025833046BDE8F081052E5ED0032EED
:103E68005CD0022E13D15B68186803888B4270D12E
:103E78004388013B9BB243800BB911F0F1FC05F17B
:103E8800080654F82630586811F0EAFC4EE0072E70
:103E980021D15E68338A8B425BD1002706E0BB1DC7
:103EA800013756F8230011F0DBFCFFB2B38ABB429E
:103EB800F5D80027B78205F1080654F82630586867
:103EC80011F0CEFC54F8260033E044F82670258320
:103ED8000120BDE8F081062E1ED1586803888B4268
:103EE80037D105F1080611F0BBFC54F8260000276D
:103EF800476011F0B5FC228B531E9D4209D0083350
:103F0800013A54F82310228344F8261044F8237009
:103F1800DEE744F826701AE0082E1AD1586803889C
:103F28008B4216D111F09CFC05F1080654F82600C6
:103F38000027476011F094FC228B531E9D42C4D089
:103F4800073254F8221044F8261044F822702383CC
:103F5800BEE701350432BD42FFF454AF0020BDE88E
:103F6800F081BDE8F08170B5044600282AD0068BA0
:103F7800751E083600EB86061EE056F8043D1A7CCE
:103F8800042A13D0012A11D0052A0FD0032A0DD0F4
:103F9800022A02D15B681B6809E0072A02D15B6824
:103FA800198A05E0062A01D0082A04D15B68198815
:103FB8002046FFF71DFF013D681CDED10023238347
:103FC800012070BD70BDF0B528B30023068B1A46DA
:103FD8001EE0046A257C072D18D16468258A8D4265
:103FE80014D1A78A002504EB83040DE004EB050C2B
:103FF8000435DCF818C09CF818C0BCF1010F03F1B7
:10400800010301D1D8B2F0BDBB42EFD30132043075
:10401800B242DED30020F0BD70B508B3048B002394
:104028001BE0026A157C072D15D15268158A8D424E
:1040380011D10023958A11461C46012007E013B9C7
:104048009669307601E08E69347601330431AB42EB
:10405800F5D3012070BD01330430A342E1D3002021
:1040680070BD2DE9F04128B30023078B1A461EE0E6
:10407800046A257C072D18D16468258A8D4214D1DD
:10408800B4F814C0002504EB83040CE06619043569
:10409800B66996F81880B8F1010F03D106F1080047
:1040A800BDE8F08101336345F0D301320430BA42F0
:1040B800DED30020BDE8F0812DE9F04700282FD09D
:1040C8000023B0F818C01D4627E0046A267C072E96
:1040D80021D16468268A8E421DD1B4F81480002646
:1040E80004EB830915E009EB0604A7693C7E012C63
:1040F8000DD192F800A0BAF1000F08D007F108001E
:1041080011461022FEF7E0FF2046BDE8F087013394
:1041180004364345E7D3013504306545D5D300203F
:10412800BDE8F087F0B5B0B1068B002510E0046A51
:10413800277C062F0AD1646827888F4206D12381FD
:104148009DF814306260A3720120F0BD013504307F
:10415800B542ECD30020F0BD10B500210446FEF7AF
:1041680093FF20460121BDE81040FEF78DBF38B50A
:1041780098B1048B024600230CE0106A05880432CB
:104188008D4206D100F10802436906CA984701200A
:1041980038BD0133A342F0D3002038BD10B50C461A
:1041A8000021FEF771FF20460121BDE81040FEF70F
:1041B8006BBF13B502AC04E90C00BDF802308342B2
:1041C80006D8BDF80030834234BF0020012000E04B
:1041D8000020BDF806308B4206D8BDF804308B426B
:1041E80034BF0021012100E00021002818BF084643
:1041F800C0B21CBD38B5114B114A1988002319E00B
:1042080052F8045FA87D012812D100240CE004F1C3
:10421800080355F82300037C082B03D143680021C9
:104228001B6998470134A4B22B8BA342EFD838BD41
:1042380001339BB28B42E3D138BD00BF640E00202E
:10424800A81A0020704770B5094CA5787DB9094BAC
:104258001E78012E0BD16368013363606268064BD8
:104268009A4204D9284601F0C5FCA670656070BD65
:10427800640E00208401002040420F00054A90602F
:10428800134602E099680139996091680029F9D1CB
:10429800704700BF640E0020F0B585B001F058FFEC
:1042A800002800F04981002502A80DF10A01ADF8A7
:1042B8000850ADF80A5001F04DFF03A80DF10E01AA
:1042C800ADF80C50ADF80E5001F090FFBDF80C1091
:1042D800BDF808200091BDF80E10BDF80A30019114
:1042E8002C46964D964908200AF0CAF8A878012865
:1042F80003D101F07FFCAC7019E1924B5B78012B84
:1043080040F01581AB78002B40F011816B60298853
:104318008D4A09E152F8046FB07D012840F002810E
:104328000025FAE005F10803BDF8080056F8234017
:10433800BDF80A1004F108030CCBFFF73AFF002878
:1043480000F0E980237C013B062B00F29F80DFE828
:1043580003F00429159D1F9D4C006668012304F194
:104368000805337795E806006369204698470023D7
:1043780033772046636995E8060086E0636893F81A
:10438800252012F1FF3218BF012283F8252077E09B
:10439800636893F82C2012F1FF3218BF012283F8CA
:1043A8002C206DE06268137E1568002B6ED16E8834
:1043B8002F462946184606E051F804EFDEF804E0D7
:1043C80001338EF81800B342F6D301231376002682
:1043D80007E057F8040F00F10802436906CA984736
:1043E80001366B889E42F4D350E0656820892E68B8
:1043F800A37B227B0096A0F1160189B2FFF721F872
:104408001420FFF73BFF2B7AC3B9AF8A29461A4617
:104418001E4609E0886990F818E00676BEF1010F9B
:1044280008BF134604310132BA42F3D301220BB953
:10443800AB6924E0053355F8233020E06368DB6876
:104448005A680023908A154619461F4609E0AE6946
:1044580096F818E03776BEF1010F08BF0B46043511
:1044680001318142F3D3411E8B4203D1053052F80A
:10447800203003E004D2073352F8233001221A76A1
:1044880004F1080206CA636920469847237C013B69
:10449800072B4CD8DFE803F00410074B0A0D123A3B
:1044A80063681B6A34E063689B6A2DE063681B6B72
:1044B8002AE063681B6927E0636824E063681A7A66
:1044C8007AB9988A1946013800E00132824204D24A
:1044D8008C69247E0431002CF7D0063253F8223040
:1044E80011E0DB685A68908A11460138002300E021
:1044F8000133834204D28C69247E0431002CF7D026
:10450800063352F82330DB69984710E06368DB68AC
:10451800204698470BE00135ADB2338BAB423FF6EE
:1045280001AF04E001339BB28B427FF4F3AE01F09C
:1045380055FE0F20FFF7A2FE05B0F0BD640E002067
:1045480048DC050884010020A81A0020034B9A685B
:1045580012B19A68013A9A60704700BF640E002051
:104568002DE9F3470120DFF8D080DFF8D09001462D
:104578000BF020FB012400254FF4807602274046EB
:10458800694600968DF804708DF805408DF8065040
:104598008DF807400AF066FF4046082122460AF0D7
:1045A800E1FF244BDFF898801A6844F2A243B2FB7B
:1045B800F3FA0AF1FF3A204621461FFA8AFA0BF06D
:1045C80029FBC8F804A048464146A8F80050A8F8B6
:1045D8000250A8F8085088F80A500BF0B7FE70236C
:1045E800A8F80C300423A8F810300AF1FF3A632326
:1045F800642203FB0AF3B3FBF2F39BB2C8F814304E
:1046080008F10C014846A8F80E40A8F81870A8F858
:104618001A50A8F81C60A8F81E500BF0B5FF4846C1
:1046280021460BF028FF484621460CF02EFABDE83B
:10463800FC8700BF980200200000024000000140F3
:10464800740E002083B50E460746154910201C46F7
:10465800154609F015FF1020124909F011FF102026
:10466800114909F00DFF10200E4909F009FF002338
:1046780010200E49019309F003FF334610200C491E
:104688003A4609F0FDFE10200A492A4609F0F8FECC
:1046980010200949224609F0F3FE019B0133E7E7A0
:1046A80082DC050887DC0508A7DC0508B7DC0508F7
:1046B800C7DC0508DCDC0508EDDC050808B5164B89
:1046C8001A6A01321A621A6A012A1A4603D0134872
:1046D80040F21E210FE05862194602E04B6A013B86
:1046E8004B62506A0C4B0028F8D11A6A012A06D08E
:1046F8000A4840F229210A4A0A4BFFF7A3FF1A6A1F
:10470800013A1A621B6A2BB10448054A064B40F26B
:104718002B21F2E708BD00BF740E0020FEDC05085F
:104728005098040828DD050839DD050810B5084C3F
:104738000221002220460AF00AFF44F6FF70FFF724
:10474800BDFF204602210122BDE810400AF0FFBE4D
:10475800000402400C4B0D491A6844F2A243642835
:10476800B2FBF3F3D4BF20EAE0706420013B9BB2B4
:104778004B60013B58436422B0FBF2F080B24861C1
:1047880003480C310BF083BE98020020740E002001
:104798000000014010B5134B93F828202AB11248A5
:1047A800124A134B40F209310EE0012283F8282007
:1047B80066234FF0C042013BDBB2108033B90A4890
:1047C8000A4A0C4B40F21331FFF73CFF1488A4B29D
:1047D8008442F0D1084B1980024B002283F828202C
:1047E80010BD00BF740E0020FEDC05085A980408AE
:1047F8004ADD050820DC05080000026010B5FFF757
:10480800AFFE6420FFF7A6FF21210720FFF7C2FFB4
:104818003220FFF753FF01210020FFF7BBFF3220B2
:10482800FFF74CFF23210720FFF7B4FF3220FFF7E3
:1048380045FF00211020FFF7ADFF41F28830FFF758
:104848003DFF33210720FFF7A5FF3220FFF736FF92
:10485800112046F63001FFF79DFF3220FFF72EFFAB
:104868004FF4C0610220FFF795FF3220FFF726FFC3
:10487800122046F6EB41FFF78DFF3220FFF71EFFAF
:1048880003204AF6A401FFF785FF3220FFF716FF41
:1048980000210C20FFF77EFF3220FFF70FFF0D20CD
:1048A80040F60C01FFF776FF3220FFF707FF0E20D6
:1048B8004FF42C51FFF76EFF3220FFF7FFFEB021B7
:1048C8001E20FFF767FF3220FFF7F8FE012042F6AF
:1048D8003F31FFF75FFF3220FFF7F0FE0520002190
:1048E800FFF758FF3220FFF7E9FE00210620FFF707
:1048F80051FF3220FFF7E2FE16204EF61C71FFF73B
:1049080049FF3220FFF7DAFE172040F20311FFF7C4
:1049180041FF3220FFF7D2FE00210B20FFF73AFFBC
:104928003220FFF7CBFE00210F20FFF733FF3220A4
:10493800FFF7C4FE41200021FFF72CFF3220FFF7CC
:10494800BDFE42200021FFF725FF3220FFF7B6FE0B
:1049580000214820FFF71EFF40F23F143220FFF7E6
:10496800ADFE21464920FFF715FF3220FFF7A6FECE
:1049780000214A20FFF70EFF3220FFF79FFE00219B
:104988004B20FFF707FF3220FFF798FE44204FF433
:104998006F41FFF7FFFE3220FFF790FE0021452010
:1049A800FFF7F8FE3220FFF789FE21464620FFF781
:1049B800F1FE3220FFF782FE302040F20771FFF748
:1049C800E9FE3220FFF77AFE31204FF40171FFF73C
:1049D800E1FE3220FFF772FE32204FF40171FFF73B
:1049E800D9FE40F202543220FFF768FE21463320F8
:1049F800FFF7D0FE3220FFF761FE342040F2075166
:104A0800FFF7C8FE3220FFF759FE35204FF4017139
:104A1800FFF7C0FE3220FFF751FE36204FF4017138
:104A2800FFF7B8FE3220FFF749FE21463720FFF78F
:104A3800B1FEA4F500743220FFF740FE21463A206B
:104A4800FFF7A8FE3220FFF739FE2F2041F2BE21E2
:104A5800FFF7A0FE3220FFF731FE21463B20FFF78B
:104A680099FE3220FFF72AFE00212320FFF792FE4D
:104A78003220FFF723FE00212420FFF78BFE32208F
:104A8800FFF71CFE25204FF40041FFF783FE32207C
:104A9800FFF714FE00214F20FFF77CFE3220FFF7BE
:104AA8000DFE4E200021FFF775FE3220BDE81040B4
:104AB80004E608B5124B93F829202AB11148124A86
:104AC800124B40F223310FE0012283F829202221E2
:104AD80066234FF0C042013BDBB2118033B909486D
:104AE800094A0B4B4FF44F71FFF7ACFD108880B2A9
:104AF8002228F0D1024B002283F8292008BD00BFEC
:104B0800740E0020FEDC0508679804084ADD0508D5
:104B180020DC050810B51E4B032826D8DFE800F076
:104B2800021A080E1C8841F2280246F628000AE0FC
:104B38001C8841F2080246F6080004E01C8841F28D
:104B4800300246F6300049F241318C4214BF01462A
:104B580011460BE0188846F6200249F24131884296
:104B680014BF11464FF4815100E000211B8848F61C
:104B78008912934205D049F22032934204D103208E
:104B880000E01120FFF706FEBDE8104091E700BFE6
:104B980086010020014B18800A208FE50000026082
:104BA8004FF0C043188003F500331A881A88188814
:104BB80080B270474FF0C04322221A8003F50033B9
:104BC80082B01A8892B2ADF806201B889BB2ADF865
:104BD8000630BDF8060080B202B07047072040F2E8
:104BE8007311D7E507200021D4E582B0044BADF856
:104BF8000600BDF8062092B25A8502B0704700BF81
:104C0800740E002082B0044BADF80600BDF80620F3
:104C180092B25A8002B0704786010020014B80B2E0
:104C280018807047000002604FF0C04380B21880BF
:104C38007047024B80B21880704700BF00000260C6
:104C48004FF0C04380B218807047024B80B2188082
:104C5800704700BF0000026082B0044B0190019AC7
:104C6800DA62DA6A002AFCD102B07047740E0020BA
:104C780070B54FF0C0452A242C800A4C060AC0B2F1
:104C880026802080100AD2B2208022802B222A80FF
:104C98000A0A2280C9B21A0ADBB221802280238044
:104CA80070BD00BF0000026010B50B4614460246F6
:104CB800FFF7DEFF4FF0C0432C22A0B21A80BDE8F8
:104CC800104067E7114B1B8848F68912934210B5CC
:104CD80004460BD049F22032934212D1C1F1EF01C0
:104CE800202089B2FFF756FD212006E0C1F1EF012F
:104CF8004E2089B2FFF74EFD4F202146BDE81040F7
:104D080048E502460B46BDE81040B1E786010020A1
:104D180008B5FFF7D7FF0F4B1B78012B4FF0C042A8
:104D28000D4B0FD12E2111801A881A881B8892B238
:104D380002F0FC0002F4784242EAC000C3F3C42344
:104D4800184308BD222111801A881A88188880B251
:104D580008BD00BF7C1B00200000026070B5074D35
:104D68000646012421463046FFF7D2FF0134A4B29B
:104D7800C82C25F8020FF5D170BD00BFA63A002057
:104D880010B5084B1B78012B144602D1BDE8104022
:104D98008AE7FFF797FFFFF78CFE2046BDE8104033
:104DA800F8E600BF7C1B002070B5074D06460124BD
:104DB8002146013435F8022F3046A4B2FFF7E0FF50
:104DC800C82CF5D170BD00BFA63A002070B50546C5
:104DD8000E46FFF7C3FF0124214601342846324618
:104DE800A4B2FFF7CDFFC82CF6D170BD2DE9F04174
:104DF80004460D461646BDF81880032B39D8DFE85F
:104E080003F00B351927381980B229464246013775
:104E1800FFF7B6FFBFB200E00027B742F3D1BDE805
:104E2800F081E01B80B2294642460137FFF7A8FF10
:104E3800BFB200E00027B742F3D1BDE8F081E91B1B
:104E480089B2204642460137FFF79AFFBFB200E019
:104E58000027B742F3D1BDE8F081791989B220461D
:104E680042460137FFF78CFFBFB200E00027B74288
:104E7800F3D1BDE8F08170B5194B1A4A598E92F9F1
:104E8800004064180025A4B28AB0AC4208BF0124CF
:104E9800C62C28BFC62415700F264FF6FF721E8633
:104EA8005C865A8519202B46009221460A22FFF774
:104EB8009DFF21463046FFF72BFF224603460A494D
:104EC80002A811F037F802AA06A8084911F032F82A
:104ED8003220D22106AA2B4600F002FF0AB070BD8C
:104EE800740E0020E91B00205FDD050867DD05085A
:104EF8002DE9F341BDF820500C4690461F461A464E
:104F0800002306460095FFF771FF611E41443046B5
:104F18003A46002389B20095FFF768FF30462146DC
:104F2800424601230095013EFFF760FFBF19B8B262
:104F3800214642460123089502B0BDE8F04155E7F5
:104F48002DE9F0410D46C5F1F008411E5E18C2EB8F
:104F58000802C5F1EF039BB292B2B6B29A422CBFD7
:104F6800904698469A4234BF11461946864234BF45
:104F78003746074640F23F13864238BF06469E42F0
:104F880028BF1E46174B1B8848F68912B8F1EF0F49
:104F980028BF4FF0EF089342044610D049F2203260
:104FA80093421AD15020FFF7F5FB51204146FFF7F5
:104FB800F1FB52203946FFF7EDFB53200AE041EAA6
:104FC800082189B24420FFF7E5FB45203946FFF761
:104FD800E1FB46203146FFF7DDFB20462946BDE8C8
:104FE800F0416FE68601002000200146F0224FF4D0
:104FF800A073A5E770B580B202FB03F489B292B240
:105008009BB2FFF79DFF0020FFF784FD0025064EA9
:1050180004E0708D80B2FFF7BDFD0135A542F8DBD5
:10502800BDE87040E0E700BF740E002070B54FF097
:10503800C0452A242C80094C060A26802080080AAC
:10504800208021802B212980110A218022801A0AA0
:10505800228023802C232B8070BD00BF00000260BB
:1050680070B5114B1B78012B044607D1002040F284
:105078003F110246EF23FFF7D9FF04E0FFF7B4FF23
:105088000020FFF747FDF02509E0013E2046B6B2B3
:10509800FFF780FD002EF8D1013DADB215B14FF4F8
:1050A800A076F2E770BD00BF7C1B00202DE9F04F11
:1050B8001C463E4B87B01B78039183469DF84410ED
:1050C80010980591012B039B049092461FFA8BF0D0
:1050D8009AB208D1411E531E0919534489B29BB292
:1050E800FFF7A4FF09E01FFA8AF51146A3B22A4682
:1050F800FFF726FF0020FFF70DFD0027DDF80C80E5
:105108003E4640F23F1CA14639E0BBF1000F2EDBC2
:1051180065452CDC0398002829DBB8F1EF0F26DC65
:10512800220702D1002CC8BF01362149214000299D
:1051380003DA013961F00F010131059A0AB1C1F1B1
:105148000F01049830F8162003FA01F10A4012B250
:105158006AB118494A8D029392B2A8B21FFA88F12F
:10516800CDF804C0FFF70CFEDDF804C0029B013443
:1051780001354C45C9DB0136013708F101085745AF
:1051880003DA5D4600240123F3E7084B1B78012B63
:1051980008D1002040F23F110246EF2307B0BDE8D6
:1051A800F04F43E707B0BDE8F04F1DE77C1B002038
:1051B8000F000080740E00202DE9F74F1F463B4B6F
:1051C800DDF830801B7816469DF83420012B044604
:1051D80001920D4680B28AB208D1411E531EC919E8
:1051E8009B1989B29BB2FFF721FF09E01FFA86FEDF
:1051F8001146BBB27246FFF7A3FE0020FFF78AFCF8
:105208004FF0000BDA463DE0002C30DB09EB0403DD
:1052180040F23F1293422ADC002D28DB0BEB0503FA
:10522800EF2B24DC19F00F0F04D1B9F1000FC8BF20
:105238000AF1010A1E4B09EA0303002B03DA013BBA
:1052480063F00F030133019A0AB1C3F10F0301227E
:1052580002FA03F338F81A2013401BB213B1154BA6
:10526800588D01E0144A508880B2FFF793FC09F189
:10527800010901E04FF00009B945C5DB0AF1010A4F
:105288000BF1010BB345F5DB084B1B78012B08D15B
:10529800002040F23F110246EF2303B0BDE8F04F73
:1052A800C4E603B0BDE8F04F9EE600BF7C1B0020BB
:1052B8000F000080740E0020860100202DE9F041C7
:1052C8001C4F069C3F789DF81C60012F02FB03F5DC
:1052D80080B28FB209D1411ECB1899B27B1E9A18A1
:1052E80093B23A46FFF7A2FE07E092B29BB2394664
:1052F800FFF726FE0020FFF70DFC002709E034F831
:10530800020B1EB1030A43EA002080B2FFF742FCF9
:105318000137AF42F3DB074B1B78012B07D1002085
:1053280040F23F110246EF23BDE8F0417EE6BDE8BA
:10533800F04159E67C1B00202DE9F0431F2093B073
:10534800FFF78EFE4FF47840FFF78AFE4FF6E075C0
:105358004FF4FC60FFF784FE2846FFF781FE00202B
:10536800514CFFF77DFE00204FF6FF79014664227D
:105378000346A4F82A90CDF80090FFF737FD0020E7
:105388000A2164220346CDF80090FFF72FFD002084
:105398000146642201234FF4784765850095FFF79D
:1053A80025FD7720EF21C82200234FF4FC6667858E
:1053B8000097FFF71BFDBD213222012340F23F1069
:1053C80066850096FFF712FDA0203222002378217F
:1053D80067850097FFF70AFDA02078213222012374
:1053E8004FF01F0866850096FFF700FDA020782182
:1053F80032220223A4F82A80CDF80080FFF7F6FCB9
:10540800A02078213222032365850095FFF7EEFC62
:10541800264B2749A3F8028002AD3C22284610F00B
:10542800C7FCEB20C3210522302300950025A4F8F2
:105438002A900195FFF7C0FE32210A2096220B46DA
:1054480067850097FFF754FD32213C2096220B46D2
:1054580066850096FFF74CFD32210B4696226E209A
:10546800A4F82A80CDF80080FFF742FDFFF7BAFBC9
:10547800FFF7B4FB3220FFF76DF92846FFF76AF90A
:105488006420FFF767F90B4B03F110028DE8240045
:1054980028465A681B682946FFF710FF1195119B8B
:1054A80001331193FBE700BF740E00208601002032
:1054B8007C98040810BD01082DE9F14FFFF750F85A
:1054C8004FF0C0456420FFF745F90127FFF72EF993
:1054D8004FF028096D48FFF7F1F82F800520A5F84F
:1054E800009003F03DF9CF232B80694B00268322DF
:1054F8001E801A8030221A80ED222A804FF064081C
:105508000322A3F800801A8012221A8081221A80AE
:10551800E8222A8085221A8079221F801A80CB22CD
:105528002A8039221A804FF0340C02242C21F722C9
:1055380019801E80A3F800C01C802A8020221A80AF
:10554800EA222A80C0221E80C1211E802A802622AB
:105558001A80298011211980C521298035211980B7
:105568003E211980C7212980BE2119803621298032
:105578003A205521A3F8009028801980B12129806C
:105588004FF0100BF2211E80A3F800B029800821EB
:1055980019802A80E0221F804FF01F092A801A22D2
:1055A800A3F800904FF0180A1A800F210A22A3F8D6
:1055B80000A01A80198006211980452119808721A9
:1055C80019803221198007211A804FF0E10E1980C5
:1055D8001C80052419801C801E80A5F800E04FF06F
:1055E800250E1E80A3F800E04FF0270EA3F800E078
:1055F8001C80A3F800B04FF0090BA3F800B04FF0DF
:10560800780B1880A3F800B04FF04D0BA3F800B04A
:105618001C800D24A3F800A01C8038241C8018804E
:105628002A20A3F80090EF2428802B201E801E80BB
:105638001E801C8028803F201E801E801F801880AE
:10564800B720A5F800C028801980B62129801A80C3
:1056580082221A801122A3F800E040461E802927E2
:105668002A8003F07DF840462F8003F079F8094836
:10567800FFF724F82C232F8030462B8040F23F116F
:105688003246234601B0BDE8F04FCFE4400D030099
:105698000000026040420F002DE9F041022098B05E
:1056A800012100240AF086FA012502268048169670
:1056B80016A98DF85D408DF85E408DF85F408DF835
:1056C8005C5009F0CFFE182029460AF073FA2846E4
:1056D80029460AF087FA21460C22764809F042FF4B
:1056E8000C227448294609F03DFF04210C22714818
:1056F80009F038FF05210C226E4809F033FF072115
:105708000C226C4809F02EFF08210C22694809F088
:1057180029FF09210C22674809F024FF0A2165485E
:105728000C2209F01FFF0B2162480C2209F01AFF16
:105738000E210C225F4809F015FF0F210C225D484D
:1057480009F010FF07210C225B4809F00BFF082124
:105758000C22594809F006FF09210C22564809F085
:1057680001FF0A210C22544809F0FCFE0B210C22EF
:10577800514809F0F7FE0C210A464F4809F0F2FE9D
:105788000D210C224C4809F0EDFE0E210C224A484E
:1057980009F0E8FE0C2248480F2109F0E3FE4CF618
:1057A800B3734448169316A98DF85C608DF85E4073
:1057B8008DF85F408DF85D5009F054FE16A94FF63C
:1057C80080733D4816938DF85C608DF85E408DF8C7
:1057D8005F408DF85D5009F045FE40F6B830FEF7A1
:1057E8006DFFFEF7A3FF40F6B830FEF767FF0F2303
:1057F80011934FF4805310270DF13C080993684624
:105808004FF4002310941294149415940094019466
:105818000294039704940694079408940A940594B0
:105828000B940C93CDF834800F95139509F093FBE6
:105838000523684611930F961094129414941594A6
:10584800CDF83880139509F086FB2946204609F0E3
:1058580002FC40F6B830FEF731FF2046FFF7A0F90A
:1058680004461649164E3846224608F009FE41F20B
:1058780089239C4248F68918124F01D044450ED11D
:10588800FEF7BCFF00233B70A6F8008010200E49ED
:1058980048F6891241F2892308F0F2FD05E0FFF786
:1058A8000BFE49F241333D70338018B0BDE8F081FA
:1058B80000040240000C0240001002406CDD0508A4
:1058C800860100207C1B002083DD05084FF0C043C3
:1058D80036221A8003F50033012814BF68204820B7
:1058E8001880704770B5244B01228CB01A700024C0
:1058F8000AE0A9B21F2230460135FFF741FA642DAC
:10590800F7D10134642C02D00025A6B2F1E7322089
:10591800014602460346FFF7ABF94FF0C0432E227B
:105928001A8003F5003300201A881C881D88A4B249
:1059380000F09CF8ADB20023224600930F492B4695
:1059480003A810F0F7FA00230A20C82103AA00F0E0
:10595800C7F904F0FC0204F4784444EAC20242EABB
:10596800D522074903A810F0E5FA0A20DC2103AA8A
:10597800002300F0B5F9FEE77C1B0020C2DD050816
:10598800DADD05082DE9F04F40F23F19484534BFEC
:1059980004464C46EF2B34BF98464FF0EF084A4573
:1059A80038BF9146EF2934BF0D46EF25C4EB090AED
:1059B800C5EB080785B0BAF1000FB8BFCAF1000AF5
:1059C800002FB8BF7F424FF6FF734C452CBF1A46D5
:1059D80001221FFA8AFA454538BF0123BFB2029354
:1059E8000FFA8AF63BB29E42BDF838B0019202DD4A
:1059F800C6F34F0607E0022693FBF6F67642B6B2E8
:105A080001E01E4603E00FFA8AF35B420393144A4F
:105A18001378022B204629465A4602D1FDF7FDFC91
:105A280001E0FFF7ADF94C4501D1454514D0039A83
:105A380033B2934205DD019AF31BA4189BB2A4B2BA
:105A480000E0334636B23AB29642DADA029A534462
:105A5800AD189BB2ADB2D4E705B0BDE8F08F00BF7A
:105A6800C42E002000487047841B002082B0064BDB
:105A7800ADF80600BDF8062092B21A80188880B2E8
:105A880002B0FFF7B2B800BF801B0020014B188896
:105A980080B27047801B002082B0064BADF806002C
:105AA800BDF8062092B21A80188880B202B0FFF7BB
:105AB800A9B800BF821B0020014B188880B270472C
:105AC800821B0020FFF7CCBAFFF73ABA10B5BDF831
:105AD80008400294BDE81040FFF788B910B5BDF83A
:105AE80008400294BDE81040FFF702BAFFF782BAF7
:105AF8002DE9F04F4FEA420800253D4C85B082461B
:105B08008B46C8F1030817462E461FFA87F909EB9A
:105B18000B0C228805EB0A031FFA8CFC9BB261462A
:105B2800184692B2CDF804C00293FFF729F9C9EBE1
:105B38000B0292B20392029B22880399184692B2F2
:105B4800FFF71EF9DDF804C02288C5EB0A039BB2F3
:105B58006146184692B20293FFF712F9029B228817
:105B68000399184692B2FFF70BF905EB0B0292B2B4
:105B7800039209EB0A03228803999BB2184692B252
:105B88000293FFF7FDF8029B2288C5EB0B0C1FFA66
:105B98008CFC1846614692B2CDF804C0C9EB0A09DC
:105BA800FFF7EEF8228803991FFA89F992B248465E
:105BB800FFF7E6F82288DDF804C092B2484661464D
:105BC800FFF7DEF8B8F1000F04DA08EB860808F1F1
:105BD800060805E0F31B08F10A0808EB8308013FF3
:105BE80001360135BE42ADB28FD905B0BDE8F08FA0
:105BF800801B002008B9FEF7F5BF012801D1FEF788
:105C0800EDBF7047704700200146F0224FF4A073A3
:105C1800FFF796B9704708B505280CD8DFE800F0FB
:105C2800121403050709094808BD094808BD0948B1
:105C380008BD094808BD0948094A0A4B40F2411104
:105C4800FEF700FD084808BD084808BD740100209B
:105C5800640100205C01002054010020E5DD0508F6
:105C6800B898040820DC05087C0100206C0100209D
:105C780010B50446FFF7CFFF014B18601C7110BD2B
:105C88008C010020014B1879704700BF8C0100205F
:105C980008B5FFF7C0FF808808BD08B5FFF7BBFF50
:105CA800C08808BDF7B51F460B4B0C4E1D6814463F
:105CB800EA882B68203C5443A4B2AE1B03EB44048F
:105CC80018BF0126AB888DE8500017B1FFF7EEF931
:105CD80001E0FFF771FAFEBD8C0100207C01002075
:105CE8002DE9F0410F46984615460446084E08E04F
:105CF800204643463946FFF7D5FF33689B88E418AA
:105D0800A4B215F8012B002AF2D1BDE8F08100BF3A
:105D18008C01002010B5044608462146BDE8104015
:105D2800DEE7094B70B5044618790E461546FFF7AD
:105D3800B4FFC6F1F001091A89B220462A460023A9
:105D4800BDE87040CCE700BF8C010020704700BF61
:105D5800044B1A680AB9044A1A601A6810181860BD
:105D680010467047A80E0020403F00204FF0FF303B
:105D7800704708B50248034A034B3721FEF762FC17
:105D880004DE0508CE98040820DC050801207047C9
:105D980010B504460A4802210AF092F90028F9D001
:105DA800074821460AF055F9054801210AF088F903
:105DB8000028F9D00248BDE810400AF047B900BFF2
:105DC8000038004010B5194802210AF079F9002876
:105DD800F9D0164800210AF03CF9144801210AF0CC
:105DE8006FF90028F9D011480AF030F90402A4B27A
:105DF800002301E001339BB2002BFBD00B480221AA
:105E08000AF05EF90028F9D0084800210AF021F9C3
:105E1800064801210AF054F90028F9D003480AF08D
:105E280015F92043C0F3CB0010BD00BF0038004077
:105E38002DE9F0478AB00AAF0A20012109F0BAFE1D
:105E48004FF4604347F8143D474EDFF824A101247E
:105E580000254FF00208304639468DF81A508DF863
:105E680018808DF819808DF81B4009F0FBFA304630
:105E78000D21052209F076FB30460E21052209F096
:105E880071FB052230460F2109F06CFB21464FF4C7
:105E9800804009F0B3FE504609F08EFF4FF482733C
:105EA800ADF802304FF40073ADF80A303823ADF87E
:105EB8000C30504607236946ADF81030ADF8005055
:105EC800ADF80450ADF80650ADF80850ADF80E50D6
:105ED80009F0A4FF504621460AF03BF8A9468DF880
:105EE8001A5030464FF48055394605958DF81840BC
:105EF8008DF819808DF81B4009F0B4FA3046294610
:105F080009F021FB4025394618488DF818908DF87E
:105F180019808DF81A908DF81B40059509F0A2FAA2
:105F280021464FF4804009F075FE062103200AF04F
:105F3800FFF80C2307A88DF8213007958DF82090DD
:105F48008DF8224008F082FF17238DF8243009A825
:105F58000F238DF825308DF826308DF8274002F074
:105F68001DFE0AB0BDE8F08700040240000C0240A4
:105F780000380040014B1878704700BFAC0E002075
:105F8800024B5A889B8802800B807047AC0E002019
:105F9800014B00221A707047AC0E0020F0B593B088
:105FA8006846002148220FF045FF6D4600246448EA
:105FB8004FF4805109F0C9FA002301E001339BB284
:105FC800002BFBD09020FFF7E3FE002301E0013314
:105FD8009BB2002BFBD0FFF7F5FE4FF4805107462C
:105FE800574809F0B0FA002301E001339BB2002BB7
:105FF800FBD053484FF4805109F0A7FA002301E081
:1060080001339BB2002BFBD0D020FFF7C1FE002349
:1060180001E001339BB2002BFBD0FFF7D3FE4FF416
:1060280080510646464809F08EFA45F8047B01344B
:106038002E6244484021E4B209F073FA10B9092CE1
:10604800B5D101E0092C78D19DE80C00D218029B4B
:1060580003980699D218049BC018059BC018079B83
:10606800CB180899032490FBF4F092FBF4F25B1828
:1060780093FBF4F3151AC11A9C1A002DB8BF6D4290
:106088000029B8BF4942002CB8BF6442502D03DD37
:10609800502909DD502C50DC8D4205DAAC424FF016
:1060A800020405DB111806E08C424FF0020401DA05
:1060B800D11800E0C1180A9B099A0C980F9DD218B4
:1060C8000B9BD2180D9BC0180E9BC018109BEB1889
:1060D800119D91FBF4F1032492FBF4F290FBF4F090
:1060E8005B1993FBF4F3161AC41A9D1A002EB8BF55
:1060F8007642002CB8BF6442002DB8BF6D42502EC6
:1061080089B203DD502C09DD502D16DCA64205DAD4
:10611800B5424FF0020405DB131806E0A5424FF024
:10612800020401DAD31800E0C318074A93FBF4F31A
:106138009BB2938001235180137013B0F0BD00BF50
:1061480000040240000C0240AC0E002000000000D9
:10615800FFF710BFF7B505460C4601A80DF106017B
:10616800FFF70EFF1B4BBDF80660BDF8040093E86F
:106178000600724301FB002299685218164992FBE7
:10618800F1F207EE102AF8EEC77A40F23F17FCEE5C
:10619800E77A17EE902A92B2B2F5207F28BF3A46E6
:1061A8002A801D69DA685B696E4302FB0060C018CB
:1061B80090FBF1F107EE101AF8EEC77AFCEEE77AD9
:1061C80017EE903A9BB2B3F5F07F28BFEF232380F8
:1061D800FEBD00BFB40E002040420F00FFF7D8BE3E
:1061E800014B187E704700BFB40E0020FFF7C8BEF1
:1061F800042808B505D90748074A084B7D21FEF74A
:1062080021FA054B03EB8000038B0B80438B138033
:1062180008BD00BF25DE0508D498040843DE05083C
:1062280008B5082001F0F6F942F69643C31A584219
:1062380040EB030008BD10B50A2001F013FA0C4C1E
:1062480020600E2001F00EFA6060122001F00AFAB8
:10625800A060162001F006FAE0601A2001F002FAA8
:1062680020611E2001F0FEF901236061237610BD34
:10627800B40E002010B5FFF7DBFD01F0A7FA0446C5
:1062880001F0B0FA074903462246202008F0F8F842
:10629800FFF7C6FF28B101F0B3FA10B9BDE8104006
:1062A800C9E710BD7FDE050810B5104C0A2021682B
:1062B80001F0BFF961680E2001F0BBF9A168122056
:1062C80001F0B7F9E168162001F0B3F921691A2045
:1062D80001F0AFF961691E2001F0ABF9082042F620
:1062E8009641BDE8104001F087B900BFB40E002008
:1062F8002DE9F04F0346A7B0B0F800C01C89868886
:10630800DF885D89CDF810C0B249B0F802C0B3F893
:106318000C90B3F80E80CDF824C00FFA84FB30B28D
:1063280001220FFA87FE0BEB000C0A7629B20FFA4E
:1063380089FACDF888C001EB0E0C0FFA88F2CDF877
:1063480090C00AEB0B0CCDF830C002EB010CCDF875
:1063580058C0B3F810C05B8ACDF800C00FFA8CFCA7
:1063680006910CEB00010A9102930CEB0A011BB297
:10637800239103EB0E010E9199182591049900FAC7
:1063880081F0584450446044DDF824C006990EFA60
:106398008CFEDDF810C01FFA80FB1CFB0CF08E444D
:1063A80016FB0600964414FB0400009A19FB09002A
:1063B8009E4412FB02001FFA8EFA0AF08BFFDDF8EA
:1063C80024C0029ACDE912011CFB0CF017FB070050
:1063D80015FB050018FB080012FB02000AF07AFF03
:1063E800DDF824C0029ACDE9140104991CFB01F3DD
:1063F80017FB063615FB0466009B18FB096612FBA3
:1064080003600AF067FFDDE91423CDE90001DDE947
:1064180012010AF0D5FF04460D46DDE900010246E7
:106428000B460AF0CDFF02460B46204629460AF0E5
:1064380013FECDE9180158460AF05CFFCDE91001BA
:10644800DDE91023DDE900010AF0BAFFCDE9060114
:1064580050460AF04FFF804689464246DDE9120160
:106468004B460AF0ADFFDDE91023CDE91C01DDE95B
:1064780014010AF0A5FF002206460F46564BDDE937
:1064880018010AF09DFF424604460D464B46DDE9D9
:1064980006010AF095FF02460B460AF0DFFD0246A8
:1064A8000B46204629460AF0D9FD424604460D46C9
:1064B8004B46DDE91C010AF083FF02460B462046E5
:1064C80029460AF0C9FDDDE9102304460D46304689
:1064D80039460AF075FF02460B46204629460AF05F
:1064E800BBFDDDF828C0CDE902014FEA8C10DDF8CC
:1064F80030C000EB0C20DDF810C0A0241CFB040009
:106508000AF0E8FEDDF838C0CDE90A014FEA8C1040
:10651800DDF858C000EB0C20DDF824C01CFB04009B
:106528000AF0D8FECDE90C0150460AF0D3FEDDE9A9
:106538001023CDE91601DDE90C010AF041FF4246BE
:10654800CDE91E014B46DDE90A010AF039FF424652
:10655800CDE920014B46DDE900010AF031FF324662
:106568003B460AF079FDCDE90E0158460AF0B2FE25
:10657800DDE91C23CDE91A01DDE906010AF06CFD0D
:10658800DDF88CC0C024CDE9060104FB0CF0DDF871
:1065980088C0302505FB0C00DDF810C078261CFBF0
:1065A80006000AF097FEDDF894C0824604FB0CF062
:1065B800DDF890C005FB0C00DDF824C01CFB0600CC
:1065C8008B460AF087FEDDE9102306460F460AF0DF
:1065D800F7FE03E0B40E0020000014404246CDE967
:1065E80004014B46504659460AF0EAFEDDE91423F9
:1065F80080468946DDE90A010AF0E2FEDDE900236A
:1066080004460D46DDE90C010AF0DAFE02460B46A7
:10661800204629460AF020FD0022A14B0AF0D0FEB0
:10662800DDE9202304460D46DDE91E010AF014FDCC
:1066380002460B46DDE916010AF0C2FE02460B4689
:10664800204629460AF00AFD002204460D46954BCD
:10665800DDE90E010AF0B4FE02460B462046294643
:106668000AF0FCFCDDE902230AF0D4FF88A3D3E991
:1066780000230AF0A5FE0BF03DF98B490860DDE91F
:106688001223DDE90C010AF09BFEDDE90023044634
:106698000D46DDE90A010AF093FE02460B46204644
:1066A80029460AF0D9FC00227D4B0AF089FEDDE973
:1066B8001E2304460D46DDE920010AF0CDFC024602
:1066C8000B46DDE91A010AF07BFE02460B4620461E
:1066D80029460AF0C3FC002204460D46714BDDE949
:1066E80006010AF06DFE02460B46204629460AF0CE
:1066F800B5FCDDE902230AF08DFF65A3D3E9002389
:106708000AF05EFE0BF0F6F8674A5060DDE90E23EA
:10671800DDE90A010AF054FEDDE9062304460D46C8
:10672800DDE90C010AF04CFE02460B4620462946DC
:106738000AF094FC002204460D465A4BDDE9180184
:106748000AF03EFE02460B46204629460AF086FC21
:10675800DDE902230AF05EFF4DA3D3E900230AF026
:106768002FFE0BF0C7F8504B59469860DDE914230B
:1067780050460AF025FEDDE9002304460D46304662
:1067880039460AF01DFE02460B46204629460AF005
:1067980063FC0022424B0AF013FE424604460D46B3
:1067A8004B46DDE904010AF057FC02460B46DDE9D9
:1067B80016010AF005FE02460B46204629460AF055
:1067C8004DFC35A3D3E9002304460D46DDE90E014F
:1067D8000AF0F6FD02460B46204629460AF03EFC22
:1067E800DDE902230AF016FF29A3D3E900230AF002
:1067F800E7FD0BF07FF8DFF8B0C0DDE91223CCF835
:106808000C00394630460AF0DBFDDDE9002304467A
:106818000D46504659460AF0D3FD02460B4620461F
:1068280029460AF019FC00221D4B0AF0C9FDDDE9D2
:10683800042304460D46404649460AF00DFC02462C
:106848000B46DDE91A010AF0BBFD02460B4620465D
:1068580029460AF003FC10A3D3E9002304460D4699
:10686800DDE906010AF0ACFD02460B462046294642
:106878000AF0F4FBDDE902230AF0CCFE04A3D3E915
:1068880000230AF09DFD0BF035F8074908610DE07B
:106898000000000080842E410000000000C08240FB
:1068A8000000144000008940B40E0020DDE90E23EA
:1068B800504659460AF084FDDDE9062304460D4694
:1068C800304639460AF07CFD02460B4620462946EA
:1068D8000AF0C4FB11A3D3E9002304460D46DDE901
:1068E80018010AF06DFD02460B46204629460AF0BB
:1068F800B5FBDDE902230AF08DFE0AA3D3E90023E4
:106908000AF05EFD0AF0F6FF034A506127B0BDE8C1
:10691800F04FC9E4AFF30080B40E0020000000007F
:1069280000C082400000000080842E41AFF3008048
:10693800064B074A596811601969064A1160D969F6
:10694800054A11609A6A054B1A6070479401002045
:10695800B4280020D42E0020A82E00206028002073
:10696800014B1878704700BFD00E0020032808B5E7
:1069780005D90548054A064B7321FDF763FE0C232C
:106988005843044B185808BDBADE05080099040896
:10699800D4DE050894010020032808B505D9064867
:1069A800064A074B7821FDF74DFE064B0C2202FBE9
:1069B8000030406808BD00BFBADE05081099040819
:1069C800D4DE050894010020034B044A1B780C21EF
:1069D80001FB032398687047D00E00209401002023
:1069E800034B044A1B780C2000FB03239960704773
:1069F800D00E002094010020144B1B78012B10B5F9
:106A0800134B144C0ED11968C82000F012FE2168EF
:106A1800CC2000F00EFE104BD020196800F009FEC3
:106A2800D4200DE01968D82000F003FE2168DC208E
:106A380000F0FFFD084BE020196800F0FAFDE420A3
:106A4800064B1968BDE8104000F0F3BD800F002028
:106A5800B4280020D42E0020A82E00206028002072
:106A6800144B1B78012B10B5134C0FD1C82000F024
:106A7800F9FD2060CC2000F0F5FD104B1860D02007
:106A880000F0F0FD0E4B1860D4200EE0D82000F086
:106A9800E9FD2060DC2000F0E5FD084B1860E020EF
:106AA80000F0E0FD064B1860E42000F0DBFD054B2C
:106AB800186010BD800F0020B4280020D42E0020BC
:106AC800A82E00206028002008B504F065FD10B14C
:106AD800BDE80840C4E7BDE8084029E70148FAF7DF
:106AE80006BE00BFBC1800200148FAF700BE00BF70
:106AF800BC1800200148FAF7FABD00BFBC180020F6
:106B08000148FAF7F4BD00BFBC180020032808B5F7
:106B180005D91648164A174B4F21FDF793FD164B1A
:106B28001870164B1870164B012202281A70154B54
:106B38000FD0032813D0904205D0134A12681A6068
:106B4800BDE80840CAE7114A12681A60BDE8084063
:106B5800CAE70F4A12681A60BDE80840CAE70D4A3A
:106B680012681A60BDE80840CAE700BFBADE050827
:106B780021990408FEDE0508D00E0020AB2800206D
:106B8800DC0E0020940200208C02002088020020E5
:106B98008402002080020020064B07495960C0216A
:106BA800002219721E211A70D9601A745A611A7655
:106BB800DA617047B01B002040787D0110B50321D1
:106BC800FF22C02001F0AEFB1F4C10212060802264
:106BD800C02001F0A7FB112120608022C02001F015
:106BE800A1FB122120608022C02001F09BFB132111
:106BF80020608022C02001F095FB142120608022B3
:106C0800C02001F08FFB152120608022C02001F0F8
:106C180089FB802220601621C02001F083FB2060C0
:106C2800C0201721802201F07DFB2060074CC02086
:106C3800227AB72101F076FB00232374636123765F
:106C4800E3610123237010BD8C280020B01B0020B5
:106C580038B5C0200321FF2201F064FB0B4D00244E
:106C68002B19615D5A78C020023401F05BFBC82CF7
:106C7800F6D1B121AC22C02001F054FBC020032181
:106C8800002201F04FFB002038BD00BF35990408F1
:106C98002DE9F34706460F4692461D461AB90C1FC2
:106CA800E401914635E005EE902A06EE903AB8EEFA
:106CB800657AF8EE667AFC01C7EE277AA4F50074C7
:106CC8009FED5C7A67EE877A17EE900A0AF024FB4C
:106CD80041EC100B0CF0CCFB59EC108B49464046AC
:106CE8000AF030FE24184FEACA100AF0F3FACDE988
:106CF800000128460AF0EEFA4B4642460AF060FBCD
:106D080002460B46DDE900010AF0A6F90AF01AFE70
:106D18008146002E14BF4FF022084FF01A08C5F321
:106D280007224146C02001F0FDFA08F10101EAB24C
:106D3800C02001F0F7FAC4F3014208F10201C020B3
:106D480001F0F0FAC4F3072208F10301C02001F0B2
:106D5800E9FAE2B208F10401C02001F0E3FAC9F34C
:106D6800034305F4702243EA123208F10501C020FA
:106D780001F0D8FA08F10601C9F30722C02001F092
:106D8800D1FA08F107015FFA89F2C02001F0CAFAC6
:106D9800C020B121A02201F0C5FA07EE107A264CD6
:106DA800F8EEC77A0EBBD4ED015A06EE90AAB8EEFB
:106DB800657A05EE905AB8EE666AF8EE656A0123C0
:106DC800C6EE266A237477EEA67A67EE277A17EE60
:106DD800900A0AF0A1FA41EC100B0CF049FB51ECB7
:106DE800100B0AF0AFFD606120E005EE90AAD4ED2B
:106DF800016AB8EE656A05EE905AB8EE667AF8EE62
:106E0800656A0123C6EE266A237677EEA67A67EED0
:106E1800277A17EE900A0AF07FFA41EC100B0CF073
:106E280027FB51EC100B0AF08DFDE0610020BDE856
:106E3800FC8700BF00000043B01B00200022012394
:106E480026E7012838B50D4604D002280CBF3C249B
:106E58002C2400E034242146C02001F0DDFA05F09E
:106E6800070200F00F0040EA02122146C020BDE8E8
:106E7800384001F057BA2DE9F3470A9C1D460746EA
:106E88008A461646524B01E06D0864089C42FBD8BE
:106E98002DB906F10076043EF601A94634E006EE67
:106EA800905AB8EE667A06EE904AF8EE667AF601DF
:106EB800C7EE277AA6F500769FED467A67EE877AC1
:106EC80017EE900A0AF028FA41EC100B0CF0D0FAF1
:106ED80059EC108B494640460AF034FD3618E80153
:106EE8000AF0F8F9CDE9000120460AF0F3F94B461B
:106EF80042460AF065FA02460B46DDE900010AF04F
:106F0800ABF80AF01FFD8146022F9BBF324BDB19FD
:106F18004FF0000893F8C880C4F307224146C02008
:106F280001F000FA08F10101E2B2C9B2C02001F093
:106F3800F9F908F10201C9B2C6F30142C02001F013
:106F4800F1F908F10301C9B2C6F30722C02001F024
:106F5800E9F908F10401C9B2F2B2C02001F0E2F97E
:106F680004F47024C9F3034308F1050143EA143219
:106F7800C9B2C02001F0D6F908F10601C9B2C9F3B7
:106F88000722C02008F1070801F0CCF95FFA89F25E
:106F98005FFA88F1C02001F0C5F9BAF1010F0CBF02
:106FA8002F220F220DB942F04002012F06D002D342
:106FB800022F0AD105E0C020102104E0C0201121D1
:106FC80001E0C020122101F0ADF90020BDE8FC87E6
:106FD800FFFF0F00000000433599040807B501239F
:106FE80000930023FFF747FF0EBD00280CBFFF22C8
:106FF800002208B5C020032101F094F9002008BD43
:1070080008B5C020B121AC2201F08CF9002008BDE0
:1070180008B50420012108F0CDFD4FF4807001214E
:10702800BDE8084008F0F6BD07B502230093032326
:107038008DF804300348002369468DF8073008F0BE
:1070480011FA0EBD0008024030B5124D8BB0002475
:1070580006A8069407940894099407F0D1FB0094B5
:107068008DF804408DF80540029403940494284652
:10707800012469468DF8144007F093FB28460B213C
:107088002246062307F008FC2846214607F0D2FBD3
:107098000BB030BD0020014010B50021044601228C
:1070A800302001F03FF9C0B9012001F059FB002C54
:1070B800B8BF4034E4B210212246302001F032F942
:1070C800012001F04DFB30201121224601F02AF960
:1070D8000120BDE8104001F043BB10BD10B50021F0
:1070E80004460122302001F01DF9C0B9012001F049
:1070F80037FB002CB8BF4034E4B2122122463020BE
:1071080001F010F9012001F02BFB30201321224659
:1071180001F008F90120BDE8104001F021BB10BDC5
:1071280038B5012205460C463020002101F0FAF856
:10713800F0B9012001F014FB25EAE5725F2AA8BF27
:107148005F223B21D2B2302001F0ECF8012001F09F
:1071580007FB24EAE4725F2AA8BF5F22D2B230207C
:107168003C2101F0DFF80120BDE8384001F0F8BA11
:1071780038BD302810B504460ADC10F17F0F02DB59
:10718800002802DB05E06FF07E0404F5807400E05F
:107198003024002130200A4601F0C4F8A8B90120A3
:1071A800E4B201F0DDFA41212246302001F0BAF8BC
:1071B800012001F0D5FA30204221224601F0B2F830
:1071C8000120BDE8104001F0CBBA10BD282810B549
:1071D800044609DC10F1180F02DB002802DB04E08A
:1071E8006FF017047F3400E02824002130200A467D
:1071F80001F098F8A8B90120E4B201F0B1FA5321DE
:107208002246302001F08EF8012001F0A9FA302042
:107218005421224601F086F80120BDE8104001F013
:107228009FBA10BD08B530200021012201F07AF87C
:1072380060B9012001F094FA30203321402201F096
:1072480071F80120BDE8084001F08ABA08BD10B500
:1072580030200021012201F065F8044660B90120C0
:1072680001F07EFA30203321224601F05BF801203C
:10727800BDE8104001F074BA10BD10B530200021EF
:10728800012201F04FF80446A0B9012001F068FA84
:1072980034212246302001F045F8012001F060FA3F
:1072A80030203721224601F03DF80120BDE810408A
:1072B80001F056BA10BD4020EEE640200EE708B5B2
:1072C80000210122302001F02DF8012001F048FAB8
:1072D80030203421024601F025F8012001F040FA5F
:1072E80030203721024601F01DF80120BDE8084092
:1072F80001F036BA08B500210122302001F012F859
:10730800012001F02DFA302034210C2201F00AF876
:107318000120BDE8084001F023BA00000000000089
:107328002DE9F04F984B994A1968994B002914BFD9
:1073380091469946974B2DED048BC3F80090964BD8
:107348000025002287B01A80AA46AB46A8465AE014
:10735800A2004046CDF804C0029209F0DDFF0746BE
:10736800584601F1004609F0D7FF02460B46384659
:10737800314609F071FE39F9243007EE103AF8EE7B
:10738800C77A064617EE900A0F4609F0C5FF02466F
:107398000B463046394609F061FE0AF0F3FA074613
:1073A800504609F0B9FF0446284601F1004609F0A5
:1073B800B3FFCDE90401DDE904232046314609F095
:1073C8004BFE029A09EB02030446B3F9023007EEBA
:1073D800103AF8EEC77A0D4617EE900A09F09CFFAE
:1073E80002460B462046294609F038FE0AF0CAFA3A
:1073F800DDF804C0684A0CF1010CC3465546A2F8F2
:1074080000C08246B846644BB3F800C00FFA8CF44B
:10741800B32C9DDD584609F07FFFCDE902014046B7
:1074280009F07AFF002206460F465C4BDDE90201AF
:1074380009F0C6FF02460B463046394609F00EFEF3
:107448000022574B0AF0E6F80AF09CFA4CA3D3E95D
:10745800002309EE900ADDE9020109F0B1FF0022DC
:107468004F4B0AF0D7F80AF08DFA09EE100A2846B1
:1074780009F052FF044650460D4609F04DFF002220
:1074880006460F4620462946444B09F099FF024616
:107498000B463046394609F0E1FD0022404B0AF020
:1074A800B9F80AF06FFA36A3D3E9002308EE900A78
:1074B8002946204609F084FF0022394B0AF0AAF831
:1074C8000AF060FA08EE100A69EE287A58EE297A6E
:1074D80017EE900A09F020FF68EE097A48EEA97ABB
:1074E800044617EE900A0D4609F016FF45EC104BBE
:1074F80041EC110B0CF0C0F851EC100B0AF042FAF9
:1075080028EE088A08EEA88A07EE100A254B264CB2
:10751800F1EE477AC3ED007A18EE100A09F0FCFE86
:1075280041EC100B0CF0B6F929EE099A51EC100B4E
:1075380009EEA99A0AF026FA206019EE100A09F055
:10754800EBFE41EC100B0CF0A5F951EC100B0AF016
:1075580019FAD4ED007A07EE100A87EE877A134BF2
:107568001860134BFDEEE77A83ED007A114BC3EDFB
:10757800007A07B0BDEC048BBDE8F08FAFF3008054
:10758800912B50E67AB6EB3FD81B00205E250020F1
:10759800BE1F0020D41B0020E01B00200000E03F9D
:1075A80000005940DC2E0020F82E0020EC2E002090
:1075B800E42E0020DC1B002010B5084C204607F004
:1075C8009EFB074B1860FFF7ABFE064B06490122EE
:1075D80020461A80BDE8104007F012BC1060024037
:1075E800D81B0020D20E002020800010014B186804
:1075F800704700BFDC1B002038B505460C46013536
:10760800C1F3072101F0BAF8A8B2E1B201F0B6F867
:1076180000B238BD38B5044600F0C6FF013405464F
:10762800A0B200F0C1FFEDB2C0B240EA052000B23E
:1076380038BD37B50B0E8DF804300B0C8DF80530BE
:107648000B0A8DF806308DF80710002400E0284654
:1076580001AB451CE15C013401F090F8042CADB29B
:10766800F5D13EBD37B5002400E02846451C00F0A2
:107678009BFF01ABADB2E0540134042CF5D19DF869
:1076880005009DF80430000440EA03609DF80730C7
:1076980018439DF8063040EA03203EBD37B5002365
:1076A8000193002400E02846451C00F07DFF01AB53
:1076B800ADB2E0540134042CF5D19DED010A3EBD74
:1076C80038B50446642001F04BF825786068AD00B1
:1076D800EDB2257007F02BFF237A40FA03F000F093
:1076E80003000543104B257005F00F055A5D6378BC
:1076F800D218D2B2D3B20132D2B2022A637001D800
:107708000022A2705BB2012B03DD0123A3700023CA
:10771800637094F90130013303DAFF23A370002367
:10772800637094F9020038BD009A0408F7B5042084
:107738000121234F08F03EFA02AD01214FF48040A9
:10774800012408F067FA00264FF4B07338466946FA
:1077580045F8083D8DF804608DF8074007F082FE73
:107768001020214608F026FA782369461548009328
:107778008DF804608DF8074007F074FE0420214658
:1077880008F018FA21464FF4804008F043FA1C2309
:107798003846694600938DF804608DF8074007F075
:1077A80061FE0220214608F005FAB02306488DF84C
:1077B800046069468DF80740009307F053FEFEBD4C
:1077C800000802400010024000040240802108B571
:1077D800034807F0A6FED0F1010038BF002008BD1D
:1077E8000004024008B54FF48071044807F099FE80
:1077F800D0F1010038BF002008BD00BF00080240DA
:1078080008B5FFF7E3FF08B1FFF7ECFFC0B208BD0A
:1078180070B500283AD01E4B1A7880181D4AC0B29D
:1078280092F90020187040B282421B4A02DD11789A
:107838000139197093F9001092F9002091FBF2F4C4
:1078480002FB14141549E4B21C700A88144B1A8000
:10785800144B154A18881080144A92F9000064B233
:10786800013094FBF0F200FB1240114C2688114CB9
:10787800258800FB065008800F4908880F490988A9
:1078880002FB00121A800E4B01221A7070BD00BF55
:107898007E3C0020B13800208D380020AE3C00200E
:1078A800D23800207C3C0020843A0020B03C0020E4
:1078B800E0390020143D0020403D0020623A0020BD
:1078C8008C380020F0B5264A264C00231370264A2F
:1078D80025681678254A12680FE0D45C2F197F783E
:1078E80017F0040F07D0302C02D12023135431E0B5
:1078F8001B4A137003E00133DBB29E42EDDA184BEA
:107908001B788342194B16D9A9B11A68164C312134
:10791800115430210BE01A681518125C2E2A19D060
:10792800303AD2B2092A88BF29700130C0B2227811
:107938008242F0DA0EE01B681A5C79B12E2A0DD06B
:107948005118C9B2392903D82F2998BF302100E02E
:1079580039211954BDE8F040FCF74CBCF0BD00BF1C
:10796800D40E0020CC040020343E0020A03C00208F
:1079780010B5642000F0F4FE7E48FFF7A1FE7E4BB0
:107988001B7804460A2B00F2D280DFE813F00B00C4
:107998000B00D0007100710034008700D000870010
:1079A8009000AA00FFF71EFF10B1F9F775FCBEE0C2
:1079B800724B1888724B1B88C01A724B1B8890FB3D
:1079C800F3F0714B1A88714B1B88D31A704A1288CE
:1079D80093FBF2F3DBB2C0B2032B00F2A580DFE821
:1079E80003F0020406086B4A3FE06B4A3DE06B4A2D
:1079F8003BE06B4A39E0FFF7F5FED8B100210A22D7
:107A080068480FF0E7FB684B002118600A226748B6
:107A18000FF0E0FB664B18600420FEF729F996206A
:107A28000521644A0023FEF75BF90020FEF720F9E0
:107A380006F006FB514B1888514B1B88C01A514B56
:107A48001B8890FBF3F0504B1A88504B1B88D31AB5
:107A58004F4A128893FBF2F3DBB2C0B213B1012B89
:107A680062D101E04F4A00E0504A534B1A605BE094
:107A780000285CD0514B1A7806DD0132D2B20F2AA9
:107A88001A7008D9102205E0013AD2B2102A1A70E9
:107A980001D900221A70F9F7FFFE48E0002846D005
:107AA800474B93F90020002A41D118703FE0FFF7B7
:107AB80099FEA0B1002143480FF0D8FA424B0420A8
:107AC80083ED000AFEF7D4F8B42005213F4A0023CD
:107AD800FEF706F9FAF7E8FA0020FEF7C9F8394A7E
:107AE80016E0FFF77FFE90B1002139480FF0BEFA8B
:107AF800384B042083ED000AFEF7BAF896200521DA
:107B0800324A0023FEF7ECF80020FEF7B1F8304ABD
:107B1800294B1A60194B1888194B1B88C01A194B26
:107B28001B8890FBF3F0C0B22146FFF7CBFE2A4832
:107B3800FFF7C6FD104B1B78013B0A2B19D8DFE86D
:107B480003F015181818150A0A1806060A00234B18
:107B58001B78022B0AD10028214B01D1187010BDC7
:107B680002DD01221A7010BDFF22FBE7BDE81040BC
:107B78004EE610BDC401002034280020AE3C002091
:107B8800143D0020E03900207C3C0020623A0020AF
:107B9800403D002078280020A0280020B62E002094
:107BA800642800201C3D002078020020903C002022
:107BB8007402002046DF0508A03C0020B2280020FF
:107BC800AC3C0020A4380020D403002056DF050870
:107BD800C8380020D0030020D0010020A43A00209B
:107BE800E91B002010B58CB01E490F2268460EF024
:107BF800DFF81D490F2204A80EF0DAF81B490F22FE
:107C080008A80EF0D5F800210822302000F08AFBE1
:107C1800012000F0A5FD002404AB1DF80420E15C60
:107C2800302000F07FFB0134012000F099FD0F2C7B
:107C3800F2D100210922302000F074FB012000F06D
:107C48008FFD002408AB1DF80420E15C302000F013
:107C580069FB0134012000F083FD0F2CF2D10CB038
:107C680010BD00BF129A0408219A0408309A04082B
:107C780010B58CB01E490F2268460EF099F81D49C0
:107C88000F2204A80EF094F81B490F2208A80EF042
:107C98008FF800210822302000F044FB012000F07A
:107CA8005FFD002404AB1DF80420E15C302000F0E7
:107CB80039FB0134012000F053FD0F2CF2D10021D3
:107CC8000922302000F02EFB012000F049FD00249D
:107CD80008AB1DF80420E15C302000F023FB0134E0
:107CE800012000F03DFD0F2CF2D10CB010BD00BFFB
:107CF8003F9A04084E9A04085D9A040810B58CB09F
:107D08001E490F2268460EF053F81D490F2204A899
:107D18000EF04EF81B490F2208A80EF049F8002172
:107D28000822302000F0FEFA012000F019FD00249E
:107D380004AB1DF80420E15C302000F0F3FA0134B4
:107D4800012000F00DFD0F2CF2D100210922302076
:107D580000F0E8FA012000F003FD002408AB1DF84C
:107D68000420E15C302000F0DDFA0134012000F04D
:107D7800F7FC0F2CF2D10CB010BD00BF6C9A0408B0
:107D88007B9A04088A9A040807B50220012107F0A3
:107D980011FF012300938DF8043002238DF805307C
:107DA8000448002369468DF806308DF8073007F03F
:107DB80059FB0EBD0004024010B5084C01210022F9
:107DC800204607F0C4FB40F2FF4000F0C9FC012147
:107DD80020460A46BDE8104007F0B9BB000402403F
:107DE80008B5FFF7E9FF00210A46302000F09AFAAB
:107DF800012000F0B5FC01210A46302000F092FA7B
:107E0800012000F0ADFC00210122302000F08AFAA8
:107E1800012000F0A5FC01210822302000F082FAA0
:107E2800012000F09DFC02210122302000F07AFAA6
:107E3800012000F095FC00210A46302000F072FA7B
:107E4800012000F08DFC1B21CD22302000F06AFAC1
:107E5800012000F085FC04210322302000F062FAA2
:107E6800012000F07DFC06210922302000F05AFA9A
:107E7800012000F075FC07210822302000F052FA9A
:107E8800012000F06DFC08217022302000F04AFA31
:107E9800012000F065FC1E213020B02200F042FADB
:107EA800012000F05DFC05219122302000F03AFA13
:107EB800012000F055FC0D210322302000F032FA99
:107EC800012000F04DFC0E210022302000F02AFA9B
:107ED800012000F045FC14218022302000F022FA15
:107EE800012000F03DFC0B218822302000F01AFA16
:107EF800012000F035FC0C218222302000F012FA1B
:107F0800012000F02DFC12218822302000F00AFA0E
:107F1800012000F025FC13218C22302000F002FA09
:107F2800012000F01DFC00210A46302000F0FAF97B
:107F3800012000F015FC3D210222302000F0F2F96A
:107F4800012000F00DFCFFF74DFEFFF791FEFFF753
:107F5800D5FE30200021012200F0E4F9012000F0D4
:107F6800FFFB3D216422302000F0DCF9012000F005
:107F7800F7FB03210022302000F0D4F9012000F0A3
:107F8800EFFB04210022302000F0CCF9012000F0A2
:107F9800E7FB00210122302000F0C4F9012000F0A5
:107FA800DFFB0C210822302000F0BCF9012000F092
:107FB800D7FB0D210822302000F0B4F9012000F091
:107FC800CFFB0E210822302000F0ACF9012000F090
:107FD800C7FB0F210822302000F0A4F9012000F08F
:107FE800BFFB00210A46302000F09CF9012000F078
:107FF800B7FB02224021302000F094F9012000F064
:10800800AFFB30204121002200F08CF9012000F064
:10801800A7FB3F21D422302000F084F9012000F092
:108028009FFB00210122302000F07CF9012000F0A4
:1080380097FB10210F22302000F074F9012000F086
:108048008FFB11210F22302000F06CF9012000F085
:1080580087FB12210022302000F064F9012000F093
:108068007FFB13210022302000F05CF9012000F092
:1080780077FB09213C22302000F054F9012000F060
:108088006FFB00210122302000F04CF9012000F0A4
:1080980067FB30203421024600F044F9012000F04B
:1080A8005FFB30203721024600F03CF9012000F048
:1080B80057FB36210322302000F034F9012000F06C
:1080C8004FFB39210322302000F02CF9012000F069
:1080D80047FB3B213C22302000F024F9012000F02E
:1080E8003FFB3C210A46302000F01CF9012000F03B
:1080F80037FB00210A46302000F014F9012000F077
:108108002FFB5121C022302000F00CF9012000F093
:1081180027FB52213020002200F004F90120BDE89D
:10812800084000F01DBB00BF2DE9F04F454E464DFD
:1081380093B001214FF4001007F03CFD304606F0E3
:10814800DFFC4FF0C0630293404B0393404B002485
:1081580004934FF4B4794FF400334FF480684FF42C
:1081680000674FF4005A4FF4807B304602A90C9305
:1081780001930997CDF8189005940794CDF82080BD
:10818800CDF828A0CDF82CB00D9406F045FD224678
:108198003046304906F09BFD3046012106F0A1FD2E
:1081A80001210A464FF0402007F072FF284606F0EA
:1081B800A7FC294A019B0392284A0C93049228465B
:1081C800402202A9059209970294CDF818900794C5
:1081D800CDF82080CDF828A0CDF82CB00D9406F06D
:1081E8001BFD224628461E4906F071FD284601213E
:1081F80006F077FD42F2107701220221194807F0B4
:1082080047FF384600F0ACFA3046012106F03FFD42
:108218000121284606F03BFD384600F0A1FA0B2361
:108228008DF8443011A801238DF845408DF846405B
:108238008DF8473000F0B2FC384600F091FA13B0E0
:10824800BDE8F08F10600240886002400C4000409A
:108258005E250020BE1F00200C3C00408E2200201E
:10826800EE1C0020003C004002481021012206F0CC
:1082780085BD00BF1060024013B50220012107F040
:1082880099FC4FF410730E4C009302238DF80430C0
:108298008DF8053001238DF8063020460023694605
:1082A8008DF8073007F0DEF820460621042207F093
:1082B80059F920460921042207F054F91CBD00BFD2
:1082C8000004024030B5154D85B001214FF400106F
:1082D80007F094FC284607F05BF90023ADF804305A
:1082E8004BF6FF73ADF806303323ADF808304FF482
:1082F8008063ADF80A304FF48043ADF80C3004AC1D
:10830800074B2846012144F8103D07F0E3F92846B9
:10831800694607F06BF905B030BD00BF0054004056
:10832800801A060073B54FF4961306460D46144698
:10833800019304E0019B5A1E0192002B57D031484B
:108348004FF4003107F0DEFA0028F3D12D4801215F
:1083580007F0CCF94FF48053019304E0019B5A1EB7
:108368000192002B45D02748274907F0B6FA002884
:10837800F4D024483146002207F0D0F94FF4805356
:10838800019304E0019B5A1E0192002B33D01D4833
:108398001E4907F0A2FA0028F4D01A48294607F027
:1083A80040FA4FF48053019303E0019B5A1E019257
:1083B8001BB31448164907F090FA0028F5D0114865
:1083C800214607F02EFA4FF49613019303E0019B20
:1083D8005A1E01929BB10B480E4907F093FA0028E8
:1083E800F5D00848012107F08DF9002008E00120A8
:1083F80006E0022004E0032002E0042000E005205B
:108408007CBD00BF0054004001000300820007004B
:10841800800007000400001037B54FF49613044697
:108428000D46019305E0019B5A1E0192002B00F0B6
:108438009B8056484FF4003107F064FA0028F2D1C7
:108448005248012107F052F94FF48053019305E097
:10845800019B5A1E0192002B00F088804B484C4922
:1084680007F03BFA0028F3D048482146002207F0DD
:1084780055F94FF48053019304E0019B5A1E019271
:10848800002B75D04148434907F027FA0028F4D05B
:108498003E48294607F0C5F94FF48053019304E09C
:1084A800019B5A1E0192002B64D038483A4907F0C4
:1084B80029FA0028F4D03548012107F017F94FF4BC
:1084C8008053019304E0019B5A1E0192002B53D064
:1084D8002E482F4907F001FA0028F4D02B482146EE
:1084E800012207F01BF94FF48053019304E0019B2C
:1084F8005A1E0192002B41D0244C2849204607F0EF
:1085080001FA0028F3D02046002107F00FF9204691
:108518000121238B07F0F6F84FF48053019304E010
:10852800019B5A1E0192002B2AD018481C4907F0BB
:10853800E9F90028F4D0154807F075F94FF480538D
:108548000193124A03E0019B591E0191D3B113888C
:108558009B05F8D4012104460C4807F0E7F80B48BE
:10856800104907F0E9F90EE001240CE002240AE0C2
:10857800032408E0042406E0052404E0062402E0BD
:10858800072400E0082420463EBD00BF00540040F8
:108598000100030082000700040000100200001020
:1085A800400000100004001013B54FF49613044661
:1085B800019305E0019B5A1E0192002B00F0AF8049
:1085C80060484FF4003107F09DF90028F2D15D486A
:1085D800012107F08BF84FF48053019305E0019BCC
:1085E8005A1E0192002B00F09C805648564907F00D
:1085F80074F90028F3D05348A021002207F08EF820
:108608004FF48053019305E0019B5A1E0192002B01
:1086180000F089804B484D4907F05FF90028F3D0F6
:10862800210A484807F0FDF84FF48053019304E00D
:10863800019B5A1E0192002B77D04248444907F00B
:1086480061F90028F4D0E1B23E4807F0EAF84FF4A7
:108658008053019304E0019B5A1E0192002B66D0BF
:1086680038483B4907F04EF90028F4D03548012135
:1086780007F03CF84FF48053019304E0019B5A1E25
:108688000192002B55D02F482F4907F026F90028D2
:10869800F4D02C48A121012207F040F84FF4805370
:1086A800019304E0019B5A1E0192002B43D0254CF4
:1086B8002849204607F026F90028F3D02046002153
:1086C80007F034F820460121238B07F01BF84FF4FC
:1086D8008053019304E0019B5A1E0192002B2CD079
:1086E80018481D4907F00EF90028F4D0154807F07E
:1086F8009AF84FF480530193124A03E0019B591EE4
:108708000191E3B113889905F8D4012104460D4875
:1087180007F00CF80B48114907F00EF910E0012496
:108728000EE002240CE003240AE0042408E00524F7
:1087380006E0062404E0072402E0082400E00924F7
:1087480020461CBD005400400100030082000700C1
:108758000400001002000010400000100004001087
:1087680082B0002304E0019B01330193009B013395
:108778000093009B8342F6D302B0704737B54FF49D
:10878800805304460D46019304E0019B5A1E019252
:10879800002B6DD03C484FF4003107F0B3F80028A7
:1087A800F3D13948012106F0A1FF4FF4805301931A
:1087B80004E0019B5A1E0192002B5BD032483349DA
:1087C80007F08BF80028F4D02F48A021002206F0EB
:1087D800A5FF4FF48053019304E0019B5A1E0192B8
:1087E800002B49D028482A4907F077F80028F4D008
:1087F800210A254807F015F84FF48053019304E047
:10880800019B5A1E0192002B38D01F48214907F0BE
:1088180064F80028F4D0E1B21B4807F002F84FF4DE
:108828008053019303E0019B5A1E019243B31648FB
:10883800184907F052F80028F5D01348294606F0E1
:10884800F0FF4FF49613019303E0019B5A1E019227
:10885800C3B10D48104907F055F80028F5D00A486B
:10886800012106F04FFF0D48FFF77AFF00200AE0CC
:10887800012008E0022006E0032004E0042002E0D2
:10888800052000E006203EBD005400400100030022
:10889800820007008000070004000010A086010085
:1088A800F7B54FF4805304460D461646019304E08D
:1088B800019B5A1E0192002B74D040484FF400319E
:1088C80007F020F80028F3D13C48012106F00EFFFC
:1088D8004FF48053019304E0019B5A1E0192002B30
:1088E80062D03648364906F0F8FF0028F4D03348FD
:1088F800A021002206F012FF4FF48053019304E0F8
:10890800019B5A1E0192002B50D02C482D4906F08D
:10891800E4FF0028F4D0210A284806F082FF4FF42B
:108928008053019304E0019B5A1E0192002B3FD013
:108938002248254906F0D1FF0028F4D0E1B21F48AB
:1089480006F06FFF4FF48053019304E0019B5A1E19
:108958000192002B2ED019481B4906F0BEFF0028B3
:10896800F4D000244FF4961710E0295D134806F060
:1089780058FF019703E0019B5A1E0192E3B10F488B
:10898800124906F0BFFF0028F5D00134E3B2B34224
:10899800EBD30A48012106F0B5FE0D48FFF7E0FECB
:1089A80000200AE0012008E0022006E0032004E09D
:1089B800042002E0052000E00620FEBD005400402F
:1089C8000100030082000700800007000400001077
:1089D800A086010013B50520012107F0EBF8184C1B
:1089E8004FF4E053009302238DF804308DF80530DE
:1089F8002046002369468DF806308DF8073006F0CA
:108A080031FD20460A21062206F0ACFD20460C2145
:108A1800062206F0A7FD062220460B21A4F50064D5
:108A280006F0A0FD4FF4004320466946009306F087
:108A380019FD20460F21062206F094FD1CBD00BF3B
:108A4800000802401FB50446FFF79EF9FFF73AFCFD
:108A5800FFF7C6F9FFF7BEFF01214FF4004007F00A
:108A6800CDF802940F4C1023ADF8023020460023B5
:108A78006946ADF80430ADF80C30ADF80030ADF80B
:108A8800063007F0EAF969464FF0402007F0B9FAD6
:108A98002046012107F069FA4FF04020012107F034
:108AA80064FA1FBD003C004082B0002304E0019B33
:108AB80001330193009B01330093009B8342F6D35B
:108AC80002B0704707B50420012107F073F80121AF
:108AD8004FF4804007F09EF84FF400730093002392
:108AE8008DF804300348012369468DF8073006F0F5
:108AF800B9FC0EBD000802400D4B07B51A680D48B9
:108B08004FF47A73B2FBF3F20B4B013A5A600B4AFB
:108B1800F02182F8231000229A6007221A60084B7D
:108B2800084A00930121084B02F022F80EBD00BF4D
:108B380098020020B828002010E000E000ED00E0D6
:108B4800B40300209803002000030020054B1A6896
:108B580012B11A68013A1A60034B1A6801321A6096
:108B6800704700BF742800209028002082B0044B72
:108B78000190019A1A601A68002AFCD102B0704765
:108B880074280020704700BF40F0BE60024B40F4DC
:108B98002020D860704700BF00ED00E0C37810B512
:108BA80003B3164B4278DB688478DB43C3F30223B4
:108BB800C3F10401C9B202FA01F10F2242FA03F229
:108BC800C9B222400A430E4B01781201CB18D2B227
:108BD80083F8002303780122590903F01F0302FADE
:108BE80003F307E003780122590903F01F0302FA8F
:108BF80003F32031024A42F8213010BD00ED00E0B5
:108C080000E100E021F0604121F07F01014B0843C1
:108C18009860704700ED00E0044B1A6909B11043F1
:108C280001E022EA00001861704700BF00ED00E093
:108C3800044B1A6804280CBF42F0040222F0040214
:108C48001A60704710E000E0034A044B1A60044AB7
:108C5800044B1A60704700BF00A00C46842800200F
:108C6800920A064070280020034B00221A60034A2B
:108C7800034B1A60E8E700BFF02E002000A00C4666
:108C88003C28002007EE100A024BF8EEC77AC3ED25
:108C9800007A70473C28002038B510EE100A08F01A
:108CA8003BFB0DA3D3E9002308F08AFB084B0446DD
:108CB80018680D4608F030FB0B4602462946204648
:108CC80008F0A8FC08F05EFE024B186038BD00BF33
:108CD8008428002070280020182D4454FB211940B6
:108CE800014B93ED000A7047E42E0020014B93EDF1
:108CF800000A7047DC2E0020014B93ED000A7047F4
:108D0800F42E0020014B93ED000A7047E02E00205E
:108D1800014B93ED000A7047F82E0020014B93EDAC
:108D2800000A7047EC2E002010B5FDF747FF002021
:108D3800012324210246FDF7ABFF114B1C780020CC
:108D4800012C05D10146FEF77CF82046002104E0FD
:108D58000721FEF776F801200721FEF772F8632253
:108D68001221C020FFF7DEFA02200121FEF769F880
:108D7800FEF746F90120BDE81040FEF736B900BFFE
:108D8800800F00200D4B1B78062B05D10C4B0D4A8C
:108D9800196812688A181A600B4B1B78012B084B4C
:108DA800196805D1094A914207DD01321A607047F6
:108DB800074A914201DD01321A60704734280020C9
:108DC800B02E002030280020800F00207FD1F0082E
:108DD800FF27ED080E4B1B78062B05D10D4B0E4ACD
:108DE800196812688A1A1A600C4B1B78012B094BF8
:108DF80005D10B4A1968914208DC1A6070471A6855
:108E0800B2F57A2FDCBF4FF47A221A60704700BFA0
:108E180034280020B02E002030280020800F0020A9
:108E280020A107002DE9F04F8DB00C460A90644848
:108E3800B0FBF1F008F04EFA41EC100B0AF018FB09
:108E480051EC100B08F07EFD10F0010F804618BFA2
:108E580000F1FF3804FB08F008F03CFA52A3D3E90C
:108E6800002308F0D7FB04460D4645EC104B0AF0EA
:108E7800FFFA57EC106B204632463B46294608F06D
:108E8800EBF8CDE902013946304608F05BFD48A30E
:108E9800D3E900230B90DDE9020108F00DFD00285D
:108EA80058D1012000264FF01509314607464FF0EA
:108EB800000A4FF0000B03E030463946069E049F37
:108EC800A7FB0A23541807FB0B333E4A43F100055E
:108ED8000023A242AB41CDE904453ED3A6FB0A23B9
:108EE800141806FB0B33374843F100050021A04254
:108EF800A941CDE9064530D3DDE902012EA3D3E926
:108F08000023049C069D08F0D7FC40BBDDE9022342
:108F180000202D4908F07EFB82468B464BEC10ABB7
:108F28000AF0A6FA5046594653EC102B8DED080B63
:108F380008F092F8CDE90201DDE9080108F0D0FF58
:108F480009F1FF395FFA89F982468B46B9F1000FBA
:108F5800B2D104E00125002401E035463C460B9AD5
:108F68000A9BD1B25BB9184622462B46FDF790FE04
:108F78000A980123009301464246034609E0224627
:108F88002B460120FDF784FE012000900146424651
:108F98000023FDF770FFFEF733F801200DB0BDE8A0
:108FA800F04FFEF722B800BF0000000084D77741D9
:108FB800956479E17FFDA53DBBBDD7D9DF7CDB3D5D
:108FC80000E9A435FFFF0F000000F03F224A234BC1
:108FD8001278012A10B5186009D1214A904201DDA2
:108FE80001321A601F4A1B6893420DDC0AE01E4AD0
:108FF800904201DD01321A601B68B3F57A2F03DC59
:109008004FF47A22154B1A60144B184A1968184BFA
:10901800184C1B68CB189342236018DC0020FFF71C
:1090280001FF01202168FFF7FDFE0B4B1C78002093
:10903800012C05D10146FDF704FF2046002104E07C
:109048000721FDF7FEFE01200721FDF7FAFE034B7D
:109058001A68094B1A6010BD800F0020B02E00203E
:109068007FD1F00820A10700FF27ED0880D1F00884
:10907800C82E0020D02E0020A0380020014B1868F0
:10908800A4E700BFAC2800207047FEE7FEE7FEE734
:10909800FEE770477047704702F01AB910B5094CDF
:1090A800A37A4BB1084B1A6822F006021A6000F046
:1090B80013F8204600F039FE4FF48020BDE8104038
:1090C80005F02CBFB828002010ED00E0014800F0A2
:1090D800FBBF00BFB8280020364BD3F8882042F4E5
:1090E8007002C3F88820344B1A6842F001021A60F3
:1090F80000229A60196821F0847121F48031196086
:109108002E495960196882B021F480211960DA600B
:10911800009201921A6842F480321A601A6802F4C6
:1091280000320192009A01320092019A1AB9009A0B
:10913800B2F5A06FF2D1204B1B6813F4003318BFAF
:1091480001230193019B012B2ED11B4B1A6C42F07A
:1091580080521A641A4A116841F4804111609A6871
:109168009A609A6842F400429A609A6842F4A0525F
:109178009A60144A5A601A6842F080721A60196834
:109188000D4A8901FBD5104B40F2056119609368BF
:1091980023F003039360936843F00203936093689A
:1091A80003F00C03082BFAD1024B4FF000629A60CF
:1091B80002B0704700ED00E0003802401030002493
:1091C8000070004008544007003C0240184B194A00
:1091D800996801F00C01042903D0082903D0164B23
:1091E80019E0164B17E059685A6811F4800F59684E
:1091F80014BF124B104B02F03F02B3FBF2F30C4AC0
:109208005268C2F30142C1F38811013252004B4344
:10921800B3FBF2F3074A1360054B9A68054BC2F398
:1092280003129A181968127921FA02F21A60704723
:1092380000380240980200200024F40000127A004E
:1092480037B51C230124002501A88DF804308DF8BA
:1092580005508DF806408DF80740FFF79FFC204623
:10926800214606F0CBFC0A4941F287334B6040F2B5
:109278004F130B800D814D804FF0804007F066F84A
:109288004FF080402146224607F025FC3EBD00BF36
:10929800FC2E002008B54FF08040012107F030FC7B
:1092A80040B14FF08040012107F035FCBDE808408F
:1092B800FEF75EBB08BD00BF08B5402005F020FEE4
:1092C80030B1FCF76BFE4020BDE8084005F026BE33
:1092D80008BD0000014608B5044807F0DBFD034857
:1092E800402107F084FE0028F9D008BD0044004062
:1092F800F0B589B04FF4E1330120019300232B4CE2
:10930800ADF808301E460146ADF80A30ADF80C300D
:10931800ADF810300C23ADF80E3006F04BFC4FF4CE
:109328000030012106F06AFC20680221072206F0BD
:1093380019F907226068032106F014F901250227AC
:1093480004232068059305A98DF81A608DF81B5031
:109358008DF818708DF8197006F084F80823606885
:10936800059305A98DF8187006F07CF8A06801A986
:1093780007F0E6FC2A4640F225510D4807F01EFE8C
:10938800262307A88DF81C308DF81D608DF81E6007
:109398008DF81F50FFF702FCA068294607F04DFD25
:1093A800044A054B1A6009B0F0BD00BFAC020020AA
:1093B80000440040DD920008383E0020024B9868C7
:1093C800002107F03ABD00BFAC02002010B5094CDF
:1093D80040F22551204607F014FE50B1A288D2B2BF
:1093E800112A02D1044B01211970044B19884A40F3
:1093F8001A8010BD00440040E30E0020EC0E00204F
:109408007047704773B50120014606F0D3FB264C20
:109418004FF4D8530093022303268DF804302046D6
:10942800002369468DF806308DF807308DF8056001
:1094380006F018F8204608210A2206F093F820467C
:1094480009210A2206F08EF820460B210A2206F08E
:1094580089F80A2220460C2106F084F801254FF4E9
:1094680080632046694600938DF806508DF80750B2
:109478008DF8056005F0F6FF0A210A46204606F039
:1094880071F829464FF4804006F0C4FB8020294635
:1094980006F09CFB4FF08050294606F0EBFB28466F
:1094A80005F03CFD7CBD00BF0000024007B54FF44D
:1094B800C060FFF769FB43238DF8043003220123C2
:1094C80001A88DF805308DF806208DF80730FFF7D4
:1094D80065FB0EBD782358430723B0FBF3F0002348
:1094E80001338342FCD970474FF47A735843F1E74C
:1094F80037B50023104C019305460320FFF7EAFF18
:10950800EB681A69013C019213D0019A002AF4DA37
:10951800019A42F001020192019A1A61064A1969F8
:10952800013A019102D00199C907F8D40320FFF745
:10953800D1FF00203EBD00BF410D030010B5C47827
:1095480074B900EB820003339B10D0F8D000224698
:1095580003E051F8044C0132046004319A42F8D116
:10956800002010BD033230B59210D0F8D0400B4621
:10957800002003E02568013043F8045C043390427E
:10958800F8D101EB800030BD0122F0B500238270D4
:1095980040220129C37082800CD108230370042360
:1095A80043704FF4A073C38002230372C1724FF05B
:1095B800A04309E041B90C230370062343704FF41C
:1095C800A063C3801F4BC17203F500620261C360D0
:1095D8004678044601461A46002508E002F5106C54
:1095E80002F530620A65C1F814C001353A46043103
:1095F800B54202F12007F1D303F58062426103F519
:109608008862C0F8CC20067803F5A06501460022E0
:1096180003E0C1F88C50013220350431B242F8D34E
:109628001946002202E0C4F8CC1001320434B242D8
:1096380001F58051F7D303F56063C0F80C310020C1
:10964800F0BD00BF0000044038B5037AC2680025A9
:10965800012B044625D1936B417A65F3104309B178
:1096680043F480139363D36823F4800323F05003F7
:1096780043F010036FF3C3036FF3C7136FF3514342
:109688006FF3D343D3602046FFF732FFE378012B13
:109698003ED1052363F34405E36845F020059D604A
:1096A80036E0D36843F04003D360FFF721FF237A05
:1096B800627A032B14BF4FF434134FF43C130AB1EE
:1096C80043F48013E26814209363FFF70DFFE26808
:1096D800217AD368032908BF43F48033D360237AFF
:1096E800032B15D1156B012363F39B656FF3D755D6
:1096F8002D2345F0805563F316451563C820FFF701
:10970800F3FEE36845F400051D63C820FFF7ECFE8F
:10971800E378012B07D1E3689D68052262F34405CD
:1097280045F020059D60002038BDC3689A6842F066
:1097380001029A6000207047C3689A6822F001020B
:109748009A600020704707B500230193019B43F0FE
:1097580020030193019B61F38A130193019BC26863
:109768001361064B1169013B019102D001998806EA
:10977800F8D40320FFF7AEFE00200EBD410D030014
:1097880007B500230193019B43F010030193019B4C
:10979800C2681361064B1169013B019102D001991E
:1097A800C906F8D40320FFF795FE00200EBD00BFC0
:1097B800410D030008B5C268D36801296FF35D73D2
:1097C8006FF39E7302D143F0005302E009B943F0EE
:1097D80080433220D360FFF787FE002008BDC368AE
:1097E800586900F001007047C3685B6913F0010F06
:1097F80014BF002001207047C368586900F00100B9
:109808007047C3685A69986910407047C3685868B8
:10981800704703691A6861F301021A607047C268E9
:10982800002393614FF0FF335361536053610B4B37
:109838009361C3789169002B14BF4FF400634FF410
:10984800016343F4701343F4405343F0080321EADF
:1098580003010B4393610020704700BF000800809C
:10986800F8B5D0F80C3100221A60036915461A6859
:1098780065F3CC221A60C37A012B04461BD103215D
:10988800FFF7C7FFE36880214FF4800261F30F02FE
:1098980059629A62C02262F30F0561F31F454FF4C3
:1098A800A072C3F8045162F30F056FF31F45C3F8A4
:1098B8000851C3F80C5110212046FFF744FF2046F9
:1098C800FFF75EFF226900234FF0FF311361204646
:1098D80053611E469161FF25D361214610E08269DC
:1098E8001768C7F3076707F08007FFB2002F14BF98
:1098F8004FF09047002717600133166104309560D8
:1099080062789342EBD300231D46FF2010E04A6D96
:109918001668C6F3076606F08006F6B2002E14BF76
:109928004FF09046002616600133156104319060AF
:1099380062789342EBD323691A6942F480721A6100
:10994800E278012A04D1054A402161F359421A6399
:109958002046FFF764FF0020F8BD00BF03010100A7
:1099680003699B68C3F34103013B022B9ABF024A78
:10997800D05C0320704700BFD0DA040810B5036933
:1099880081699C680A68C4F34100022802D06FF319
:109998000A0202E0032060F30A020A605A6842F4ED
:1099A80080725A60002010BD30B54D780B780022C7
:1099B800012D00EB830405D105FA03F3A46963F3D1
:1099C8000F0205E0012505FA03F3646D63F31F42F6
:1099D8002368C3F3072505F08005EDB26DB98D68DE
:1099E80065F30A03CD78C98865F3934361F3995306
:1099F80043F0805343F4004323600369D9690A4361
:109A0800DA61002030BD30B54D780B780024012D87
:109A1800224600EB830105D105FA03F3896963F354
:109A28000F0205E0012505FA03F3496D63F31F42B0
:109A380003696FF3CF340C60D96921EA0202DA6155
:109A4800002030BDF8B54F780B78012F00EB830369
:109A580049D19E694C69356833692A4664F3120313
:109A680014B967F3DC430BE08F68E419013CB4FBDD
:109A7800F7F7CC7867F3DC43012C08BF64F35E7317
:109A88003361C378012B06D10B780C6900EB830393
:109A98009B695C610CE0CB78012B09D04B693BB129
:109AA80003690C785E6B012707FA04F434435C639E
:109AB800CB78012B07D103699B68DB0554BF45F0C0
:109AC800005245F080520B7800EB830342F00442C9
:109AD8009B691A60CB78012B38D10A788B8AC968C0
:109AE800FFF72CFD32E05E6D4F6935688C6833698D
:109AF8002A462FB964F31203012464F3DC430AE015
:109B08003F19013FB7FBF4F7BF05BF0D67F3DC430F
:109B18007C4364F312033361C378012B05D10B78BE
:109B28000C6900EB83035B6D5C61CB78012B06D17C
:109B38004B7913B145F0005201E045F080520B78A3
:109B480000EB830042F00442436D1A600020F8BD28
:109B580073B54D78012D3DD183694A691E681C692A
:109B68000094E4B242B962F306048DF800409DF80F
:109B7800024065F3C4040EE08D68AA4286BF4D61B9
:109B880065F3060462F306048DF800409DF8024070
:109B9800012262F3C4048DF80240009A1A61C27867
:109BA800012A05D10A780C6900EB82029269546196
:109BB80046F004421A60C378002B34D14B69002B5D
:109BC80031D003690A78586B012101FA02F2024385
:109BD8005A6328E00B784E698C6800EB83035B6D51
:109BE8001A681D690095EDB206B14C6164F306056B
:109BF8009DF802408DF80050012565F3C4048DF8E6
:109C08000240009C1C61C378012B05D10B780C69BC
:109C180000EB83035B6D5C610B7800EB830042F023
:109C28000442436D1A6000207CBD4B78012B0B78F1
:109C380000EB83000AD182691368C3F3076101F05E
:109C48008001C9B221B143F0804301E0426D13683D
:109C580043F400131360002070474B78012B0B78F6
:109C6800C97800EB83000CBF8269426D0239136822
:109C7800C9B26FF35553012998BF43F0805313605D
:109C88000020704703699A69D8691040000C704732
:109C980000EB810102694B6D9B6850691840704761
:109CA80003699869DB69184080B2704782B0002365
:109CB8000093C0238DF803300122002362F3C4030C
:109CC8008DF8023018238DF80030009A436D1A6120
:109CD800C278012A06D100F5B96058611A684FF0B8
:109CE80080221A6002B07047D0F8143110B50446CB
:109CF800D3B103699A68D20716D5827A42B1D0F8EF
:109D08000C21D0F80C116FF341026FF300020A60C6
:109D18005A6842F001025A600520FFF7E5FB236903
:109D28005A6822F001025A6010BD837A63B1036950
:109D38009B68D90708D5D0F80C31D0F80C216FF3FF
:109D480041036FF3000313607047012310B500222D
:109D580080F8123104460346FF2104E05869816007
:109D6800186D01328160607804338242F6D323692A
:109D780000221A615A61DA614FF0FF329A61204677
:109D8800FFF7FEFC20461021BDE81040DBE44B78CD
:109D9800012B0B7800EB83000FD183691868C0F39F
:109DA800074000F02003DBB2CBB900F00200C0B2DC
:109DB80000280CBF302020207047436D1868C0F37E
:109DC800074000F02003DBB25BB900F00200C0B22C
:109DD80000280CBF4FF440504FF40050704710203B
:109DE80070474FF4805070474B78012B0B7810B5B3
:109DF80000EB83030AD19C69102A236802D1BDE8CD
:109E0800104012E7202A0CD0302A0FE05C6DB2F522
:109E1800805F236802D143F400131BE0B2F5005FB2
:109E280002D143F0006315E0B2F5405F0FD1C3F3F0
:109E3800074202F02002D2B222B100234B71BDE8E2
:109E480010400AE743F0806343F0802302E00AB938
:109E580062F3CF33236010BDF8B50446FFF794FBD7
:109E68000122002384F8122184F81331282716468A
:109E7800194640250CE007FB03F000F58C7022180A
:109E88002354D3805670D1709560D16051610133ED
:109E980062789342EFD300232826194640250CE028
:109EA80006FB03F000F55C7022182354D380517030
:109EB800D1709560D1605161013362789342EFD3DC
:109EC8002046FFF739FC2046FFF7BEFB002120465D
:109ED800FFF770FC2046FFF7C3FC2046BDE8F840BA
:109EE800FFF723BC70B5CDB20C464FF0280601F041
:109EF8007F0106FB010115F0800F14BF01F58C717D
:109F080001F55C7104F07F04ED090C704D708A60F6
:109F1800CB7005B1CC80022B01D100230B71FFF768
:109F280043FD002070BD10B5CAB201F07F034FF0A9
:109F3800280404FB030312F0800F14BF03F58C738D
:109F480003F55C7301F07F01D20919705A70194644
:109F5800FFF759FD002010BD38B501F07F05282412
:109F68006C4304F55C7401194B6100238B614B70E1
:109F7800EBB20355CA60C478012C08BF0A6113B953
:109F8800FFF7E6FD01E0FFF75DFD002038BD70B585
:109F980001F07F042825654305F58C7541190126D4
:109FA800E4B2CA600A6100224E7044558A614B616E
:109FB80014B9FFF7CDFD01E0FFF744FD002070BDA7
:109FC800CAB212F0800F10B54FF0280306D001F086
:109FD8007F0403FB040303F58C7303E003FB010315
:109FE80003F55C73D209012401F07F0119709C709C
:109FF8005A701946FFF719FE002010BDCAB212F0B8
:10A00800800F10B54FF0280306D001F07F0403FB42
:10A01800040303F58C7303E003FB010303F55C738E
:10A028000024D20901F07F0119709C705A701946FA
:10A03800FFF713FE204610BD08B50B0604D501F046
:10A048007F01FFF780FB01E0FFF79AFB002008BDC6
:10A058000369002261F30A1219680A431A607047FB
:10A0680003695A6803206FF341025A60FFF73CBA4C
:10A0780003695A68032042F002025A60FFF734BAB3
:10A0880011F0800F4FF0280306D001F07F0103FB89
:10A09800010101F58C7103E003FB010101F55C711D
:10A0A800FFF775BE11F0800F4FF0280306D001F0BE
:10A0B8007F0103FB010101F58C7103E003FB010142
:10A0C80001F55C71FFF790BE2DE9F74F0446FFF7E5
:10A0D8008BFB002800F03F822046FFF792FB0546E5
:10A0E800002800F03882C0F3074000F00800C0B232
:10A0F800002861D02046FFF7C5FDA14682462746C5
:10A108004FF00008DFF86CB32E4650E01AF0010F4C
:10A1180046D05FFA88F2114620460092FFF7B8FD54
:10A1280010F0010F0546009A20D07B6D01259D6037
:10A13800E178A94207D11B69D9F87813C3F3120350
:10A14800CB1AC9F88833DBF8003020461B68114663
:10A158009847E378012B09D1B8F1000F06D194F89C
:10A168001131052B02D12046FFF7A0FD05F00203AF
:10A17800DBB213B17B6D02259D6005F00403DBB2F1
:10A1880013B17B6D04259D6005F00805EDB23DB166
:10A19800DBF8003020469B6898477B6D0820986064
:10A1A80008F101084FEA5A0A043709F12809BAF1F7
:10A1B800000FABD135460120C5F3074303F0040374
:10A1C800DBB2002B00F0AF802046FFF769FD264682
:10A1D80083464FF0000801959FE01BF0010F00F047
:10A1E800978023695FFA88F919695D6B04EB890226
:10A1F80025FA09F59269ED019268EDB20D43154013
:10A20800EA071CD55A6B012000FA08F122EA01027C
:10A218005A63B369974A9860136805465B68204695
:10A2280049469847E378AB4209D1B8F1000F06D107
:10A2380094F81131042B02D12046FFF737FD05F0C1
:10A248000403DBB213B1B36904259D6005F008036C
:10A25800DBB213B1B36908259D6005F01003DBB2CA
:10A2680013B1B36910259D6005F02003DBB213B16B
:10A27800B36920259D6005F04003DBB213B1B369D3
:10A2880040259D6005F00203DBB213B1B3690225D6
:10A298009D6025F07F0515F0FF0F39D0282505FBB7
:10A2A800084505F58C75C246AB696A69C3EB020CB3
:10A2B800AB689C4528BF9C460CF1030CB3694FEA78
:10A2C8009C0C9B696746A04614E0AA68E9681C1BB9
:10A2D800944228BF1446A3B240464A46FFF72EF9D7
:10A2E800EB681B19EB60AB69E71C1C19AC61B3691F
:10A2F8009B69BF089BB2BB4205D9AC696B699C429C
:10A3080001D2002BE1D1B369802544469D60D04637
:10A3180008F101084FEA5B0B0436BBF1000F7FF42C
:10A328005CAF019D012005F00203DBB213B1E368C5
:10A3380002225A61C5F3076303F08003DBB2CBB195
:10A34800A37A43B1D4F80C31D4F80C216FF341034C
:10A358006FF30003136023695A6822F001025A6000
:10A36800444B1B6820469B699847E3684FF00042BE
:10A378005A610120C5F3072303F00803DBB2F3B1E8
:10A388003C4B1B6820465B6998472369E2689B68D9
:10A398004FF400615161A27A82B1DB070ED5D4F87F
:10A3A8000C311A6842F001021A601A6842F003027E
:10A3B8001A60314B1A6942F006021A61012005F051
:10A3C8000803DBB243B12B4B1B682046DB68984778
:10A3D800E36808225A61012005F01003DBB2002B64
:10A3E80033D0E3689A6922F010029A611F6A28261E
:10A3F80007F00F0306FB0346C7F34343022B06F59A
:10A408005C7602D0062B1AD10EE047F6F0733B407B
:10A41800ABB1C7F30A172046F1683A46FFF7A2F82E
:10A42800F368DB19F36007E004F5B96120460822F8
:10A43800FFF798F8C7F30A17B369DF19B761E3683C
:10A448009A6942F010029A610120C5F3072303F0CC
:10A458001003DBB2002B39D023695A68002622F09A
:10A4680001025A6031462046FFF76DF9234632460D
:10A47800FF2108E04803002000ED00E058698160F2
:10A48800186D01328160607804338242F6D3236903
:10A4980001274FF0FF3267F30F069A6167F31F46F3
:10A4A8000F22DE615A612F221A611A686FF30A12AD
:10A4B8001A602046FFF7FAFBE3684FF480525A61AE
:10A4C800264B1B6820461B6998473846C5F3072367
:10A4D80003F02003DBB2EBB12046FFF74FFAE36845
:10A4E8002046DE68FFF73CFA032806D10023A37054
:10A4F8004FF40073A380092304E00123A3704023D1
:10A50800A380052363F38D26E3684FF40052DE60D1
:10A5180001205A61C5F3074303F01003DBB24BB1C6
:10A528000E4B1B682046DB699847E3684FF480129E
:10A538005A610120C5F3074505F02005EDB255B174
:10A54800064B1B6820461B6A9847E3684FF40012C5
:10A558005A610120FFE7BDE8FE8F00BF48030020D5
:10A5680043230B8000487047B802002038B51F4BC2
:10A578001A68511C052A196035D119790022012958
:10A588001A6030D09968B1F5006F08BF9A60174B10
:10A598009968DC68A1421A4602D100221A7122E0A9
:10A5A80086BFC1F500631361C1EB0404D0F8EC3534
:10A5B80098BF14611569B3F839300C4C9D428AB2C2
:10A5C80004D95918ED1AA160256104E06918A16041
:10A5D8000021ABB22161054901240C7104498A1894
:10A5E8008121FFF7D4FC002038BD00BFF00E002009
:10A5F8009B2F002038B528230A4D03FB01010A4B85
:10A60800B1F888131B69044628469847D4F8EC35F6
:10A618002046B3F8403001212A46FFF79DFC002070
:10A6280038BD00BF532F00203403002070B50B78CD
:10A6380013F0600506460C4625D0202D1FD1CD8885
:10A64800B5B113F0800F487808D0214B21499B6899
:10A658002A469847E2881F49304625E01E4B1D4987
:10A6680058641E4B30465D612A4600F022FB1DE00F
:10A67800174B48789B6829462A46984725E000F0FA
:10A6880077FB022521E04B780A2B11D00B2B14D035
:10A69800062B1AD14B881B0A212B03D1CA883A2AC8
:10A6A80028BF3A220E49304600F0EAFA00250CE0AD
:10A6B8000C49012200F0E4FA07E08B781BB9074A3D
:10A6C8001D46936101E000F053FB284670BD00BFB2
:10A6D80034030020932F0020B8020020F00E002041
:10A6E800CA020020080F002010B581210446FFF798
:10A6F8001AFC01212046FFF716FC82212046FFF7AD
:10A7080012FC024B5B689847002010BD3403002000
:10A7180038B5D0F8EC350446B3F839208121022346
:10A72800FFF7E0FBD4F8EC350121B3F840202046D0
:10A738000223FFF7D7FB8221082203232046FFF7D5
:10A74800D1FB094B022200251A715D71074B1B686A
:10A758009847D4F8EC35064AB3F840302046012132
:10A76800FFF7FAFB284638BD7803002034030020A1
:10A77800532F002010B5074C606CFF2807D0064BFC
:10A78800064A9B68064952699847FF23636400207C
:10A7980010BD00BFB802002034030020F00E0020D6
:10A7A800932F002038B510490B79012B19D10C696A
:10A7B8000CB90C7115E0D0F8EC358D68B3F8393068
:10A7C8009C42AAB203D95D198D60E41A03E0A3B2D2
:10A7D8002C198C6000240C61044952188121FFF760
:10A7E800D6FB002038BD00BFF00E00209B2F0020B4
:10A7F80000207047002070470023F0B5084A094E32
:10A808001D4609E01468C75C375501340133B4F5B7
:10A81800006F146008BF15608B42F3D10020F0BDB3
:10A82800FC0E00209B2F0020104B114AD3F800C0CB
:10A8380000232DE9F0410F4F16461D460DE0146820
:10A8480010F8038007F804800134802C08BF2C46D8
:10A8580014603468644505D001338B42EFD1002081
:10A86800BDE8F0810220BDE8F08100BF1C3800205F
:10A87800303800209C37002021280FD1084B1A6857
:10A888000A701A68120A4A705A888A70DA78CA7086
:10A898001A790A715A794A719B798B71002070472D
:10A8A8002C03002007B502AB012103F8010D18465F
:10A8B800FFF7A2FF0EBD002100E00131435C002B31
:10A8C800FBD199E798E70B4B0B491A680968914245
:10A8D8000BD00A498A5C02701A680132802A1A6011
:10A8E80005D100221A60012070470020704701201E
:10A8F800704700BF1C380020303800209C370020EB
:10A90800204B1A68204B1B689A42F0B509D135E0F4
:10A918000133802B08BF00239A4203D11A4B1A60D7
:10A928002CE01A4CE15C0029F2D00A29F0D00D295C
:10A93800EED0154C1549134D23600E460023CF1851
:10A948002268BA5CC254226801339F18802F08BF5E
:10A9580053422F689A18974210D0B25C1AB10A2A4B
:10A9680001D00D2AEBD10022C254074A11685918A8
:10A978007F29116003D98039116000E0002318464F
:10A98800F0BD00BF303800201C3800209C37002064
:10A99800704700BFD0F8E43510B51B6904469847E6
:10A9A800032384F81231002010BD08B5042380F871
:10A9B8001231D0F8E435DB689847002008BD08B5A7
:10A9C800D0F8E035DB6903B19847002008BD08B529
:10A9D800D0F8E0351B6A9847002008BD08B5D0F8C4
:10A9E800E0355B6A9847002008BD002110B5402279
:10A9F80004460B46FFF776FA8021402200232046C2
:10AA0800FFF770FA012384F81231D4F8E435A078FE
:10AA18005B689847002010BD13B56946044600F0EE
:10AA280085F99DF8001001F01F03012B07D0022BB8
:10AA38000AD073B92046694600F026FA0FE020468E
:10AA4800694600F007FA0AE02046694600F0A2F9D4
:10AA580005E021F07F01C9B22046FFF7B1FA0020D6
:10AA68001CBD38B5044600293DD190F81131022BA0
:10AA780042D1D0F83421D0F820319A4211D9C17886
:10AA8800D21A0129C0F8342104D1D0F82411CB18E6
:10AA9800C0F8243192B22046D4F8241100F000F90D
:10AAA8002AE0D0F83821B2FBF3F503FB152565B988
:10AAB8009A420AD3D0F83C319A4206D229462A460D
:10AAC80000F0EEF8C4F83C5116E0D4F8E035DB6845
:10AAD8002BB194F81221032A01D120469847204629
:10AAE80000F00FF908E0D0F8E0355B6923B190F881
:10AAF8001221032A00D19847002038BD10B504461A
:10AB080059BB90F81131032B30D1D0F88C23D0F8F1
:10AB180078339A4214D9C178D21A0129C0F88C2303
:10AB280004D1D0F87C13C918C0F87C139A4228BF06
:10AB38001A4692B22046D4F87C1300F0CAF815E001
:10AB4800D0F8E0351B6923B190F81221032A00D10F
:10AB58009847204600F0C6F808E0D0F8E0359B6931
:10AB680023B190F81221032A00D19847002010BD84
:10AB78002DE9F041069F0446164698460D46FEF715
:10AB880041FC20462946C4F8E085C4F8E475C4F8B9
:10AB9800E865FFF761F9D4F8E4351B689847204663
:10ABA800BDE8F041FEF782BC00207047D0F8E035E0
:10ABB80010B504461B689847D4F8E4359B68984755
:10ABC800002010BD08B5D0F8E0355B689847002034
:10ABD80008BD000012230B8000487047780300204E
:10ABE80004230B80004870478A03002010B5044CEA
:10ABF80004480A46214600F075FA204610BD00BFF9
:10AC0800343800200AE005080A4608B50248034916
:10AC180000F068FA014808BD1DE005083438002036
:10AC28000A4608B50248034900F05CFA014808BD25
:10AC38002BE005083438002008B50A4608B904484E
:10AC480000E00448044900F04DFA034808BD00BF7D
:10AC580036E0050843E005083438002008B50A4600
:10AC680008B9044800E00448044900F03BFA0348E6
:10AC780008BD00BF50E0050871E005083438002021
:10AC880010B513460C46C0F83821C0F8342102220A
:10AC980080F8112100212246FFF779F9002010BD24
:10ACA80010B50C46134600212246FFF770F9002024
:10ACB80010BD10B513460C46C0F89023C0F88C237D
:10ACC800032280F8112100212246FFF745F90020D0
:10ACD80010BD10B50C46134600212246FFF73CF97B
:10ACE800002010BD0021042310B50A46044680F850
:10ACF80011310B46FFF74BF92046FEF7D7FF00202E
:10AD080010BD0021052310B50A46044680F811310C
:10AD18000B46FFF721F92046FEF7C8FF002010BDBB
:10AD2800282303FB0100B0F88803704790F8C83562
:10AD38000B7090F8C9354B7090F8CB2590F8CA3550
:10AD480003EB02234B8090F8CD2590F8CC3503EB2C
:10AD580002238B8090F8CF2590F8CE3503EB0223A1
:10AD68009BB2CB80C0F83C31012380F81131704789
:10AD780010B591F90030002B044601DBCB880BB9E4
:10AD8800802100E00021FFF71BF92046BDE81040B4
:10AD9800FEF78CBF38B50D4604466B780979012B50
:10ADA80010D027D3032B51D190F81231022B28D081
:10ADB800032B47D16B889BB991B1802910D0FFF73D
:10ADC800FFF80DE090F81231022B1AD0032B39D17D
:10ADD8006B88002B3AD149B1802907D0FFF70EF9CB
:10ADE800D4F8E03520469B68294698472046FFF767
:10ADF80079FF2BE090F81231022B02D0032B21D1DE
:10AE080006E019B3802921D02046FFF7D9F81DE0C4
:10AE180011F0800F4FF0280306D001F07F0103FBEB
:10AE2800010393F81A2103E003FB010191F872234F
:10AE3800074B02B101221A60204605490222FFF79A
:10AE48001FFF03E020462946FFF792FF002038BD88
:10AE58000C0F002038B590F81231032B04460D462C
:10AE68000CD10B79012B09D8D0F8E0359B689847AD
:10AE7800EB883BB92046FFF735FF03E0204629461B
:10AE8800FFF776FF002038BD73B54B7804460D46B2
:10AE9800092B00F21C81DFE813F0D10008011A0128
:10AEA800E4001A0172000A001A01C00092004B88DF
:10AEB8001A0A013A062A00F20A81DFE812F00700AE
:10AEC8001A0027000801080108010801D4F8E8352C
:10AED800A0781B680DF106019847EB88402B0146C6
:10AEE80003D094F81231012B3AD10823ADF806307B
:10AEF80036E0D4F8E035A0789B6A0DF10601984752
:10AF0800022343700146C4F8EC0529E0DBB2052BA7
:10AF180000F2DD80DFE803F003080D12171CD4F8F7
:10AF2800E835A0785B6817E0D4F8E835A0789B6826
:10AF380012E0D4F8E835A078DB680DE0D4F8E835FD
:10AF4800A0781B6908E0D4F8E835A0785B6903E0CD
:10AF5800D4F8E835A0789B690DF1060198470146B9
:10AF6800BDF80630002B00F0B680EA88002A00F011
:10AF7800B2809A4228BF1A46ADF806205CE08B885A
:10AF8800002B40F0A480CB88002B40F0A08094F8E0
:10AF980012214B88032A00F09A8003F07F0520468F
:10AFA80084F813512946FFF753F82046FFF79AFE15
:10AFB8000DB1022300E0012384F812318BE0897877
:10AFC800464E0129317100F2828094F81231022B29
:10AFD80002D0032B7BD108E0002962D00121032392
:10AFE80084F8101184F8123113E041B9022384F86F
:10AFF800123184F810112046FFF7E4FD51E094F86F
:10B008001011012920464DD0FFF7DCFD317984F875
:10B0180010112046FFF7CAFD43E0CA88012A56D11D
:10B0280094F81231022B02D0032B50D102E02046B3
:10B038002B4913E004F5887120460FE094F812318B
:10B04800023B012B43D8D4F814312449002B0CBF00
:10B058000123032341F80C3F20460122FFF710FE8D
:10B0680039E04B88012B29D0022B34D18B8813F07F
:10B07800FF0F30D121691B0A013B4A68042B0FD806
:10B08800DFE803F0030507090B00012306E00223AC
:10B0980004E0032302E0042300E0052363F306121F
:10B0A8004A602046FFF71EFE15E094F81231023B75
:10B0B800012B0CD84B88012B0DD10023C4F8143177
:10B0C800D4F8E03520469B6829469847E9E72046AA
:10B0D8002946FFF74DFE00207CBD00BF0C0F002065
:10B0E800140F002030B5C8B10023DDB20133C418F5
:10B0F80014F8014C002CF8D16B1C5B0013800B700A
:10B1080003234B70022305E0CA545A1CD2B20233FF
:10B118008C54DBB210F8012B002AF5D130BD00BFEA
:10B128007047704770477047704770477047000016
:10B1380008B5FCF74BFB094B5A78187002435A7054
:10B148001AB19A7801329A7030B99B78034A012B68
:10B1580002D900235370937008BD00BF1C0F002054
:10B168002DE9F84F394B1A78394B2DED028B22B95E
:10B178001A68802392FBF3F300E01B68354A536199
:10B18800354B1A8892B2002AFBD0334B00221A8022
:10B19800FDF7A6FD10EE105AFDF7A8FD284610EEA3
:10B1A800104A06F0B9F880462046894606F0B4F8F9
:10B1B80041EC100B41EC180B08F002F957EC106B3E
:10B1C800B0EE480AF0EE680A08F0FAF932463B4653
:10B1D800404649465BEC10AB06F0F2F806F0D2FBAD
:10B1E8009FED1E8A07EE100ADFED1D7A57EE087AEA
:10B1F800184C52465B46C4ED007A4046494606F074
:10B20800DFF806F0BFFB07EE900A27EE888A84ED88
:10B21800018AFDF77DFD84ED020AFDF77FFD84EDCF
:10B22800030AFCF7E3F90F4B62691B68D31A0E4A4D
:10B2380007EE100A1268F8EEC77A93FBF2F3C4ED32
:10B24800047A2383BDEC028BBDE8F88F800F0020C1
:10B25800B02E0020643A0020D20E00200000F042F8
:10B2680000008C42AC2800203028002007B50420BC
:10B27800012104F09FFC4FF46043009301238DF8F3
:10B28800043002238DF805300448002369468DF800
:10B2980006308DF8073004F0E5F80EBD00080240CE
:10B2A800084B1A684FF47A73B2FBF3F2064B013A73
:10B2B8005A60064AF02182F8231000229A60072279
:10B2C8001A6070479802002010E000E000ED00E0EE
:10B2D800034B5A6812B15A68013A5A60704700BF66
:10B2E8001C0F0020024B58605A68002AFCD1704796
:10B2F8001C0F002030B585B004460D4601A85C49F6
:10B308000A220AF055FD5B4B1B78032B10D8DFE8A7
:10B3180003F00205080B01A8574907E001A857499F
:10B3280004E001A8564901E0564901A80AF02AFE9E
:10B3380004AA131913F80C3C5D19EDB22F2D01D88E
:10B348000A3502E0392D01D90A3DEDB204AB1C19CA
:10B358004FF6FF7004F80C5CFAF788FB0020FAF748
:10B3680087FC0DF103050F24204623345A210023BE
:10B3780015F8012FA4B2FAF795FCB4F5A57FF3D11F
:10B3880064205A212C220023FAF78CFC0023CD20BC
:10B398005A212C22FAF786FC0020FAF767FB354B76
:10B3A8001B78032B62D8DFE803F002284B5601A96B
:10B3B80031480AF0E7FD0A2200212F480BF00AFF66
:10B3C800314A324B12781860012A06D1304A90422D
:10B3D80001DC01321A602F4A06E0B0F5FA5FBCBF03
:10B3E8004FF4FA521A602C4A1B689342C4BF274B89
:10B3F8001A602A4B1A682A4B20E001A91F480AF054
:10B40800C1FD0A2200211D480BF0E4FE1E4A254B0F
:10B4180012781860012A06D11D4A904201DC0132D7
:10B428001A601C4A06E0B0F5FA5FBCBF4FF4FA5246
:10B438001A60194A1B68934218DD1A4B1A6015E006
:10B4480001A90F480AF09EFD0D4800210A220BF0C1
:10B45800C1FE154B09E001A90A480AF093FD094805
:10B4680000210A220BF0B6FE104B186005B030BD63
:10B4780092E00508AB28002078280020A0280020AA
:10B48800B62E002064280020800F0020B428002059
:10B498001FA1070080D1F00850DA1100AC28002065
:10B4A800B02E0020D42E0020A82E002060280020D6
:10B4B80010B50D4B0D4C1A680D4821460AF03AFD9F
:10B4C8000C4B0D481A6821460AF034FD0B4B0C480A
:10B4D8001A6821460AF02EFD0A4B0B481A682146C5
:10B4E800BDE810400AF026BDB428002006D605089D
:10B4F80078280020D42E0020A0280020A82E002084
:10B50800B62E002060280020642800209FED010A44
:10B51800704700BF000000009FED010A704700BFA0
:10B52800000000009FED010A704700BF0000000006
:10B538007047704718B1012801D1034B00E0034B55
:10B548001868FDF743BD00BF9C280020AC280020E8
:10B5580010B9034B18687047024B1868704700BF52
:10B56800B4280020AC28002010B9034B1868704795
:10B57800024B1868704700BFD42E00209C2800207A
:10B5880008B54FF49570FCF745F840F26523C31AE7
:10B59800584240EB030008BD08B5C620FCF73AF84E
:10B5A80040F28D13C21A504240EB020008BD4FF41E
:10B5B800957040F26521FCF71FB8C62040F28D1146
:10B5C800FCF71AB8DCE760EEA00AB7EE007AF0EEF6
:10B5D800606A70EE077A40EE006A47EEA70A36EE18
:10B5E800C77A08B5C7EE200A10EE900A05F094FE57
:10B5F8000022084B05F0E4FE0022074B05F02EFD63
:10B6080006F0C0F907EE900AFDEEE77A17EE900A09
:10B618009F3008BD000059400000E03F38B52DEDCF
:10B62800028BF7EE008AB0EE608A70EE288A10EE80
:10B63800900A28EE088A05F06FFE08EEA88A002214
:10B648000F4B05F0BDFE044618EE100A0D4605F036
:10B6580063FE02460B462046294605F0DBFF002222
:10B66800084B05F0FBFC06F08DF907EE900AFDEE9D
:10B67800E77A17EE900A7730BDEC028B38BD00BF31
:10B68800000069400000E03F2DE9F04F884F2DEDA4
:10B69800068B97E80F0091B00CAC103784E80F00C8
:10B6A8000FCF05AE0FC697E807004FF6FF7386E881
:10B6B80007009F2077216422F7F77DFEA0207721DD
:10B6C80064224FF6FF73F7F776FE9E2077216422F7
:10B6D8004FF6FF73F7F76FFE9F20762164224FF62F
:10B6E800FF73F7F768FE4FF6FF73782164229F20F7
:10B6F800F7F761FE0020F9F778FA9F207721652295
:10B70800FAF7F6F90C349F2077216422FAF7F0F95A
:10B718000DF12C0A0394F7EE009A4FF00F0B00E09E
:10B728004D460AF1040AF7EE008A9AED009A0024C1
:10B73800B0EE68AA01E0B846354618EE900A05F062
:10B74800EBFD59A3D3E9002305F03AFE06F01AF9F8
:10B7580008EE900A38EEE98AB0EE490AF0EE480A97
:10B76800FFF731FFB0EE490AF0EE480A0646FFF748
:10B7780055FFB2B2074683B22CB9104619460F22BC
:10B78800F9F7FEFA06E0A8B21FFA88F1CDF800B082
:10B79800FAF7F8F80134B4F5967FCCD13D46F7EEC8
:10B7A800008A002401E045464E4618EE900A05F04E
:10B7B800B3FD3DA3D3E9002305F002FE06F0E2F84D
:10B7C80008EE900A39EEE88AB0EE490AF0EE480A27
:10B7D800FFF7F9FEB0EE490AF0EE480A8146FFF796
:10B7E8001DFF1FFA89F2804683B22CB9104619460C
:10B7F8000F22F9F7C5FA05E0B0B2A9B2CDF800B04A
:10B80800FAF7C0F80134B4F5967FCCD1039B9A457A
:10B8180086D104AD0DF12C0B4FF0000A01E0B846BB
:10B82800B146043595ED009AF7EE008A002401E050
:10B83800B846B14618EE900A05F06EFD1AA3D3E992
:10B84800002305F0BDFD06F09DF808EE900A38EEDD
:10B85800CA8AF0EE490AB0EE480AFFF7B4FEB0EE25
:10B86800480AF0EE490A0646FFF7D8FEB2B2074684
:10B8780083B22CB9104619462246F9F781FA07E037
:10B888001FFA89F01FFA88F1CDF800A0FAF77AF8C4
:10B898000134B4F5C87FCBD15D45C0D111B0BDEC42
:10B8A800068BBDE8F08F00BF295C8FC2F528F03FFA
:10B8B800D4DA0408121A06EE902A081AB8EEE67AC4
:10B8C80006EE900AF8EEE67A08B5C7EE277A17EE84
:10B8D800900A05F021FD07A3D3E9002305F070FDC8
:10B8E8000022034B05F0BAFB06F004F808BD00BFC0
:10B8F8000000E03F0000000000F073408A1A06EEE6
:10B90800902A081AB8EEE67A06EE900AF8EEE67A79
:10B9180008B5C7EE277A17EE900A05F0FDFC07A3D5
:10B92800D3E9002305F04CFD0022034B05F096FBFC
:10B9380005F0E0FF08BD00BF0000E03F0000000088
:10B9480000E0684070B506460D460024610704D53E
:10B95800A0B231462A46F9F713FA0134B4F5A07FAC
:10B96800F4D170BD70B506460D460024600704D5B5
:10B97800A1B230462A46F9F703FA0134C82CF5D1AA
:10B9880070BD114B11481B781149124A0068012BF0
:10B99800114B09D1126808601A60104B1A68104BD5
:10B9A8001A60104B1A680CE01268D2011A600B4B2F
:10B9B8001A680B4BD2011A600A4B1A68C00108605A
:10B9C800D201094B1A607047800F0020B42800206C
:10B9D800AC280020D42E00209C280020A82E00206F
:10B9E8003028002088280020C82E0020014B186825
:10B9F800FDF7ECBAAC28002008B5FFF7C2FFBDE898
:10BA08000840F3E770B500210A222748274D284E41
:10BA1800284C0BF0DFFB00210A22286026480BF097
:10BA2800D9FB00210A22306024480BF0D3FB002107
:10BA38000A22206022480BF0CDFB224B32681860A6
:10BA48002B682149D31A06EE903A2368B8EEE67AB5
:10BA580006EE903AF8EEE67AC7EE277AFCEEE77A39
:10BA680017EE903A9AB20B80531C07EE903AB8EE54
:10BA7800E77ADFED167A67EE277A154BFCEEE76A70
:10BA880016EE901A8AB206EE902AB8EEE67A198077
:10BA980077EEC77AF5EEC07AF1EE10FA01DD0132E1
:10BAA8001A80BDE87040A7E778280020B428002055
:10BAB800D42E0020A82E0020A0280020B62E00207A
:10BAC80064280020602800209C3C00200000803D65
:10BAD8002C3D00200022F0B51346202603254FF008
:10BAE8002C0C00E02646303EF6B217460132092EED
:10BAF80010F8014B0AD897FBF5F605FB16772FB916
:10BB0800CE1801F803C07470023301E0CC5401333D
:10BB1800092AE7D12022CA54CB1848225A707A221F
:10BB28009A700022DA70F0BDF0B51F46144B1E78EB
:10BB3800012E8DB005460C4620D0A6F1030CDCF191
:10BB4800000646EB0C06CEB90E4908A80AF0F2F931
:10BB580008A86946FFF7BEFF0B496A4604A80AF021
:10BB6800E9F9BDF84800F9F781FF3846F9F794FF7D
:10BB78002846214604AA3346FAF7B2F80DB0F0BDBC
:10BB88003428002006D6050867DD050810B5012110
:10BB98000446F9F71BF9014B1C8110BD1C0F00204E
:10BBA80008B50021C620FBF727FD4FF4957000214A
:10BBB800BDE80840FBF720BD014B9F221A81704762
:10BBC8001C0F002000200146C82240F23F13F9F75D
:10BBD80011BA07B50DF10700FEF775FE9DF80700CD
:10BBE8000EBD08B5FFF7F5FF0028FBD108BD30B53D
:10BBF800044687B010EE100A0D4605F08DFB02468C
:10BC08000B4601A805490AF095F92046294601AADC
:10BC18000023FAF765F807B030BD00BF9CE00508BF
:10BC280008B5084802F080FE0648022102F04DFFE0
:10BC38000028F9D0034802F0A3FE07EE900AB8EEF8
:10BC4800670A08BD0020014010B52DED028B9FED5D
:10BC5800098A1924FFF7E4FF013CE4B238EE008AB0
:10BC6800002CF7D19FED040A28EE000ABDEC028BE8
:10BC780010BD00BF00000000ACC868392DE9F04FC6
:10BC88002DED068B7E4B7F4C7F495D695F68BBB0AD
:10BC98000646324632A893ED038AD3ED04AAD3EDC3
:10BCA800028A93ED00AA93ED069A0AF043F9A06878
:10BCB80005F032FB02460B4622A874490AF03AF90D
:10BCC800E06805F029FB02460B4626A870490AF0F1
:10BCD80031F91AEE900A05F01FFBCDE90601DDE9FE
:10BCE80006236C492AA80AF025F9284605F014FB12
:10BCF80082468B4652465B4667492EA80AF01AF9D7
:10BD080018EE900A05F008FB02460B460EA8634998
:10BD18000AF010F918EE100A05F0FEFA8046894676
:10BD280042464B465E4912A80AF004F91AEE100A78
:10BD380005F0F2FACDE90801DDE90823594916A80A
:10BD48000AF0F8F8384605F0E7FACDE90401DDE92C
:10BD5800042355491AA80AF0EDF819EE100A05F05F
:10BD6800DBFA02460B461EA850490AF0E3F8D4ED68
:10BD7800047AFDEEE77A0AA817EE902A4C490AF0F1
:10BD8800D9F8B5EEC08AF1EE10FADFED4A9A37D548
:10BD9800304605F0AFFA34A3D3E9002305F010FBD1
:10BDA800F1EE487A044617EE900A0D4605F0B4FA0B
:10BDB80002460B462046294605F002FB02460B4682
:10BDC8002BA1D1E9000105F025FC05F0DBFD9FED75
:10BDD8003A7A07EE900AF4EEC77AF1EE10FAC6BF87
:10BDE800C7EEA97A354C364CF4EEE97AF1EE10FA42
:10BDF80038DD9FED307A334D334CC7EE877A6EE0ED
:10BE08001DA3D3E900234046494605F0D9FA044664
:10BE180030460D4605F06EFA13A3D3E9002305F06A
:10BE2800CFFA02460B462046294605F0F3FB05F0FB
:10BE3800A9FD07EE900AB7EE007AF4EEC77AF1EEA4
:10BE480010FA46BF67EEA97A204C214CF4EEE97A45
:10BE5800F1EE10FA42DD9FED177A1E4D1E4CC7EE2B
:10BE6800877A3CE0174D3AE01F85EB51B81E194020
:10BE7800000000A2941A6D420000000080842E4148
:10BE88004C3C0020643A0020BCE00508C6E00508E8
:10BE9800D1E00508DCE00508E6E00508F0E0050863
:10BEA800FBE0050806E1050811E105081CE10508A5
:10BEB80028E1050800007A4400247449ADE005082B
:10BEC800AAE005084EE00508B6E00508B3E0050855
:10BED800B0E0050844DF0508B9E00508924D17EE03
:10BEE800900A05F019FA2A46CDE9000136A88F49CB
:10BEF80002940AF01FF88E4B1A688E4B1B68964204
:10BF0800CCBF002201229E428B4BD8BF0022DA60B0
:10BF18008A4B1B78082B40F095800220F9F7A8FE81
:10BF28004FF6FF70F9F7B8FD1F20F9F79FFD1921AB
:10BF38000023834A2D20F9F7D3FE4FF6FF70F9F757
:10BF4800ABFD00200024F9F791FD0F20B421324603
:10BF58004FF6FF730094FFF7E7FD0F206E2122AA2A
:10BF68002346F9F7BDFEA0206E2126AA2346F9F73D
:10BF7800B7FE0F20382116AA2346F9F7B1FEA020F4
:10BF880038211AAA2346F9F7ABFE0F205C212AAA0A
:10BF98002346F9F7A5FEA0205C212EAA2346F9F72F
:10BFA8009FFE0F204A210EAA2346F9F799FEA020EA
:10BFB8004A2112AA2346F9F793FE0F209B211EAAB5
:10BFC8002346F9F78DFE0F20842136AA2346F9F778
:10BFD80087FE5C4B1B68B3F57A7FCCBF4FF4FC60DF
:10BFE8004FF47840F9F758FD0023A0209B210AAAB6
:10BFF800F9F776FE544B1B78012B08D14FF4FC60FF
:10C00800F9F74AFD4FF48C700221504A07E04FF6C9
:10C01800E070F9F741FD4E4A4FF48C70022100237D
:10C02800F9F75EFE0020F9F737FD4FF4FC60F9F7E9
:10C038001DFDFFF709FE0F20DC21FFF7D8FD1F20AB
:10C04800F9F72AFD3D4B1B789A1FD2B2012A02D973
:10C058000B2B40F026823F4B1B78023B052B00F24E
:10C068002082DFE813F006007F00E3003C01DF01D7
:10C078005901DFED397A2AEE27AA1AEE100A05F0DF
:10C088004BF99DED040B8046894607F099F9404627
:10C0980053EC102B494605F093F91FA3D3E900236D
:10C0A80004F0DCFF05F026FC9DED040B044607F0C8
:10C0B80087FA404653EC102B494605F081F90246B1
:10C0C8000B4617A1D1E9000104F0C6FF05F012FCE8
:10C0D8004FF6E0730093054600230520DC21324625
:10C0E800FFF722FD144BDB6853B11C4B18881C4B1F
:10C0F8004FF4784719880097A2B2ABB2F9F742FC1F
:10C10800164B1C60164B4FF6E0701D60F9F7AEFC3D
:10C11800C7E100BFAFF300800000000000E063400B
:10C128000000000000C05D4044DF050835E1050857
:10C13800D42E0020B42800201C0F00203428002012
:10C1480042E10508DC1B0020800F002061E10508A2
:10C1580065E10508C42E00200000C842983A002076
:10C16800383D0020A04B1868A04B9FEDA19A196894
:10C178003246FFF79FFBF4EE498AF1EE10FAC8BF8A
:10C18800F0EE498AF5EE408ADFED9A7AF1EE10FA80
:10C1980048BFF0EE678AF4EEC98AF1EE10FA044659
:10C1A8001ED8F4EEE78AF1EE10FA19DBFDEEE88A04
:10C1B800002018EE902A4FF4FA71FFF79FFB8E4B80
:10C1C800DB68054653B18D4B18888D4B4FF6FF77CA
:10C1D80019880097A2B2ABB2F9F7D4FB884B1D605F
:10C1E800B4EE498ADFED827AF1EE10FAC8BFB0EEFC
:10C1F800678ADFED847AB4EE678AF1EE10FA48BFF9
:10C20800B0EE678AB4EEC98AF1EE10FA00F24981FD
:10C21800B4EEE78AF1EE10FAC0F24381BDEEC88AA7
:10C22800794818EE102A4FF4FA71AEE06E4B186890
:10C238006E4B32461968FFF73DFBF5EEC0AAF1EEEA
:10C2480010FA044627DDDDE9060159A3D3E90023E6
:10C2580005F028FBF8B158A3D3E90023DDE906016E
:10C2680005F0AEF80B4602466849002004F0F4FEDB
:10C2780005F040FB604BDB68054653B15F4B1888FF
:10C288005F4B4FF6FF7719880097A2B2ABB2F9F768
:10C2980079FB5B4B1D605046594649A3D3E90023FF
:10C2A80005F01EFB002800F0FC805046594640A3CC
:10C2B800D3E9002305F0F6FA002800F0F28042A343
:10C2C800D3E900235046594605F07AF802460B4652
:10C2D80000204F4904F0C0FE05F00CFB57E0424B2C
:10C2E8001868424B32461968FFF7E4FA38A3D3E9D5
:10C2F80000230446DDE9080105F0F2FA50B19DED8E
:10C30800080B07F041FA002251EC100B414B05F0E5
:10C3180057F8B1E0C825B2E02FA3D3E90023DDE93F
:10C32800040105F04DF82EA3D3E9002305F072F9B6
:10C3380005F028FB2C4B08EE100A18682B4B3246E8
:10C348001968FFF7B7FADFED347A4AEE677A2A4BB5
:10C35800FDEEE77ADB6817EE905A044625EAE575A4
:10C3680053B1264B1888264B4FF6FF77198800974C
:10C37800A2B2ABB2F9F706FBBDEEC88A204B18EEA5
:10C38800102A1D606FF0B300B421FFF7B7FA1A4BFB
:10C39800DB68054653B1194B1888204B4FF4FC67EE
:10C3A80019880097A2B2ABB2F9F7ECFA1B4B75E00B
:10C3B8009A9999999999B93F0000000000409F40C7
:10C3C8009A9999999999B9BF0000000000408F4047
:10C3D80089B5F81400E3693F00000000008076404A
:10C3E8001F85EB51B81E1940B4280020D42E002018
:10C3F8000000FA43000000001C0F0020983A0020BB
:10C40800383D00200000FAC30CFEFFFF0000694021
:10C4180000005940000054C00000484390380020F4
:10C428000000C8425FED027AB4EE679AF1EE10FAA6
:10C43800C8BFB0EE679AB4EEE79AF1EE10FA30D8BA
:10C44800214B1868214B32461968FFF733FA044626
:10C4580019EE100A04F060FF41EC100B07F094F994
:10C4680000221B4B51EC100B04F0AAFF02460B46AE
:10C478000020184904F0F0FD05F03CFA0546164B7B
:10C48800DB6853B1154B1888154B4FF6FF771988A1
:10C498000097A2B2ABB2F9F775FA114B1D600F4BBA
:10C4A8001C60104B1B78022B09D043B14FF6FF7369
:10C4B80000930520DC2132460023FFF735FB3BB013
:10C4C800BDEC068BBDE8F08FB4280020D42E0020E8
:10C4D80000005940000069401C0F0020983A0020D5
:10C4E800383D0020C42E002010B54FF4C770FBF76C
:10C4F80091F8DB2805D14FF4C870FBF78BF884B2AC
:10C5080019E041F2E104214644F20100FBF774F816
:10C5180044F20100FBF77EF8A04214BF80244FF4D8
:10C52800007421B24FF4C870FBF766F84FF4C77077
:10C53800DB21FBF761F8204610BD024B00221A6090
:10C54800704700BFAC38002070EEA10A88B030EE0A
:10C55800010A08B0704770EEE10A88B030EE410A6F
:10C5680008B07047F0EE407A20EEA10A60EE810A2A
:10C5780047EEA10A88B017EE810A08B07047D0B517
:10C5880061EEA17A41EE017A2DED048B17EE900A47
:10C5980088B0B0EE409AF0EE609AF0EE418AB0EEC4
:10C5A800618A04F0B9FE0022002306460F4605F012
:10C5B8006FF9E8B969EE887A49EE287A29EE088A8F
:10C5C80017EE900A04F0A8FE32463B4605F022F822
:10C5D80019EEA88A05F0D6F9044618EE100A04F0F8
:10C5E8009BFE32463B4605F015F805F0CBF901E015
:10C5F8000448044600EE900A00EE104A08B0BDEC6C
:10C60800048BD0BD0050C347F0B5814B2DED068B90
:10C6180093ED001AD3ED011A8DB0B0EE408AF0EE1A
:10C62800608A8DED040ACDED050A30EE410A70EE00
:10C63800E10A38EE011A78EEA11A8DED0A1ACDED4D
:10C648000B1A8DED080ACDED090AFFF798FF8DED5D
:10C65800020ACDED030A02AA92E8030006AB83E8BA
:10C668000300DDED079A9DED06AA69EEA97A4AEE68
:10C678000A7A17EE900A04F04FFE41EC100B07F00F
:10C6880009F951EC100B05F07DF909EE100A19EEC5
:10C69800900A04F041FE04461AEE100A0D4604F012
:10C6A8003BFE45EC104B41EC110B06F0E5FF51EC5D
:10C6B800100B05F067F968EEA87A48EE087AB1EE33
:10C6C80068AAC8EE279A534B534D5A691B8B68606A
:10C6D800EA612B8404468AEE27AA85ED009A19EEB2
:10C6E800100A85ED028AC5ED038AC5ED049A85ED29
:10C6F80005AA04F011FE42A3D3E9002305F0F0F8DF
:10C70800DFED467A002818BFB0EE679AB7EE007AD8
:10C7180079EE077A37EE497A414BC7EE877A1B786C
:10C72800033BC5ED067A042B5CD8DFE803F003125F
:10C7380025513C0018EE100A04F0EEFD044618EEF0
:10C74800900A0D4604F0E8FDCDE900013548364968
:10C758000DE019EE900A04F0DFFD04461AEE100A07
:10C768000D4604F0D9FDCDE900012E482F49224697
:10C778002B4609F0DFFB35E019EE100A04F0CCFD7A
:10C7880041EC100B07F000F80022294B51EC100B7C
:10C7980004F016FE05F0F6F804F0BEFD02460B465E
:10C7A800204824491CE019EE100A04F0B5FD06469D
:10C7B80020460F4604F0B0FD13A3D3E9002304F08C
:10C7C800FFFD3246CDE900013B4616481A49D0E73D
:10C7D80017EE900A04F0A0FD02460B4611481749CF
:10C7E80009F0A8FB0F4C00230220CA212246F9F7C2
:10C7F80077FA002323700DB0BDEC068BF0BD00BFA7
:10C80800AE47E17A14AEEF3FF6285C8FC2A54C40E4
:10C81800D4380020643A00204C3C0020A4707D3FAE
:10C82800C42E00207038002069E1050879E1050868
:10C83800000034C089E105089BE10508B7E1050857
:10C8480000B560EEA07A40EE007A2DED028B17EE6F
:10C85800900A87B0B0EE408AF0EE608A8DED020A49
:10C86800CDED030A04F058FD41EC100B07F012F867
:10C8780051EC100B05F086F8DFED117A07EE100A7F
:10C8880078EEA78A38EE078A68EEA87A48EE087A22
:10C89800C7EE277A17EE900A04F03EFD41EC100B24
:10C8A80006F0F8FF51EC100B05F06CF800EE900A5A
:10C8B80020EE880A60EEA80A07B0BDEC028B00BD26
:10C8C80000000000F0B52DED028BDFED3A1A3A4B6F
:10C8D8008DB030EEA17AF0EE407AB7EE001A8DED09
:10C8E800020A83ED001A30EE010AC3ED011A31EE97
:10C8F800671A71EEE01ACDED030AF0EE470A8DEDE6
:10C90800077A8DED081ACDED091A8DED060AFFF7A5
:10C9180036FE8DED000ACDED010A9DE8030004AB5B
:10C9280083E803009DED058ADDED048A68EE087A48
:10C9380048EEA87A17EE900A04F0EEFC41EC100BD2
:10C9480006F0A8FF18EE100A57EC106B04F0E4FC90
:10C95800044618EE900A0D4604F0DEFC45EC104B38
:10C9680041EC110B06F088FE3946304655EC104B69
:10C9780005F008F804F0D0FC41EC100B06F07EFE40
:10C98800002251EC100B0D4B04F01AFD04F0FAFFD5
:10C9980029460646204604F0F5FF00EE900AF6EE1A
:10C9A800007A60EEA70A00EE106A0DB0BDEC028BAB
:10C9B800F0BD00BF00000000A43C00200000E03FE4
:10C9C800F0EE407A86B020EE200A67EE810A06B0C3
:10C9D80070472DE9F04F2DED028B85B0FCF780F9FB
:10C9E80010EE105AFCF782F9284610EE104A04F0AF
:10C9F80093FC80462046894604F08EFC41EC100BDF
:10CA080041EC180B06F0DCFC57EC106BB0EE480A52
:10CA1800F0EE680A06F0D4FD32463B4640464946E9
:10CA28005BEC10AB04F0CCFC04F0ACFF9FED138A78
:10CA380007EE100ADFED127A57EE087A114C5B46C2
:10CA4800C4ED007A52464046494604F0B9FC04F069
:10CA580099FF07EE900A27EE888A04AB84ED018AD5
:10CA680094E8030003E90300DDED030A9DED020AE3
:10CA780005B0BDEC028BBDE8F08F00BF0000F042AE
:10CA880000008C42303D002030B53F4B2DED088B27
:10CA9800D3ED008AD3ED019A3C4BD3ED00AAD3ED38
:10CAA80001BA3B4B93ED008A93ED019A394B93ED14
:10CAB80000AA93ED01BA38EEEA0A79EEEB0A38EEED
:10CAC8004A1A79EE4B1A93B08DED0A0ACDED0B0A8E
:10CAD8008DED0C1ACDED0D1AFFF744FD8DED000A12
:10CAE800CDED010A9DE803003AEE6A0A7BEE6B0A77
:10CAF80004AB38EE681A79EE691A83E803008DED05
:10CB0800081ACDED091A8DED0E0ACDED0F0AFFF7C3
:10CB180029FD8DED000ACDED010A9DE8030006AB65
:10CB280083E803009DED040ADDED050A9DED061A74
:10CB3800DDED071AFFF723FD8DED000ACDED010AA3
:10CB48009DE8030002AD85E80300134B9DED021A32
:10CB580093ED000AD3ED010ADDED031AFFF702FD9C
:10CB68008DED000ACDED010A9DE8030012AB03E943
:10CB780003006C46DDED110A85E803009DED100AFF
:10CB880013B0BDEC088B30BD68380020C0380020D9
:10CB9800243D0020B43C0020883A0020F7EE007ABB
:10CBA80077EEC07A20EE022A20EE210A07EEA00ACC
:10CBB800F0EE420A47EE810A88B008B07047F8B52F
:10CBC800C400A4B204F58066B0B20F46FAF766FD59
:10CBD8001C4D0436B0B285ED000AFAF75FFD04F586
:10CBE8008646B0B285ED010AFAF758FD164D0436AF
:10CBF80085ED000AB0B2FAF751FDA4F5FC4085EDC9
:10CC0800010A80B2FAF74AFD104DA4F5FA40FC3843
:10CC180085ED000A80B2FAF741FD012F85ED010A82
:10CC28000FD1A4F57C5080B2FAF738FD084DA4F571
:10CC38007A547C3C85ED000AA0B2FAF72FFD85ED09
:10CC4800010AF8BD243D0020C0380020B43C002073
:10CC5800683800202DE9F04F2DED048B8046C1B0D7
:10CC68004FF47670FAF7D6FC04464FF47570FAF76D
:10CC7800D1FC064640F2DE30FAF7F4FC189040F298
:10CC8800E230FAF7EFFC19904FF47F70FAF7C2FC24
:10CC9800B8F1030F40F0E480189A199B00900192B4
:10CCA80002931EA874493246234609F043F9C1B2DB
:10CCB8001EA8FDF707FED9E001212046FFF77FFFF8
:10CCC800B8F1010F40F091806C4A6D4B10681E68F6
:10CCD800D2ED018A93ED019AF5EEC08A694BF1EE27
:10CCE80010FAD3ED019A54BF4FF0000C4FF0010C2D
:10CCF800B5EEC09A1F68644BBCF1000F0CBF4FF033
:10CD08002B094FF02D09F1EE10FA93ED018A54BF6B
:10CD18004FF0000E4FF0010EF5EEC09ABEF1000F75
:10CD28000CBF2B252D25F1EE10FA54BF002101214F
:10CD3800B5EEC08A00290CBF4FF02B0A4FF02D0A20
:10CD4800F1EE10FA54BF00220122D3F800B0002AF5
:10CD58000CBF2B232D23BCF1000F01D0F1EE688A04
:10CD6800BEF1000F01D0B1EE499A09B1F1EE699A0E
:10CD78000AB1B1EE488A179304F0CEFACDE91A0148
:10CD880018EE900ACDF8009004F0C6FACDE9020139
:10CD9800304604F0C1FACDE9040119EE100A0695EF
:10CDA80004F0BAFACDE90801384604F0B5FACDE93D
:10CDB8000A0119EE900ACDF830A004F0ADFACDE9D9
:10CDC8000E01584604F0A8FA179BCDE9100118EE99
:10CDD800100A129304F0A0FADDE91A23CDE9140130
:10CDE8001EA82A4909F0A6F82FE0B8F1020F2DD1A4
:10CDF800FFF74AFE8DED1C0ACDED1D0A1CAB93E82A
:10CE0800030040AB03E903009DED3F8AB5EEC08AFD
:10CE1800F1EE10FA03D5B1EE488A2D2600E02B2654
:10CE2800199A189B3E9802FB043504F075FACDE96F
:10CE3800000118EE100A029604F06EFA2A46CDE9AF
:10CE480004011EA8124909F075F8C5B21EA82946A2
:10CE5800FDF738FD01340120FEF744FAA4B200E0E2
:10CE680000240C4A1388A342BFF626AF41B0BDEC9C
:10CE7800048BBDE8F08F00BFC2E10508243D002007
:10CE8800C0380020B43C002068380020DFE10508E5
:10CE980011E205089C3C0020F0B52DED028B0446FC
:10CEA8008DB0002800F0D480714B18890419A4B201
:10CEB80022B2002A05DB40F23F139A42C8BF1C4643
:10CEC80000E00024F7F770FFA0B24EF29C71F7F76C
:10CED8007DFF674B1C81674B186804F01DFA5EA341
:10CEE800D3E9002304F06CFA04F04CFD624B18609F
:10CEF800624B1B780A2B054624B23DD107EE104A37
:10CF0800F8EEC77A17EE900A04F006FA5C4B06466C
:10CF180018680F4604F0EEF902460B4650A1D1E915
:10CF2800000104F077FB02460B463046394604F010
:10CF380047FA064628460F4604F0EEF902460B4625
:10CF48003046394604F03CFA00224E4B04F062FBAE
:10CF580004F018FD04F0E0F902460B4604A84A491B
:10CF680008F0E8FF0020F8F783FE0520D72104AA7F
:10CF78000023F8F7B5FE6BE0444B1888604304F0D3
:10CF8800B9F939A3D3E9002304F044FB04F0FAFC0F
:10CF98003F4B08EE100A1B68FCEEC87A07EE103A01
:10CFA80017EE905AF8EEC77A3A4B68EE277A1B6864
:10CFB800FDEEE77AADB217EE906A28460121F61821
:10CFC800FFF7FDFDFFF760FD8DED020ACDED030AC9
:10CFD80002AC94E8030008AB83E80300681C80B245
:10CFE8000121FFF7ECFDFFF74FFD8DED020ACDEDB6
:10CFF800030A94E803000CAB07EE105A03E9030098
:10D00800B8EEC70ADDED080A38EE400A9DED091AA8
:10D01800DDED0A1A9DED0B2AFFF7C0FD8DED020A22
:10D02800CDED030A94E8030006AB83E803004FF64E
:10D03800FF73009305200023DC213246FEF774FDC0
:10D04800154B9DED060A1878DDED070AFFF7DCFAA7
:10D058000DB0BDEC028BF0BD7B14AE47E17A843F86
:10D06800000000A0D954BD410000000000F073404A
:10D078001C0F0020D0030020183D00203428002079
:10D08800D42E00200000F43F24E205089C3C002038
:10D09800A82E0020B4280020C42E00202DE9F84333
:10D0A800461F8846B6B200250D4F12E008EB040172
:10D0B80089B23046F7F72CFE29F814000A2001340B
:10D0C800FBF74EFB062CF1D116350136F22DB6B220
:10D0D80004D06FF0040407EB0509E7E7BDE8F8831F
:10D0E800D43C00202DE9F04F85B00B1A0193431E64
:10D0F8009BB20293431C441F00F1060901F1FF3A59
:10D1080001F1010B9BB20F461646A4B21FFA89F92A
:10D118001FFA8AFA1FFA8BFB039380462046514672
:10D128003246F7F72DFE204639463246F7F728FEF5
:10D13800204659463246F7F723FE019B0298E51828
:10D14800ADB229463246F7F71BFE4046294632461D
:10D15800F7F716FE0134039829463246F7F710FE12
:10D16800A4B20A20FBF7FCFA4C45D7D105B0BDE8BC
:10D17800F08F2DE9F843461F8846B6B200250E4FBA
:10D1880012E008EB040139F8142089B23046F7F7A9
:10D19800F7FD01340A20FBF7E3FA062CF1D1163526
:10D1A8000136F22DB6B204D06FF0040407EB05097E
:10D1B800E7E7BDE8F88300BFD43C00202DE9F04341
:10D1C8002DED068B70EE007A8DB017EE900AB0EE5A
:10D1D800408A10EE904A20EE009A04F09DF8064628
:10D1E80020460F4604F098F8F7EE008A41EC100B41
:10D1F80041EC1A0B06F0E4F879EE287A55EC104B5E
:10D2080017EE900A04F088F82246804689462B4695
:10D218003046394604F0D4F802460B4640464946A3
:10D2280003F01AFF04F0AEFBB0EE4A0AF0EE6A0A09
:10D2380009EE900A38EEC99ADFED377A89EE299A15
:10D2480029EE279A06F0BCF9304653EC102B3946E4
:10D2580004F0B6F8044619EE900A0D4604F05CF89E
:10D2680002460B462046294604F0D4F900222B4BEF
:10D2780004F0A6F804F086FBB4EE688ADFED287A9D
:10D28800284BF1EE10FA044619EE100A08BFB0EE6A
:10D29800678A1D6804F040F802460B4603A8224935
:10D2A80008F048FE204604F037F802460B4606A868
:10D2B8001E4908F03FFE78EE287A38EEC88A87EED5
:10D2C800888A18EE100A04F027F802460B4609A8C7
:10D2D800174908F02FFE0520014603AA0023F8F796
:10D2E800FFFC0520142106AA0023F8F7F9FCC82042
:10D2F800052109AA0023F8F7F3FC4FF6E073009321
:10D308000520DC212A460023FEF70EFC0DB0BDECFB
:10D31800068BBDE8F08300BF00004842000049408A
:10D32800A4707D3F803A00202DE2050871E10508D0
:10D3380035E205082DE9F04F494B2DED048B1D789A
:10D34800022D85B080467BD1464E348A0121204685
:10D35800FFF735FCFFF798FB8DED000ACDED010ACC
:10D368009DE8030004AB03E9030028469DED020A8B
:10D37800DDED030AFFF748F93B4B1A683B4B1B6886
:10D3880002FB04343A4B1C603A4BDFED3B7A93EDD9
:10D39800008A68EE277A5F6817EE900A03F0BCFFF0
:10D3A800824638468B4603F0B7FF41EC100B41EC40
:10D3B800190B06F005F8504653EC102B594603F0AC
:10D3C800FFFF23A3D3E9002303F048FE04F0BAFAD1
:10D3D800B0EE490AF0EE690A054684B206F0F0F8A4
:10D3E800504653EC102B594603F0EAFF0B46024611
:10D3F80019A1D1E9000103F02FFE04F0A3FAB37CD0
:10D4080081461FFA80FA1BB9B08AF18AFFF7B1FE8C
:10D41800002320465146B374FFF740FE204651468C
:10D428001F22FFF75FFEB0EE480A00EE907AFFF782
:10D43800C5FE338AB5829844A6F81080A6F81690DF
:10D4480005B0BDEC048BBDE8F08F00BFAFF30080E2
:10D458000000000000E063400000000000C05D40E4
:10D46800C42E00201C0F0020A82E0020B428002065
:10D47800803A00204C3C00200000C842124B1B7828
:10D48800022B10B50CD1114B1B78022B08D1104C74
:10D498002078C0B140B2FFF74DFF0023237010BDC4
:10D4A8000C4C237E23B99F20F7F758FC01232376E1
:10D4B800064B1B78022B06D1054C94F90000FFF7A8
:10D4C800EBFC0023237010BDC42E0020A43A0020DA
:10D4D800E91B00201C0F0020034B00201860034BA1
:10D4E8001870FEF727B800BFAC380020A43A002017
:10D4F800034B00201860034B02221A70FEF71AB87B
:10D50800AC380020A43A002037B500242546A0B244
:10D5180028213223024601340095F8F733FAB4F58E
:10D52800A07FF4D13EBD2DE9F04F2DED088B0228E8
:10D5380097B080468DED070AB34B05D0032805D078
:10D54800012805D10C2202E0092200E00B221A7002
:10D558001878F3F7C1FA042103914FF00009F3EEAC
:10D568000EAA9FEDAABADFEDAABA7DE1A94B1A6807
:10D57800A94B1B6802FB093307EE103A01211FFA79
:10D5880089F0B8EEC78AFFF71AFBFFF77DFA8DED31
:10D59800080ACDED090A08AD95E803000AAB83E84F
:10D5A80003009E4B1A6802EBC9030EAF19689C4B27
:10D5B80019600399521812685A60FFF765FA8DEDE1
:10D5C800080ACDED090A95E803000CAB83E80300CF
:10D5D800DDED0A9A9DED0BAADDED0C8A9DED0D9A05
:10D5E800B0EE690AF0EE4A0AB0EE681AF0EE491A8F
:10D5F800FEF7B8FF8DED080ACDED090A95E803009E
:10D60800B0EE691AF0EE4A1A87E80300B0EE680A2D
:10D61800F0EE490AFEF7B3FF8DED080ACDED090AD1
:10D6280095E8030010AB83E803009DED0E0ADDEDDD
:10D638000F0AFFF705F98DED080ACDED090A95E8FF
:10D64800030016AA02E903009DED100ADDED110A98
:10D65800149EFFF7F5F88DED080ACDED090A95E857
:10D66800030087E80300DDED0F0AF5EEC00AF1EECE
:10D6780010FA48BFF1EE600A9DED0E0ACDED0F0AD3
:10D68800FFF720F98DED080ACDED090A08AA92E8FE
:10D69800030012AB83E803000798129D03F03CFED9
:10D6A8005D4B139FD3F800B05E4BBDEEC87AD3F83C
:10D6B80000A0CDE9040117EE102A58465146FEF79E
:10D6C800F9F807EE10AAF8EEC77A07EE10BAB4EE2A
:10D6D800E78AF8EEC77AF1EE10FAB4EEE78A8CBF63
:10D6E80000220122504B0690F1EE10FAD4BF00221E
:10D6F80002F00102B8F1020FDA6012D0B8F1030F9C
:10D708003ED0B8F1010F68D1304603F005FE36A3CC
:10D71800D3E9002303F054FE0022444B03F09EFC9F
:10D728002AE0284603F0F8FDDDE9042304460D4607
:10D738002FA1D1E9000103F06DFF02460B462046F8
:10D74800294603F03DFE2CA3D3E9002303F038FE5D
:10D7580004F018F907EE900AC7EEAA7A17EE900AB5
:10D7680003F0DAFD41EC100B06F00EF8002251EC44
:10D77800100B2F4B03F024FE04F0BCF804462CE0F9
:10D7880018EE100A03F0C8FD044638460D4603F0AB
:10D79800C3FD17A3D3E9002303F012FEDDE9042338
:10D7A80003F038FF04F0EEF803F0B6FD14A3D3E954
:10D7B800002303F005FE02460B462046294603F0E7
:10D7C80029FF04F0DFF807EE900AB0EE6B7A07EE57
:10D7D8008B7AFDEEC77A17EE904A002C2ADBC72C0D
:10D7E800A8BFC72427E000BF8716D9CEF753F5BFD7
:10D7F8008FC2F5285CAF43400000000000907040E5
:10D8080000000080DBC48641C42E00200000C8C38D
:10D818000000C843A82E0020B42800209838002013
:10D8280068380020D42E00201C0F0020000069401A
:10D83800000049C00024114BDB685BB1104B18880D
:10D84800104B1988069B4FF6FF759AB2A3B2009544
:10D85800F8F798F80B4B039A1C600699084B0832A6
:10D86800196009F101090392074B1B884B45BFF664
:10D878007DAE17B0BDEC088BBDE8F08F1C0F002003
:10D88800983A0020383D00209C3C0020F0B51E4B03
:10D898001E4F18781E4D1F4E85B0F3F71DF91E4B0D
:10D8A8000B221A70002423E01C4B1A68336802FB11
:10D8B80004336B611A4B20461C840121FFF77FF962
:10D8C800FFF7E2F88DED000ACDED010A9DE80300AF
:10D8D80004AB03E903000C4B9DED020A1878DDED5B
:10D8E800030AFEF791FE6869FEF7C8F90134A4B28D
:10D8F8003B88A342D8DA0B4B02221A700A4B00224B
:10D908001A7605B0F0BD00BFC42E00209C3C002054
:10D91800643A0020AC280020342800203028002059
:10D928004C3C0020A43A00201C0F002030B52D4D9F
:10D9380095F9003085B0002B3CD0FDF711FC2A4A40
:10D948002A4B11682A4C526819605A60608B002172
:10D95800FFF735F9FFF798F88DED000ACDED010ACC
:10D968009DE8030004AB03E90300224B9DED020A86
:10D97800DDED030A1878FEF747FE1F4B628B186827
:10D988001E4B1B6800FB0230FEF778F995F9002062
:10D99800638BD3181A4A10681A4A12689BB200FBA4
:10D9A80003206383FBF712FB174B1868FDF79AFCFB
:10D9B80000232B700E4C154B628B1B889A420ED19C
:10D9C8004FF08040002102F056FD0E4B1868FBF71F
:10D9D800FDFA0F4B02221A7000236383237605B0E9
:10D9E80030BD00BFAC3C0020643A002068380020FD
:10D9F8001C0F0020C42E0020A82E0020B4280020D0
:10DA080030280020AC280020602800209C3C002002
:10DA1800A43A00207FB54FF08040012102F02BFD91
:10DA2800FDF79EFB264A274B1168526819605A6019
:10DA3800254C264B22681B68254DD31A06EE903AD2
:10DA4800B8EEE67AD5ED006AF8EEE67A0021C7EE80
:10DA5800277AFCEEE77A17EE906AB0B2FFF7AFF8D4
:10DA6800FFF712F88DED000ACDED010A9DE80300DD
:10DA780004AB03E9030000209DED020ADDED030A73
:10DA8800FEF7C2FD134B1868134B1B6836B200FB38
:10DA98000630124EFEF7F2F81920FDF723FC307815
:10DAA80060B12A68236840B202FB0030FBF78EFAA7
:10DAB8000B4B1868FDF716FC002333707FBD00BFC1
:10DAC800643A002068380020A0380020AC280020E4
:10DAD80030280020A82E0020B4280020AC3C0020CC
:10DAE8006028002010B500214FF0804002F0C3FCF0
:10DAF800094B00241C702046F7F7E4FF074B186811
:10DB0800FBF764FA064B074801221A70064B1C7093
:10DB1800BDE81040F3F7EBBDB0380020AC2800207A
:10DB2800C42E0020041A00203428002007EE100A12
:10DB3800034BF8EE477A0022C3ED007A5A6070472B
:10DB4800D438002007EE100A034BF8EE477A00227B
:10DB5800C3ED007A5A607047883A00200F4B10498D
:10DB68001A68104B1B68D31A06EE903A0E4B1B68C6
:10DB7800B8EEE67A06EE903AF8EEE67AC7EE277A3D
:10DB8800FCEEE77A17EE903A9AB20B80074B1888AA
:10DB980090422CBF00200120704700BFD42E0020E7
:10DBA8009C3C0020B4280020A82E0020B02800208B
:10DBB80013B502AB011D23ED010A054A89B213F81A
:10DBC800014B1454013080B28842F8D11CBD00BF0B
:10DBD800E23900202DE9F8431F4C0440002C05468B
:10DBE8000E4603DA013C64F00F040134DFF8748058
:10DBF8004FEAC4091FFA89F9484698ED000A09F165
:10DC08000409FFF7D5FF1FFA89F098ED010AFFF71D
:10DC1800CFFF124B10271B8895FBF7F7FF019D429A
:10DC2800BFB20CD1B81980B20D498022FAF738FE7C
:10DC380000B1FEE729B24FF47F70F9F7DDFC0F2C35
:10DC480007D1BE19B0B206498022FAF729FE00B101
:10DC5800FEE7BDE8F88300BF0F0000809C3C002071
:10DC6800E2390020643A00202DE9F043744B2DED91
:10DC7800028B1888FF2898BF4FF4807093B0C000BB
:10DC880007F0E6FD6F4B0546186028B90520B4215A
:10DC98006D4A2B46F8F724F80024694F6B4E4FF075
:10DCA80000086AE0FDF75CFA20464FF44141FFF7AF
:10DCB80091FF674B1A685B683260002173602046E9
:10DCC800FEF77DFFFEF7E0FE8DED020ACDED030ABB
:10DCD8000DF1080999E803000AAB83E803005D4BDE
:10DCE8009DED0A1A93ED007AD3ED017ADDED0B1A5A
:10DCF80031EE470A71EEE70A31EE071A71EEA71AFC
:10DD08008DED0E0ACDED0F0A8DED101ACDED111A1D
:10DD1800FEF735FC8DED020ACDED030A99E8030004
:10DD28000CAB83E80300FF2C4FEAC4032B4404D94F
:10DD3800C3F80080C3F8048003E00C9A1A600D9AB7
:10DD48005A603B8840F23F10604390FBF3F080B28A
:10DD58004FF4FC630246282100933223F7F712FEA2
:10DD68003D4B18683D4B1B68C018FBF72FF93C4B1F
:10DD78001868FDF7B7FA0134A4B23B88A34291DAD8
:10DD8800012213464FF4807105A804F00DFE354EAC
:10DD9800DFF8F880294605A805F0E8F8082333706D
:10DDA800314B01241C700020F7F75AF92F48F3F77C
:10DDB8009EFC3078F2F790FE2D4B9FED2E8ADFED1A
:10DDC8002E8A1C700024D5ED007AB0EE687A07EE32
:10DDD800C87A2046FCEEC77A17EE906A03F08AFAF2
:10DDE800264B002203F0ECFA03F0ACFDB6B2A3B266
:10DDF800C72E28BFC72687B253B1214BB8F80000F9
:10DE080019884FF6FF7300933A463346F7F7BAFD81
:10DE18001B4BC8F8007001340835B4F5807F1E60CC
:10DE2800D1D1184B1868FBF7D1F8114B02221A70A0
:10DE3800154B00221A7613B0BDEC028BBDE8F083B7
:10DE48009C3C0020983800205CDA050868380020DF
:10DE5800643A0020D4380020A03800203028002060
:10DE680060280020C42E0020E10E00206019002048
:10DE7800A43A0020000016430000C8420000F43F06
:10DE8800383D0020AC2800201C0F0020983A0020C4
:10DE9800F0B5294B294F2A4D2A4E012285B01A7018
:10DEA80000243AE0284B1A68336802FB04336B619C
:10DEB800264B1C84FDF754F920464FF44141FFF7E7
:10DEC80089FE234B2A681A606A6820465A60002136
:10DED800FEF775FEFEF7D8FD8DED000ACDED010ABF
:10DEE8009DE8030004AB03E903001A4B9DED020A09
:10DEF8001878DDED030AFEF787FB6869FDF7BEFEBB
:10DF0800154B1868154B1B68C018FBF75FF8144BC6
:10DF18001868FDF7E7F90134A4B23B88A342C1DAD7
:10DF2800104B1868FBF752F8034B02221A700E4B7D
:10DF380000221A7605B0F0BDA43A00209C3C0020CF
:10DF4800643A0020B4280020A82E00204C3C002071
:10DF580068380020C42E0020A03800203028002077
:10DF680060280020AC2800201C0F002038B5FDF7E1
:10DF78003DFD124B124D9F221A81124B0124187835
:10DF88002C70F2F7A9FD104B00221A600F4B1B787A
:10DF9800072B04D00B2B0DD0062B0ED102E0BDE8C9
:10DFA800384075E74FF0804021462C70BDE8384076
:10DFB80002F061BABDE8384068E438BD1C0F0020A3
:10DFC800A43A0020C42E0020AC38002034280020B9
:10DFD8002DE9F743002581462C46154E154FDFF8ED
:10DFE8005C801FE0FDF7BCF849462046FFF7F2FDCC
:10DFF800D8F800303868C018FAF7E8FF0E4B1868F0
:10E00800FDF770F9308895FBF0F080B24FF4FC63AF
:10E018000093282102463223F7F7B4FC05F59E75D4
:10E02800013403353388A342DCDABDE8FE8300BF40
:10E038009C3C0020A03800206028002030280020C8
:10E0480010B5104C4FF47570B4F90010F9F7D4FA04
:10E058000D4B4FF47670B3F90010F9F7CDFA40F292
:10E06800D230F9F7D7FAB02804D040F2D230B02134
:10E07800F9F7C2FA2088FFF759FD034B1888BDE865
:10E0880010405FE5780200207402002000210A2277
:10E0980008B509F09FF8D0F1010038BF002008BD8D
:10E0A80073B5041D0E46A4B20C2200234FF6E0758A
:10E0B800204601360095F7F709FD00230C22B1B27E
:10E0C80020460095F7F702FD0D4B1B78012B16D162
:10E0D8000C4E0D4D308829880024043080B20C2263
:10E0E80023460094F7F7F2FC30882988009404301E
:10E0F800013180B289B20C222346F7F7E7FC7CBDD8
:10E108008C380020D2380020843A002008B54FF619
:10E11800FF70F7F7ABFC0020F7F7AAFD2148FFF7DF
:10E12800B5FF20B11F482049012207F003FF4B200B
:10E1380023211C4A0023F7F7D3FD1C48FFF7A6FF4D
:10E1480020B11A481849012207F0F4FE4B20462155
:10E15800164A0023F7F7C4FD1548FFF797FF20B1CB
:10E1680013481149012207F0E5FE4B206921104AA6
:10E178000023F7F7B5FD0F48FFF788FF20B10D48DA
:10E188000949012207F0D6FE4B208C210023094AB9
:10E19800F7F7A6FD084B1888084B1988BDE8084012
:10E1A8007EE700BF7828002006D60508A0280020B2
:10E1B800B62E002064280020AE3C00207C3C0020C5
:10E1C80070B5044600200D461646F7F751FD0020AD
:10E1D800F7F762FC4FF4FC60F7F748FC2046294645
:10E1E80056BB1E4A3346F7F77BFD1D48FFF74EFF27
:10E1F80020B11B481B49012207F09CFE04F1700660
:10E20800B6B230462946164A0023F7F769FD164884
:10E21800FFF73CFF20B114481249012207F08AFE9B
:10E228003235ADB220462946104A0023F7F758FD8B
:10E23800304629460C4A07E00D4A0023F7F750FDFF
:10E2480032350B4AA9B220460023F7F749FD094B9E
:10E258001888094B1988BDE8704021E741E2050894
:10E268001C3D002004DA0508903C002049E205081E
:10E27800A7DA0508AE3C00207C3C002030B5144DE0
:10E288009DF80C402C70134D2880134D02FB0400A0
:10E298002980124D80B22880114D2980114D2A8085
:10E2A800114A1380114B1880114B1980114B1249D8
:10E2B800E2B21A7000230B7010490A709DF8102002
:10E2C8000134013254430E4A14700E4A137030BDA3
:10E2D800343E0020143D0020623A0020AE3C00206D
:10E2E8007C3C0020E0390020403D0020D23800204E
:10E2F800843A00207E3C0020B1380020B03C002049
:10E308008D3800208C38002038B5054600200C4692
:10E31800F7F7AEFC0020F7F7BFFB4FF4FC60F7F708
:10E32800A5FB0B48FFF7B2FE28B1094809490A4B7B
:10E33800002207F0FFFD284621460023044AF7F78C
:10E34800CFFC064B1888064B1988BDE83840A7E66D
:10E35800C838002063DF05080000F03FAE3C00200D
:10E368007C3C002038B5054600200C46F7F780FCB9
:10E378000020F7F791FB4FF4FC60F7F777FB0B48A9
:10E38800FFF784FE28B1094809490A4B002207F023
:10E39800D1FD284621460023044AF7F7A1FC064B85
:10E3A8001888064B1988BDE8384079E6A43800205B
:10E3B80063DF05080000F03FAE3C00207C3C0020F5
:10E3C80070B53020002108222A4E2B4CF9F7AAFFFD
:10E3D8000023337020E0172B04D1302000210922BC
:10E3E800F9F7A0FF00232370244D0EE032780321B3
:10E3F8004A43D118AA18D318695C93F84B203020E7
:10E40800F9F790FF2378013323702378194A022BF8
:10E41800ECD91378013313703378164D182BDAD9E9
:10E4280000232B70144C20E0152B04D13020002140
:10E438000A22F9F777FF00232370104E0EE02B789D
:10E44800032101FB03639A18302092F8961092F882
:10E458004B20F9F767FF2378013323702278054BA7
:10E46800022AECD91A7801321A702B78182BDBD9CA
:10E4780070BD00BFE01B0020353E0020D8030020FF
:10E488000EB403B070470A2810B5044602D10D2017
:10E49800FFF7F9FF064A13681BB103F8014B136035
:10E4A80010BD044B1B680BB12046984710BD00BF38
:10E4B8003C0F0020383E002010B5044601E0FFF76D
:10E4C800E2FF14F8010B0028F9D110BD2DE9F04F37
:10E4D800044685B00D464FF00A0A00E0354620781C
:10E4E800002800F0C480252801D0013467E0607856
:10E4F800302803D1A0780123033407E02D2802D067
:10E508000234002302E0A078022303344FF000080D
:10E5180005E00AFB080814F8010BA8F13008A0F17F
:10E528003002D2B2092AF4D96C2801D04C2803D180
:10E5380014F8010B43F00403002800F098806028C9
:10E5480086BFA0F12002D2B202464F2A3DD006D89B
:10E55800432A2DD0442A09D0422A30D133E0552A03
:10E5680004D0582A29D0532A29D101E00A272DE0BE
:10E578002E1D2F68002500E001357A5D002AFBD1A9
:10E5880004E02020FFF77FFF4D4601E0980704D400
:10E59800454505F10109F4D34D463846FFF78CFF90
:10E5A80003E02020FFF76FFF01354545F9D395E7D4
:10E5B80028782E1DFFF767FF90E7102706E0FFF782
:10E5C80062FF2E468AE7022700E008272E1D442A0C
:10E5D800296804D1002902DA494243F008030022DD
:10E5E80000E02A46B1FBF7FE07FB1E11CDB2092D4C
:10E5F800714607D9782814BF4FF0070C4FF0270C45
:10E608006544EDB230350DF80250551CBEF1000FCF
:10E6180002D0102DE5D10F22190705D504A94D19EF
:10E628002D2105F8101C951C13F0010F0CBF4FF09D
:10E63800200B4FF0300B9B072F4604D508E05846B7
:10E64800FFF721FF4F46474507F10109F7D34F462A
:10E65800013D1DF80500FFF716FF002DF8D103E076
:10E668002020FFF710FF01374745F9D336E705B0FB
:10E67800BDE8F08F70B5064D0C462E68286001E0A5
:10E68800FFF701FF14F8010B0028F9D12E6070BDC7
:10E69800383E00200FB407B504A951F8040B0191C6
:10E6A800FFF714FFBDE80E4004B070470EB417B56D
:10E6B80005A9084C51F8043B206018460191FFF762
:10E6C80005FF2268002313702360BDE81E4003B0D5
:10E6D800704700BF3C0F00200EB433B505A9074CA6
:10E6E80051F8043B2568206018460191FFF7EEFEBB
:10E6F8002560BDE83C4003B0704700BF383E0020AD
:10E7080070B51E4604461C481546FFF7C3FF022E87
:10E718001FD0042E25D0012E2AD105E0A15D17486F
:10E72800FFF7B8FF013600E00026AE42F6DB2020F6
:10E73800FFF7A9FE002609E0A05DA0F12003DBB2E7
:10E748005E2B88BF2E20FFF79EFE0136AE42F3DB1C
:10E758000EE034F8021B0A48FFF79CFF013DF8D190
:10E7680006E054F8041B0748FFF794FF013DF8D171
:10E778000A20BDE8704086E651E2050858E205081F
:10E788005EE2050864E2050808B501214FF48070CF
:10E7980001F07CFA4FF480700021BDE8084001F0D8
:10E7A80075BA43680A6823F0407323F480731343EF
:10E7B8000A7943EA02234360CA680B6930B51A43F1
:10E7C80084688D68084B2A43234013434A7943EAF7
:10E7D800420383600B7DC26A013B22F47002DBB204
:10E7E80042EA0353C36230BDFDF7FFC00023036054
:10E7F800037143718360C36003610123037570472C
:10E80800074A084B516810B50B4090E812002143A5
:10E818008468C068214301430B43536010BD00BFA7
:10E8280000230140E030FCFF002303604360836065
:10E83800C3607047836811B143F0010301E023F01E
:10E84800010383607047436823F4400323F4007393
:10E858000B4343607047416282627047436823F00C
:10E868001F030B4343607047044B5A6810B142F4CE
:10E87800000201E022F400025A60704700230140C0
:10E88800044B5A6810B142F4800201E022F480027D
:10E898005A60704700230140092970B50CB20CD9A1
:10E8A80004EB44041E3CC6680725A54026EA050576
:10E8B800A34045EA0304C4600AE0066904EB440483
:10E8C8000725A54026EA050513FA04F42C4304613C
:10E8D800062A0CD80523013A5A43446B1F23934058
:10E8E80024EA0303914043EA0102426370BD0C2A03
:10E8F80012B20CD802EB8202233A046B1F23934016
:10E9080024EA0303914043EA0102026370BD02EB6B
:10E918008202413AC46A1F23934024EA03039140C8
:10E9280043EA0102C26270BD836843F0804383609A
:10E9380070478068C0F380507047836811B143F412
:10E94800806301E023F4806383607047836811B1BA
:10E9580043F0020301E023F0020383607047436839
:10E96800013923F4604343EA413343607047436805
:10E9780011B143F4006301E023F40063436070477E
:10E98800C06C80B27047014B18687047082301407B
:10E99800836811B143F4807301E023F480738360CA
:10E9A8007047836811B143F4007301E023F40073E6
:10E9B80083607047044B5A6810B142F4005201E07A
:10E9C80022F400525A60704700230140092970B5AB
:10E9D8000CB20CD904EB44041E3CC6680725A540BC
:10E9E80026EA0505A34045EA0304C4600AE006696F
:10E9F80004EB44040725A54026EA050513FA04F4A8
:10EA08002C430461836BC3F30154121B0232D2B24C
:10EA180002EB82021F24944023EA040391400B4333
:10EA2800836370BD836B013923F4401343EA0153B8
:10EA38008363704782B0002301930190019BCB1838
:10EA48000193019B1A6002B07047836823F4702316
:10EA58000B4383607047836823F440130B43836040
:10EA68007047836843F48003836070478068C0F30D
:10EA780080507047436811B143F4806301E023F488
:10EA8800806343607047436811B143F4805301E0E9
:10EA980023F480534360704782B0002301930190B0
:10EAA800019B28335B180193019B186880B202B060
:10EAB80070470123C9B213FA01F143680AB1194337
:10EAC80001E023EA010141607047036819420CBF65
:10EAD800002001207047C9430160704743680068FF
:10EAE80010EA112007D00122C9B212FA01F1194225
:10EAF8000CBF0020012070476FEA112101607047A8
:10EB0800036823F00103036000230360436083600C
:10EB1800C3600361212343612C4B98421CD02C4BCA
:10EB2800984220D02B4B984225D02B4B98422AD084
:10EB38002A4B98422FD02A4B984233D0294B9842DF
:10EB480037D0294B984204D14FF03D5243F8AC2CB2
:10EB58007047264B984203D13D2243F8082C704752
:10EB6800234B984204D14FF4746243F8202C704729
:10EB7800204B984204D14FF4741243F8382C704754
:10EB88001D4B984204D14FF0746243F8502C7047E3
:10EB98001A4B984203D11A4A43F8642C7047194B10
:10EBA800984203D1184A43F87C2C7047174B984277
:10EBB80003D1174A43F8942C7047164B984204BF68
:10EBC8004FF03D5243F8AC2C704700BF1060024034
:10EBD8002860024040600240586002407060024075
:10EBE80088600240A0600240B860024010640240A1
:10EBF8002864024040640240586402407064024045
:10EC08003D00002088640240400F0020A0640240BC
:10EC180000003D20B86402400268134B10B5134051
:10EC2800CC680A6822434C6922438C692243CC6928
:10EC380022430C6A22434C6A22438C6A22434C6B5F
:10EC480022438C6B22431343036042690C6BCB6AEB
:10EC580022F007022343134343610B6943604B6867
:10EC680083608B68C36010BD3F801CF00023036085
:10EC780043608360C360036143618361C36103626E
:10EC880043628362C36203634363836370470368B9
:10EC980011B143F0010301E023F001030360704761
:10ECA800036811B143F4004301E023F40043036017
:10ECB8007047036811B143F0200301E023F02003FB
:10ECC8000360704741607047406880B270470368CE
:10ECD80012B143F4002301E023F40023036001612F
:10ECE8007047036811B143F4802301E023F48023C3
:10ECF800036070470AB101617047C16070470068DE
:10ED0800C0F3C0407047006800F0010070474069D8
:10ED180000F0380070470A4A0A4B10B50A4CA04266
:10ED280088BF13468A004CBF5B681B6821F0F0213E
:10ED380021F0821119420CBF0020012010BD00BF34
:10ED480000640240006002400F64024010B5084BA6
:10ED5800084A094CA04288BF134611F0005F21F011
:10ED6800F02121F0821114BFD960996010BD00BF55
:10ED780000600240006402400F6402400B0607D5A1
:10ED8800436912B143F0800301E023F0800343613B
:10ED9800802909D001F01E01036812B119430160EE
:10EDA800704723EA010101607047124B124A10B5FF
:10EDB800124CA0428CBF14461C4621F0F02323F0CD
:10EDC800C3132BB1026802F01E0202EAD12202E04C
:10EDD800426902F0800288004CBF6368236821F012
:10EDE800F02121F08210184002D0101C18BF012019
:10EDF80010BD00BF00600240006402400F64024082
:10EE080010B5084B084A094CA04288BF134611F0B8
:10EE1800005F21F0F02121F0821114BFD9609960C0
:10EE280010BD00BF00600240006402400F64024051
:10EE3800044B00221A605A609A60DA60024A5A61EA
:10EE4800704700BF003C0140FFFF7F00837910B589
:10EE5800002B29D01A4B01681C68CA4314401C6057
:10EE68005C6822405A60027902F1804202F59E32C3
:10EE780014682143116002689C68D1430C409C606F
:10EE8800DC682140D9604179102906D1996811437D
:10EE98009960D9680A43DA6010BD01F1804303F52F
:10EEA8009E3319680A4308E00379016803F1804337
:10EEB80003F59E331A6822EA01021A6010BD00BFEA
:10EEC800003C014000230C220360037142718371EE
:10EED8007047024B1A6902431A617047003C0140AF
:10EEE800034B5B6918420CBF00200120704700BF2C
:10EEF800003C0140014B5861704700BF003C014095
:10EF0800054B1A685B69034004D010420CBF00200F
:10EF18000120704718467047003C0140014B58617A
:10EF2800704700BF003C01404FF0204318B943F23E
:10EF3800DB021A6003E043F2D20243F820204FF0CC
:10EF48002042411C6FF0704342F8213002F5827272
:10EF580042F82030704770B584684568C368C16A54
:10EF6800026825431D4303691D4343691D438369A3
:10EF78001D43C3691D43036A1D43436A1D43836AD6
:10EF88001D43036B0D431D434FF02043082C43F8EA
:10EF9800225005D153F8224044F0400443F822405F
:10EFA800436B9E691D6835435E6845EA06159E6891
:10EFB80045EA0625DE6845EA06451E695B6945EAB5
:10EFC8000655541C45EA03654FF02043B1F5804FC0
:10EFD80043F8245010D1836B986919680143586825
:10EFE80041EA0011986841EA002118695B6941EA21
:10EFF800005141EA036101E06FF07041014B43F8B1
:10F00800221070BD040100A0022242604FF4805219
:10F018004262416B4FF4005210B5826200230F2206
:10F02800FF2403608360C360036143618361C3613C
:10F038000362C36203630A604A608C60CA600A6143
:10F048004A618B61816B0A604A608C60CA600A61A0
:10F058004A618B6110BD4FF0204321B153F8202045
:10F0680042F0010203E053F82010024A0A4043F834
:10F0780020207047FEFF0F0010280CBF064B074BDF
:10F088004FF040024FF0180119605A604FF0FC32FF
:10F098009A60DA60704700BF600000A0800000A09E
:10F0A80030B5836844681C43C36844F008041C43B3
:10F0B80003691C43436944EA4324836944EA4334AB
:10F0C800C36999685A68090441EA02211A68DB6829
:10F0D800114341EA0361036A9A685D68120442EACF
:10F0E80005221D68DB682A4342EA03620368102B85
:10F0F8000CBF034B034B1C609960DA6030BD00BF46
:10F10800600000A0800000A010230360C2690023F3
:10F1180043608360C360036143618361FC231360C0
:10F1280053609360D360026A136053609360D36046
:10F13800704741B110280CBF074B084B1A6842F0C2
:10F1480004021A60704710280CBF034A034A044B94
:10F1580011680B4013607047600000A0800000A099
:10F16800FBFF0F0041B110280CBF084B084B1A6871
:10F1780042F040021A60704710280CBF034A044A44
:10F18800044B11680B401360704700BF600000A07B
:10F19800800000A0BFFF0F00102802D1024B586961
:10F1A8007047024B58697047600000A0800000A0BB
:10F1B800054B18221A6000225A604FF0FC329A6000
:10F1C800DA601A61704700BFA00000A002684368B7
:10F1D80042F0100242EA4322836842EA4332144B67
:10F1E80010B51A60C26891685468090441EA04219C
:10F1F8001468D268214341EA02629A600269916800
:10F208005468090441EA04211468D268214341EA98
:10F218000262DA60426991685068090441EA002193
:10F228001068D268014341EA02621A6110BD00BF4A
:10F23800A00000A0C2680023036043608360FC2331
:10F24800136053609360D3600269136053609360E6
:10F25800D3604269136053609360D3607047054B75
:10F2680018B11A6842F0040202E01968024A0A401A
:10F278001A607047A00000A0FBFF0F0062B11028C1
:10F2880001D10E4B03E0B0F5807F03D10C4B5A68D7
:10F29800114311E00B4BFAE7102804D1074B5A68C9
:10F2A80022EA010108E0B0F5807F0CBF044B054B52
:10F2B8005A686FEA0101114059607047600000A068
:10F2C800800000A0A00000A0102801D1064B04E097
:10F2D800B0F5807F0CBF054B054B5B680B420CBF3C
:10F2E80000200120704700BF600000A0800000A03F
:10F2F800A00000A0102804D1074B5A6822EA010197
:10F3080008E0B0F5807F0CBF044B054B5A686FEAE4
:10F318000101114059607047600000A0800000A002
:10F32800A00000A0102801D1084B04E0B0F5807FB0
:10F338000CBF074B074B5B6813EA010004D013EAC4
:10F34800D1010CBF00200120704700BF600000A061
:10F35800800000A0A00000A0102804D1084B5A6823
:10F3680022EAD10109E0B0F5807F0CBF054B064BBE
:10F378005A684FEAD10122EA01015960704700BF7B
:10F38800600000A0800000A0A00000A008B52C4BE1
:10F39800984205D10120014600F048FC012048E0D0
:10F3A800284B984205D10220012100F03FFC0220A1
:10F3B8003FE0254B984205D10420012100F036FC9E
:10F3C800042036E0214B984205D10820012100F0A5
:10F3D8002DFC08202DE01E4B984205D1102001215C
:10F3E80000F024FC102024E01A4B984205D120207C
:10F3F800012100F01BFC20201BE0174B984205D18F
:10F408004020012100F012FC402012E0134B9842EA
:10F4180005D18020012100F009FC802009E0104B73
:10F4280098420BD14FF48070012100F0FFFB4FF49C
:10F4380080700021BDE8084000F0F8BB08BD00BF9F
:10F44800000002400004024000080240000C024094
:10F45800001002400014024000180240001C024044
:10F46800002002402DE9F0470023D1F800801A4619
:10F478004FF0010C03270CFA02F404EA0805A54230
:10F488002ED1066817FA03F4E443264006600E7985
:10F49800D0F8009006FA03FA013E4AEA0909012E5B
:10F4A800C0F8009014D8866891F8059026408660C8
:10F4B800866809FA03F949EA06068660466826EA74
:10F4C800050545608D7946689540ADB23543456080
:10F4D800C5682C40C460CC79C5689C402C43C46086
:10F4E80001320233102AC6D1BDE8F0874FF6FF7308
:10F4F80003600023037143718371C371704782B045
:10F508004FF480330193019B0B430193019BC3612B
:10F51800C161019BC361C3690193C369019302B0CF
:10F528007047036919420CBF002001207047006929
:10F5380080B27047436919420CBF00200120704710
:10F54800406980B2704701837047418370470AB1B0
:10F5580001837047418370474161704743694B405D
:10F568004361704701F00703C908083130B59B00B3
:10F5780050F821500F249C4025EA040440F821400B
:10F5880050F8214012FA03F31C4340F8214030BDE3
:10F5980008B5134B984207D14FF40010012100F031
:10F5A80069FB4FF4001014E00E4B984207D14FF45A
:10F5B8008000012100F05EFB4FF4800009E00A4B57
:10F5C80098420BD14FF40000012100F053FB4FF497
:10F5D80000000021BDE8084000F04CBB08BD00BF9A
:10F5E8000054004000580040005C00407FB50446CD
:10F5F800868868460D4600F06DFA02992C482B68FB
:10F6080026F03F063604B1FBF0F0360C80B2064314
:10F61800A680228822F001021204120C2280254AB8
:10F6280093420AD85B00B1FBF3F301309BB280B27E
:10F638002084032B98BF042321E0EE884BF6FF7249
:10F64800964205D103225343B1FBF3F39BB206E084
:10F6580019225343B1FBF3F39BB243F480431A05D9
:10F668004FF4967208BF43F0010350434FF47A7287
:10F6780090FBF2F0013080B243F400432084A3836E
:10F6880023886989AA889BB243F0010323802388D1
:10F6980023F4816323F002031B040A431B0C134366
:10F6A8009BB223802A89AB8913439BB223817FBDF8
:10F6B80040420F00A086010041F288330360002316
:10F6C80083804BF6FF72038143814FF48043C280ED
:10F6D80083817047038819B19BB243F0010303E0AB
:10F6E80023F001031B041B0C03807047038819B126
:10F6F8009BB243F4807303E023F480731B041B0C58
:10F7080003807047038819B19BB243F4007303E088
:10F7180023F400731B041B0C0380704712B141F0E3
:10F72800010101E001F0FE0101827047038819B16F
:10F738009BB243F4806303E023F480631B041B0C37
:10F748000380704783899BB201F0FE0123F0FE031A
:10F758000B4383817047838919B19BB243F001033E
:10F7680003E023F001031B041B0C8381704703880B
:10F7780019B19BB243F0400303E023F040031B049C
:10F788001B0C03807047038829B16FEA43436FEA73
:10F7980053439BB201E05B045B0C03807047038812
:10F7A80019B99BB243F0800303E023F080031B04E4
:10F7B8001B0C03807047B1F5804F838B04D023F472
:10F7C80080431B041B0C02E09BB243F480438383F9
:10F7D8007047B1F5006F038803D19BB243F400630F
:10F7E80003E023F400631B041B0C03807047B1F58E
:10F7F800005F038803D19BB243F4005303E023F472
:10F8080000531B041B0C03807047038819B19BB27B
:10F8180043F0100303E023F010031B041B0C0380C8
:10F82800704701827047008AC0B27047038819B1D7
:10F838009BB243F4805303E023F480531B041B0C56
:10F8480003807047B1F5006F038803D19BB243F47E
:10F85800006303E023F400631B041B0C0380704760
:10F86800038819B19BB243F0200303E023F020037F
:10F878001B041B0C03807047008BC0F307207047E4
:10F88800838819B19BB243F4006303E023F4006357
:10F898001B041B0C83807047838819B19BB243F407
:10F8A800805303E023F480531B041B0C83807047B0
:10F8B80082B0002301930190019BCB180193019B17
:10F8C800188880B202B0704783889BB20AB1194386
:10F8D80001E023EA010181807047838A008B9BB293
:10F8E80043EA0040084020F07F40431A584240EB6A
:10F8F80003007047838A008B9BB243EA004020F0E4
:10F908007F40704782B00023009301930B0F019052
:10F918000093009B21F07F4113B1019B143302E057
:10F92800019B090C18330193019B1B6819420CBFFA
:10F938000020012002B07047C94389B28182704714
:10F948008388808A80B208409BB206D001F0E061CB
:10F9580013EA11410CBF002001207047C94389B246
:10F96800818270470A4B1A6842F001021A6000222D
:10F978009A60196821F0847121F480311960054971
:10F988005960196821F480211960DA60704700BF56
:10F998000038024010300024024B00221A70187000
:10F9A800704700BF02380240034B1A6822F0F80281
:10F9B80042EAC0021A60704700380240014B1860E2
:10F9C800704700BF00004742064B002201281A700A
:10F9D8001A7002D0042804D101E01870704705227B
:10F9E8001A70704770380240014B1860704700BFAA
:10F9F800800E4742014341EA821200995B08013BAD
:10FA080042EA016141EA0341014B5960704700BF76
:10FA180000380240014B1860704700BF6000474241
:10FA28008001034B40EA0171C3F88410704700BF9E
:10FA380000380240014B1860704700BF6800474219
:10FA4800014B1860704700BF4C004742034B9A684F
:10FA580022F0EC6202430A439A6070470038024081
:10FA6800034B9A6822F0784202430A439A6070472F
:10FA780000380240034B9A6822F0030202439A605E
:10FA8800704700BF00380240024B986800F00C0035
:10FA9800704700BF00380240034B9A6822F0F0021A
:10FAA80002439A60704700BF00380240034B9A68CF
:10FAB80022F4E05202439A60704700BF00380240C7
:10FAC800034B9A6822F4604242EAC0029A60704787
:10FAD800003802401E4B9A6802F00C02042A10B546
:10FAE80003D0082A03D01B4B18E01B4B16E05968BB
:10FAF8005A6811F4800F596814BF174B154B02F060
:10FB08003F02B3FBF2F3124A5268C2F30142C1F357
:10FB1800881101324B435200B3FBF2F30C490360E6
:10FB28008B680E4A0468C3F30313D35C34FA03F3F7
:10FB380043608C68C4F38224145D33FA04F484604F
:10FB48008968C1F34231525CD340C36010BD00BF25
:10FB5800003802400024F40000127A00B9040020A2
:10FB680000F44073B3F5407F084B08D1996820F042
:10FB7800704221F4F81122F440720A439A601A6F15
:10FB8800000542EA10501867704700BF003802406D
:10FB9800014B1860704700BF3C0E4742014B18608C
:10FBA800704700BF400E4742014B1860704700BFC6
:10FBB8005C014742044B1A6B09B1104301E022EA89
:10FBC80000001863704700BF00380240044B5A6BAE
:10FBD80009B1104301E022EA00005863704700BFF2
:10FBE80000380240044B9A6B09B1104301E022EA45
:10FBF80000009863704700BF00380240044B1A6C3D
:10FC080009B1104301E022EA00001864704700BF00
:10FC180000380240044B5A6C09B1104301E022EA53
:10FC280000005864704700BF00380240044B1A694E
:10FC380009B1104301E022EA00001861704700BFD3
:10FC480000380240044B5A6909B1104301E022EA26
:10FC580000005861704700BF00380240044B9A69A1
:10FC680009B1104301E022EA00009861704700BF23
:10FC780000380240044B1A6A09B1104301E022EA35
:10FC880000001862704700BF00380240044B5A6AEF
:10FC980009B1104301E022EA00005862704700BF32
:10FCA80000380240044B1A6D09B1104301E022EA02
:10FCB80000001865704700BF00380240044B5A6DB9
:10FCC80009B1104301E022EA00005865704700BFFF
:10FCD80000380240044B9A6D09B1104301E022EA52
:10FCE80000009865704700BF00380240044B1A6E48
:10FCF80009B1104301E022EA00001866704700BF0E
:10FD080000380240044B5A6E09B1104301E022EA60
:10FD180000005866704700BF00380240044B1A784C
:10FD280009B1104301E022EA00001870704700BFD3
:10FD38000D3802404309012B074A01D1136803E03B
:10FD4800022B0CBF136F536F00F01F0033FA00F043
:10FD580000F00100704700BF0038024007B50023DB
:10FD680001933120FFF7E6FF019B01330193019BCB
:10FD7800B3F5A06F01D00028F3D03120FFF7DAFFE8
:10FD8800003018BF01200EBD024B5A6F42F080723E
:10FD98005A67704700380240034BDB6818420CBFB3
:10FDA80000200120704700BF00380240014B187046
:10FDB800704700BF0E38024008B5154B98420BD16A
:10FDC80001214FF48050FFF761FF4FF4805000216C
:10FDD800BDE80840FFF75ABF0E4B984207D14FF4D1
:10FDE80080400121FFF746FF4FF4804009E00A4BAD
:10FDF80098420BD14FF400400121FFF73BFF4FF42D
:10FE080000400021BDE80840FFF734BF08BD00BF2F
:10FE18000030014000380040003C00400B88028858
:10FE280010B54C8823438C882343CC8823430C8902
:10FE380023434C8923438C892343CC8902F44152C0
:10FE4800234313439BB20380838B23F400631B0477
:10FE58001B0C83830B8A038210BD838B23F47B6383
:10FE680023F00F031B041B0C8383022303848B687A
:10FE7800F0B5858B022BADB238D0294A8E889468AC
:10FE8800002E14BF02260126240203D5946824F408
:10FE980000049460D2F88440D2F884705268DFF885
:10FEA80084C002F03F02BCFBF2F2C4F3881454434E
:10FEB800C7F30272B4FBF2F4CA88B2F5007F4FF0C0
:10FEC8000A0201D1240A02E07601B4FBF6F4624387
:10FED800B2FBF3F305330A229BB2B3FBF2F303F050
:10FEE80001021202C3F34F0392B200E000229C1EEB
:10FEF800A4B2FE2C28BF0022CC8828BF02231343BB
:10FF080023439BB203840B884A882B4343F4006342
:10FF180013438A8813438A8913439BB28383F0BDB2
:10FF28000038024000127A00002303804380838057
:10FF3800C380038143818381C38107230382704780
:10FF480000230222038043808380C38082608381F0
:10FF58007047038819B19BB243F0400303E023F0D4
:10FF680040031B041B0C03807047838B19B19BB2A1
:10FF780043F4806303E023F480631B041B0C838336
:10FF88007047038823F400631B041B0C0380038859
:10FF98009BB20B4303807047B1F5804F038803D1B0
:10FFA8009BB243F4804303E023F480431B041B0CFF
:10FFB800038070474FF6FF639942038803D09BB2D2
:10FFC80043F4807303E023F480731B041B0C038049
:10FFD8007047838819B19BB243F0040303E023F010
:10FFE80004031B041B0C83807047838819B19BB2E0
:08FFF80043F0100303E023F0C5
:020000040801F1
:1000000010031B041B0C83807047838B23F47B63DA
:1000100023F00F031B041B0C8383022303840B8830
:10002000828BB3F5007F10B592B205D0002B0CBFC8
:100030004FF48073002301E04FF480734C88224317
:100040008C88898942F4006222430A4392B21343A6
:10005000838310BD808980B2704781817047038897
:1000600019B19BB243F4005303E023F400531B0483
:100070001B0C0380704703889BB243F480530380BA
:100080007047012902D0008B80B27047808A80B20D
:100090007047008A80B2704783889BB20AB11943C7
:1000A00001E023EA010181807047090901238B40A7
:1000B0009BB21AB1828892B2134303E0828892B253
:1000C00022EA030383807047038919420CBF002092
:1000D00001207047C94389B20181704710B58488F7
:1000E0000089012301F00F0280B213FA02F21040DE
:1000F000A4B205D009098B401C420CBF002001208E
:1001000010BD01F00F0101238B40DB439BB2038143
:10011000704700BF08B501214FF48040FFF7BAFDDA
:100120004FF480400021BDE80840FFF7B3BD014B0C
:10013000186070470038014001F0030289080A4B3B
:10014000023130B5920053F821500F24944025EA33
:10015000040443F8214053F8214010FA02F21443FA
:1001600043F8214030BD00BF00380140014B18600A
:10017000704700BFDC002742014B1860704700BF8A
:1001800000042742024B186AC0F30020704700BFEA
:100190000038014030B5048C24F001042404240C00
:1001A0000484058B048CADB2A4B225F0F30515438D
:1001B00024F00A0445EA031544F00104ADB20C43EF
:1001C0000583048430BD30B5048C24F0100424046D
:1001D000240C0484048B058C24F44074ADB22405F3
:1001E000240D25F0A00544EA022445F0100544EA58
:1001F000033445EA0115A4B2ADB20483058430BDD1
:1002000008B5474B984205D101200146FFF742FD52
:1002100001203DE0B0F1804F05D101200146FFF7FC
:100220002DFD012076E03F4B984205D102200121AF
:10023000FFF724FD02206DE03B4B984205D10420DE
:100240000121FFF71BFD042064E0384B984205D1E3
:1002500008200121FFF712FD08205BE0344B984293
:1002600005D110200121FFF709FD102052E0314B8C
:10027000984205D120200121FFF700FD202049E010
:100280002D4B984209D102200121FFF703FD0220E6
:100290000021BDE80840FFF7FDBC284B984207D17C
:1002A0004FF480300121FFF7F5FC4FF48030EFE789
:1002B000234B984207D14FF400300121FFF7EAFCAD
:1002C0004FF40030E4E71F4B984207D14FF48020F1
:1002D0000121FFF7DFFC4FF48020D9E71A4B984249
:1002E00005D140200121FFF7C9FC402012E0174B47
:1002F000984205D180200121FFF7C0FC802009E051
:10030000134B98420BD14FF480700121FFF7B6FCDC
:100310004FF480700021BDE80840FFF7AFBC08BD76
:10032000000001400004004000080040000C0040B4
:100330000010004000140040000401400040014053
:10034000004401400048014000180040001C0040EB
:10035000002000401C4A038890429BB212D002F554
:10036000806290420ED0B0F1804F0BD0A2F5803267
:10037000904207D002F58062904203D002F580627D
:10038000904203D14A8823F0700313430F4A9042EE
:1003900008D002F58062904204D023F440730A89A9
:1003A0009BB2134303804B68C3620B880385064BE3
:1003B000984203D003F58063984201D18B7A03867B
:1003C00001238382704700BF0000014000100040FD
:1003D0004FF0FF3343600023038003814380837227
:1003E0007047018582827047038823F070031B04E5
:1003F0001B0C0B430380704741627047C16270471A
:10040000406A7047008D80B27047038819B19BB273
:1004100043F0020303E023F002031B041B0C0380E0
:100420007047038819B19BB243F0040303E023F043
:1004300004031B041B0C03807047038819B19BB293
:1004400043F0800303E023F080031B041B0C0380B4
:100450007047038823F008031B041B0C03800388E8
:100460009BB20B4303807047038823F440731B0443
:100470001B0C038003889BB20B43038070470388E7
:1004800019B19BB243F0010303E023F001031B0405
:100490001B0C03807047038C23F001031B041B0C0F
:1004A000038470B5038C8488028B0D884E8822F0FB
:1004B00073021204120C2A438D8923F002031B04D9
:1004C00035431B0CADB22B430E4DA842A4B203D052
:1004D00005F58065A8420ED1CD894E8A23F0080328
:1004E0002B438D8823F004032B430D8A354324F4DA
:1004F0004074ADB22C43848002838A6842630384D3
:1005000070BD00BF00000140038C23F010031B04EA
:100510001B0C0384038C828830B5048B0D8824F473
:10052000E6442404240C23F0200344EA05241B049D
:100530008D891B0C43EA05134D8843EA0513134DBF
:10054000A84292B2A4B29BB203D005F58065A8423E
:1005500015D1CD8923F080039BB243EA05134FF6F2
:10056000BF751D408B8845EA03130D8A22F4406253
:1005700042EA85024D8A42EA85029BB292B28280AB
:100580008A6804838263038430BD00BF0000014099
:10059000038C23F480731B041B0C0384038C82885C
:1005A00030B5848B0D8824F073042404240C23F4C8
:1005B00000731B042C438D891B0C43EA05234D88D3
:1005C00043EA0523124DA84292B29BB203D005F52F
:1005D0008065A84215D1CD8923F400639BB243EA1C
:1005E00005234FF6FF351D408B8845EA03230D8A0E
:1005F00022F4405242EA05124D8A42EA05129BB2A9
:1006000092B282808A688483C263038430BD00BF53
:1006100000000140038C23F480531B041B0C038453
:10062000038C30B58488828B0D8822F4E642120454
:10063000120C23F4005342EA05221B048D891B0C83
:1006400043EA05334D8843EA05330B4DA842A4B273
:1006500092B29BB203D005F58065A84205D10D8A00
:1006600024F4804444EA8514A4B2848082838A6896
:100670000264038430BD00BF0000014000230380FA
:100680004380838083608381C38103824382704778
:1006900030B5058C0124ADB28C4025EA040400F18C
:1006A0001803048409B1082907D149084FF68F704F
:1006B000CC582040C850C8580AE00439C1F34E0154
:1006C00048F6FF70CC582040C8501202C85892B269
:1006D0000243CA5030BD4163704781637047C163B4
:1006E000704701647047038B23F070031B041B0CDD
:1006F0000B4303837047038B23F4E0431B041B0C61
:1007000043EA01239BB203837047838B23F070037A
:100710001B041B0C0B4383837047838B23F4E04340
:100720001B041B0C43EA01239BB283837047038B9A
:1007300023F008031B041B0C0B4303837047038B3C
:1007400023F400631B041B0C43EA01239BB20383C5
:100750007047838B23F008031B041B0C0B4383831C
:100760007047838B23F400631B041B0C43EA0123B3
:100770009BB283837047038B23F004031B041B0C81
:100780000B4303837047038B23F480631B041B0C10
:1007900043EA01239BB203837047838B23F0040356
:1007A0001B041B0C0B4383837047838B23F48063F0
:1007B0001B041B0C43EA01239BB283837047038B0A
:1007C00023F080031B041B0C0B4303837047038B34
:1007D00009025B0441EA53439BB203837047838B56
:1007E00023F080031B041B0C0B4383837047838B14
:1007F00009025B0441EA53439BB283837047038C35
:1008000023F002031B041B0C0B4303847047038C6F
:1008100023F008031B041B0C0B4303847047038C59
:1008200023F020031B041B0C43EA01139BB2038437
:100830007047038C23F080031B041B0C43EA011355
:100840009BB203847047038C23F400731B041B0CBE
:1008500043EA01239BB203847047038C23F40063B3
:100860001B041B0C43EA01239BB203847047038CD7
:1008700023F400531B041B0C43EA01339BB2038493
:10088000704710B5048C01238B40A4B224EA030303
:100890000384038C12FA01F10B439BB2038410BD55
:1008A00010B5048C04238B40A4B224EA0303038410
:1008B000038C12FA01F10B439BB2038410BD002399
:1008C0000122038043808280C38003817047406B94
:1008D0007047806B7047C06B7047006C7047038B2C
:1008E00023F00C031B041B0C0383038B9BB20B43F1
:1008F00003837047038B23F440631B041B0C0383A7
:10090000038B9BB243EA01239BB203837047F8B584
:100910000C464988A288B4F800E0238905460029DE
:100920000CBF02270027012A14BF01260226BEF1B0
:10093000000F10D1FFF72EFC2846E188FFF7CFFF0C
:100940002846394632462389FFF73DFCE188284690
:10095000BDE8F840CEE7FFF736FC2846E188FFF710
:10096000C9FF2846394632462389FFF713FCE18840
:100970002846BDE8F840B2E7838B23F00C031B0444
:100980001B0C8383838B9BB20B4383837047838BC6
:1009900023F440631B041B0C8383838B9BB243EAC9
:1009A00001239BB283837047F8B50D460B88AA8854
:1009B000498804463BB92B89FFF7ECFBE9882046C0
:1009C000BDE8F8408BE7042B07D12B89FFF7FBFB31
:1009D000E9882046BDE8F8408CE7082BB5F808C048
:1009E000078C1DD127F480773F043F0C0784868B4A
:1009F000038CB6B29BB226F0F30623F4206346EADA
:100A00000C1C43EA01211FFA8CFC89B24CEA020259
:100A100041F4807182830184E988BDE8F840ABE746
:100A200027F480573F043F0C0784868B038C26F401
:100A3000407623F4005336055B04360D5B0C46EA22
:100A4000022243EA013342EA0C329BB2E98892B2B5
:100A500043F4805382830384BDE8F84097E74A88D3
:100A60000B8813438A881343CA8813430A891343A4
:100A70004A8913438A8913439BB2A0F844307047D4
:100A80000023038043808380C3800381438183816B
:100A90007047B0F8443029B16FEA43436FEA5343DB
:100AA0009BB201E05B045B0CA0F844307047838884
:100AB00019B19BB243F0040303E023F004031B04C9
:100AC0001B0C83807047838819B19BB243F00103EC
:100AD00003E023F001031B041B0C83807047838910
:100AE0009BB20AB1194301E023EA010181817047F9
:100AF00081827047038A19420CBF00200120704791
:100B0000C94389B201827047038A828911EA0300CE
:100B100092B203D011420CBF002001207047C9439C
:100B200089B2018270470A43A0F848207047838940
:100B30009BB20AB1194301E023EA010181817047A8
:100B4000838819B19BB243F0080303E023F0080344
:100B50001B041B0C83807047038923F007031B04CD
:100B60001B0C03817047038923F070031B041B0CCB
:100B70000B43038103899BB243F007030381704752
:100B800038B50D4611460122602D044602D1FFF70B
:100B90001AFB01E0FFF7FEFA238923F070031B0420
:100BA0001B0C1D43258123899BB243F0070323813E
:100BB00038BD038923F070031B041B0C0B43038116
:100BC0007047838823F070031B041B0C8380838889
:100BD0009BB20B4383807047038923F007031B04F8
:100BE0001B0C038103899BB20B430381704703896C
:100BF00023F080031B041B0C038103899BB20B436E
:100C00000381704710B50489E4B20C43144344EAED
:100C10000324A4B2048110BD10B50446FFF7F2FF0F
:100C200023899BB243F48043238110BD10B5044651
:100C3000FFF7E8FF238923F077031B041B0C43F025
:100C40007703238110BD70B50489068B058C26F4CB
:100C50004076ADB226F0030624F00704360425F0F2
:100C600022052404360C1543240C46F4807645EA0C
:100C70000315214346F00106ADB2018106830584C8
:100C800070BD838819B19BB243F0800303E023F069
:100C900080031B041B0C83807047A0F85010704722
:100CA00008B5234B984205D110200121FEF7F2FF31
:100CB000102037E01F4B984207D14FF4003001213C
:100CC000FEF7DCFF4FF4003009E01B4B98420BD1DC
:100CD0004FF480200121FEF7D1FF4FF48020002146
:100CE000BDE80840FEF7CABF144B984207D14FF445
:100CF00000200121FEF7C2FF4FF40020EFE7104B68
:100D0000984207D14FF480100121FEF7B7FF4FF44E
:100D10008010E4E70B4B984209D120200121FEF717
:100D2000B9FF20200021BDE80840FEF7B3BF08BD91
:100D3000001001400044004000480040004C0040CA
:100D40000050004000140140038ACA889BB223F47B
:100D5000405330B513430D46038283890989AA881D
:100D600023F4B0530A43698923F00C031B040A439C
:100D70001B0C92B213438381838AAA899BB223F40A
:100D80004073134385B0838204466846FEF7A6FE8F
:100D90001A4B9C4203D003F580639C4201D1039B14
:100DA00000E0029BA28912B2002A4FF019012A68C2
:100DB00001FB03F101DA520000E092006423B1FB71
:100DC000F2F1B1FBF3F21201100903FB1011A0893B
:100DD00000B2002806DAC9003231B1FBF3F303F0A8
:100DE000070305E009013231B1FBF3F303F00F0310
:100DF0001A4392B2228105B030BD00BF00100140FD
:100E00004FF4165303600C2200238380C3800381B8
:100E10004281838170470B88028A10B54C88234336
:100E20008C88C988234392B20B4322F470629BB230
:100E30001343038210BD0023038043808380C3805B
:100E40007047838919B19BB243F4005303E023F444
:100E500000531B041B0C83817047038B03F47F43F7
:100E60000383038B9BB20B4303837047838929B1B0
:100E70006FEA43436FEA53439BB201E05B045B0CB0
:100E800083817047838A19B19BB243F4006303E006
:100E900023F400631B041B0C83827047C905C90D32
:100EA000818070478088C005C00D7047038A23F099
:100EB0000F031B041B0C0382038A9BB20B430382A8
:100EC0007047838919B19BB243F0020303E023F01A
:100ED00002031B041B0C83817047838923F4006386
:100EE0001B041B0C838183899BB20B438381704756
:100EF000038A23F020031B041B0C0382038A9BB28A
:100F00000B4303827047038A19B19BB243F48043B9
:100F100003E023F480431B041B0C03827047838986
:100F20009BB243F0010383817047838A19B19BB25E
:100F300043F0080303E023F008031B041B0C838227
:100F40007047038BDBB20383038B9BB243EA01231D
:100F500003837047838A19B19BB243F0200303E0F7
:100F600023F020031B041B0C83827047838A19B172
:100F70009BB243F0100303E023F010031B041B0C8F
:100F800083827047838A23F004031B041B0C838233
:100F9000838A9BB20B4383827047838A19B19BB2C9
:100FA00043F0020303E023F002031B041B0C8382C3
:100FB0007047838A9BB20AB1194301E023EA010119
:100FC00081827047C1F3421310B501F01F01012463
:100FD00014FA01F1A34201D10C3004E0022B01D13B
:100FE000103000E0143003680AB1194301E023EA2D
:100FF0000101016010BD038819420CBF00200120CF
:101000007047C94389B201807047012210B501F0D1
:101010001F03C1F342149A40012C01D1838903E0DC
:10102000022C0CBF038A838A9BB21340028892B2BF
:1010300043B1090A012313FA01F111420CBF002048
:10104000012010BD184610BD090A01238B40DB4367
:101050009BB20380704700BF81F0004102E000BFF7
:1010600083F0004330B54FEA41044FEA430594EA68
:10107000050F08BF90EA020F1FBF54EA000C55EAA3
:10108000020C7FEA645C7FEA655C00F0E2804FEA74
:101090005454D4EB5555B8BF6D420CDD2C4480EA56
:1010A000020281EA030382EA000083EA010180EA86
:1010B000020281EA0303362D88BF30BD11F0004FD4
:1010C0004FEA01314FF4801C4CEA113102D040420A
:1010D00061EB410113F0004F4FEA03334CEA133345
:1010E00002D0524263EB430394EA050F00F0A7805D
:1010F000A4F10104D5F1200E0DDB02FA0EFC22FA58
:1011000005F2801841F1000103FA0EF2801843FA4B
:1011100005F359410EE0A5F120050EF1200E012A3C
:1011200003FA0EFC28BF4CF0020C43FA05F3C0187A
:1011300051EBE37101F0004507D54FF0000EDCF1F3
:10114000000C7EEB00006EEB0101B1F5801F1BD39C
:10115000B1F5001F0CD349085FEA30004FEA3C0CA0
:1011600004F101044FEA445212F5800F80F09A8096
:10117000BCF1004F08BF5FEA500C50F1000041EB9A
:10118000045141EA050130BD5FEA4C0C404141EB9E
:10119000010111F4801FA4F10104E9D191F0000FC5
:1011A00004BF01460020B1FA81F308BF2033A3F148
:1011B0000B03B3F120020CDA0C3208DD02F1140C3F
:1011C000C2F10C0201FA0CF021FA02F10CE002F17A
:1011D0001402D8BFC2F1200C01FA02F120FA0CFC73
:1011E000DCBF41EA0C019040E41AA2BF01EB0451BC
:1011F000294330BD6FEA04041F3C1CDA0C340EDCBA
:1012000004F11404C4F1200220FA04F001FA02F3FC
:1012100040EA030021FA04F345EA030130BDC4F1BA
:101220000C04C4F1200220FA02F001FA04F340EAAF
:101230000300294630BD21FA04F0294630BD94F060
:10124000000F83F4801306BF81F480110134013D47
:101250004EE77FEA645C18BF7FEA655C29D094EAB8
:10126000050F08BF90EA020F05D054EA000C04BF36
:101270001946104630BD91EA030F1EBF0021002021
:1012800030BD5FEA545C05D14000494128BF41F0C0
:10129000004130BD14F580043CBF01F5801130BD24
:1012A00001F0004545F0FE4141F470014FF00000AF
:1012B00030BD7FEA645C1ABF194610467FEA655C60
:1012C0001CBF0B46024650EA013406BF52EA033502
:1012D00091EA030F41F4002130BD00BF90F0000FF0
:1012E00004BF0021704730B54FF4806404F132042C
:1012F0004FF000054FF0000150E700BF90F0000FE5
:1013000004BF0021704730B54FF4806404F132040B
:1013100010F0004548BF40424FF000013EE700BFDB
:1013200042004FEAE2014FEA31014FEA02701FBF6B
:1013300012F07F4393F07F4F81F06051704792F03D
:10134000000F14BF93F07F4F704730B54FF46074B7
:1013500001F0004521F0004120E700BF50EA010202
:1013600008BF704730B54FF000050AE050EA0102AF
:1013700008BF704730B511F0004502D5404261EB1F
:1013800041014FF4806404F132045FEA915C3FF460
:10139000DCAE4FF003025FEADC0C18BF03325FEAF9
:1013A000DC0C18BF033202EBDC02C2F1200300FAAE
:1013B00003FC20FA02F001FA03FE40EA0E0021FAD3
:1013C00002F11444C1E600BF70B54FF0FF0C4CF4BD
:1013D000E06C1CEA11541DBF1CEA135594EA0C0F73
:1013E00095EA0C0F00F0DEF82C4481EA030621EAAE
:1013F0004C5123EA4C5350EA013518BF52EA0335E9
:1014000041F4801143F4801338D0A0FB02CE4FF09A
:101410000005E1FB02E506F00042E0FB03E54FF0CA
:101420000006E1FB03569CF0000F18BF4EF0010EC2
:10143000A4F1FF04B6F5007F64F5407404D25FEABE
:101440004E0E6D4146EB060642EAC62141EA555171
:101450004FEAC52040EA5E504FEACE2EB4F1FD0CB3
:1014600088BFBCF5E06F1ED8BEF1004F08BF5FEA31
:10147000500E50F1000041EB045170BD06F00046E3
:1014800046EA010140EA020081EA0301B4EB5C0490
:10149000C2BFD4EB0C0541EA045170BD41F4801188
:1014A0004FF0000E013C00F3AB8014F1360FDEBFAD
:1014B000002001F0004170BDC4F10004203C35DA89
:1014C0000C341BDC04F11404C4F1200500FA05F30C
:1014D00020FA04F001FA05F240EA020001F00042AD
:1014E00021F0004110EBD37021FA04F642EB060123
:1014F0005EEA430E08BF20EAD37070BDC4F10C044D
:10150000C4F1200500FA04F320FA05F001FA04F210
:1015100040EA020001F0004110EBD37041F10001FC
:101520005EEA430E08BF20EAD37070BDC4F1200507
:1015300000FA05F24EEA020E20FA04F301FA05F26F
:1015400043EA020321FA04F001F0004121FA04F217
:1015500020EA020000EBD3705EEA430E08BF20EAE7
:10156000D37070BD94F0000F0FD101F00046400021
:1015700041EB010111F4801F08BF013CF7D041EAA3
:10158000060195F0000F18BF704703F000465200A7
:1015900043EB030313F4801F08BF013DF7D043EA78
:1015A0000603704794EA0C0F0CEA135518BF95EA2E
:1015B0000C0F0CD050EA410618BF52EA4306D1D1B5
:1015C00081EA030101F000414FF0000070BD50EAD4
:1015D000410606BF1046194652EA430619D094EA5E
:1015E0000C0F02D150EA013613D195EA0C0F05D148
:1015F00052EA03361CBF104619460AD181EA03019C
:1016000001F0004141F0FE4141F470014FF0000053
:1016100070BD41F0FE4141F4780170BD70B54FF0EE
:10162000FF0C4CF4E06C1CEA11541DBF1CEA13556E
:1016300094EA0C0F95EA0C0F00F0A7F8A4EB050450
:1016400081EA030E52EA03354FEA013100F0888047
:101650004FEA03334FF0805545EA131343EA126310
:101660004FEA022245EA111545EA10654FEA0026C5
:101670000EF000419D4208BF964244F1FD0404F57E
:10168000407402D25B084FEA3202B61A65EB0305DA
:101690005B084FEA32024FF480104FF4002CB6EB97
:1016A000020E75EB030E22BFB61A754640EA0C0017
:1016B0005B084FEA3202B6EB020E75EB030E22BF57
:1016C000B61A754640EA5C005B084FEA3202B6EB98
:1016D000020E75EB030E22BFB61A754640EA9C0057
:1016E0005B084FEA3202B6EB020E75EB030E22BF27
:1016F000B61A754640EADC0055EA060E18D04FEAE5
:10170000051545EA16754FEA06164FEAC30343EA84
:1017100052734FEAC2025FEA1C1CC0D111F4801F51
:101720000BD141EA00014FF000004FF0004CB6E74A
:1017300011F4801F04BF01430020B4F1FD0C88BFE9
:10174000BCF5E06F3FF6AFAEB5EB030C04BFB6EBF4
:10175000020C5FEA500C50F1000041EB045170BDE7
:101760000EF0004E4EEA113114EB5C04C2BFD4EB14
:101770000C0541EA045170BD41F480114FF0000E98
:10178000013C90E645EA060E8DE60CEA135594EA14
:101790000C0F08BF95EA0C0F3FF43BAF94EA0C0F17
:1017A0000AD150EA01347FF434AF95EA0C0F7FF48C
:1017B00025AF104619462CE795EA0C0F06D152EAE0
:1017C00003353FF4FDAE1046194622E750EA4106C4
:1017D00018BF52EA43067FF4C5AE50EA41047FF4D5
:1017E0000DAF52EA43057FF4EBAE12E74FF0FF3C3A
:1017F00006E000BF4FF0010C02E000BF4FF0010C0B
:101800004DF804CD4FEA410C7FEA6C5C4FEA430C83
:1018100018BF7FEA6C5C1BD001B050EA410C0CBFD2
:1018200052EA430C91EA030F02BF90EA020F002034
:10183000704710F1000F91EA030F58BF994208BF9B
:1018400090422CBFD8176FEAE37040F00100704758
:101850004FEA410C7FEA6C5C02D150EA013C07D1AF
:101860004FEA430C7FEA6C5CD6D152EA033CD3D0FA
:101870005DF8040B704700BF8446104662468C46F4
:101880001946634600E000BF01B5FFF7B7FF002827
:1018900048BF10F1000F01BD4DF808EDFFF7F4FF50
:1018A0000CBF012000205DF808FB00BF4DF808EDDB
:1018B000FFF7EAFF34BF012000205DF808FB00BFFE
:1018C0004DF808EDFFF7E0FF94BF012000205DF820
:1018D00008FB00BF4DF808EDFFF7CEFF94BF0120D5
:1018E00000205DF808FB00BF4DF808EDFFF7C4FFCE
:1018F00034BF012000205DF808FB00BF4FEA410221
:1019000012F5001215D211D56FF47873B3EB625251
:1019100012D94FEAC12343F0004343EA505311F078
:10192000004F23FA02F018BF404270474FF000000A
:10193000704750EA013005D111F0004008BF6FF048
:10194000004070474FF00000704700BF4A0011D2BE
:1019500012F5001211D20DD56FF47873B3EB625209
:101960000ED44FEAC12343F0004343EA505323FA15
:1019700002F070474FF00000704750EA013002D18A
:101980004FF0FF3070474FF0000070474FEA4102C0
:10199000B2F1E04324BFB3F5001CDCF1FE5C0DD9CD
:1019A00001F0004C4FEAC0024CEA5070B2F1004F17
:1019B00040EB830008BF20F00100704711F0804F1A
:1019C00021D113F13872BCBF01F00040704741F4DF
:1019D00080114FEA5252C2F11802C2F1200C10FAE3
:1019E0000CF320FA02F018BF40F001004FEAC123C7
:1019F0004FEAD32303FA0CFC40EA0C0023FA02F36B
:101A00004FEA4303CCE77FEA625307D150EA013340
:101A10001EBF4FF0FE4040F44000704701F0004010
:101A200040F0FE4040F40000704700BF80F00040EE
:101A300002E000BF81F0004142001FBF5FEA4103A6
:101A400092EA030F7FEA226C7FEA236C6AD04FEAA6
:101A50001262D2EB1363C1BFD218414048404140EB
:101A6000B8BF5B42192B88BF704710F0004F40F49D
:101A7000000020F07F4018BF404211F0004F41F4B9
:101A8000000121F07F4118BF494292EA030F3FD085
:101A9000A2F1010241FA03FC10EB0C00C3F1200398
:101AA00001FA03F100F0004302D5494260EB400027
:101AB000B0F5000F13D3B0F1807F06D340084FEA92
:101AC000310102F10102FE2A51D2B1F1004F40EB87
:101AD000C25008BF20F0010040EA030070474900EF
:101AE00040EB000010F4000FA2F10102EDD1B0FABA
:101AF00080FCACF1080CB2EB0C0200FA0CF0AABFAF
:101B000000EBC25052421843BCBFD040184370474C
:101B100092F0000F81F4000106BF80F40000013252
:101B2000013BB5E74FEA41037FEA226C18BF7FEA29
:101B3000236C21D092EA030F04D092F0000F08BF6B
:101B40000846704790EA010F1CBF0020704712F052
:101B50007F4F04D1400028BF40F00040704712F191
:101B600000723CBF00F50000704700F0004343F0F6
:101B7000FE4040F4000070477FEA226216BF08462C
:101B80007FEA23630146420206BF5FEA412390EAEF
:101B9000010F40F4800070474FF0000304E000BFE5
:101BA00010F0004348BF40425FEA000C08BF704796
:101BB00043F0964301464FF000001CE050EA01025A
:101BC00008BF70474FF000030AE000BF50EA01026F
:101BD00008BF704711F0004302D5404261EB41015C
:101BE0005FEA010C02BF84460146002043F0B64381
:101BF00008BFA3F18053A3F50003BCFA8CF2083AA6
